:100000000C94E9080C9408090C9408090C949C09B8
:100010000C94D2090C9408090C9408090C94080952
:100020000C9408090C9408090C9408090C9408090C
:100030000C9408090C9408090C9408090C94F20C0F
:100040000C9408090C9408090C9408090C940809EC
:100050000C94D26A0C9483620C9408090C940809DD
:100060000C9408090C9458630C9408090C944C6384
:100070000C9408090C9408090C9408090C940809BC
:100080000C9405760C9408090C9408090C94080942
:100090000C9496630C9408090C948A630C940809D8
:1000A0000C9408090C9408090C9408090C9408098C
:1000B0000C9408090C9408090C9408090C9408097C
:1000C0000C9408090C9408090C9408090C9408096C
:1000D0000C9408090C9408090C9408090C9408095C
:1000E0000C9408090C948B6A0C94956A0C94816AA0
:1000F0000C94416A0C94C66A0C94B76A0C94AB6A6F
:100100000C949F6A0C9408090C9408090C94080933
:100110000C9408090C9408090C9408090C9408091B
:100120003E7F5D7FDC7FCB80EB800B811381C080C5
:10013000084AD73B3BCE016E84BCBFFDC12F3D6C4E
:1001400074319ABD56833DDA3D00C77F11BED9E4B4
:10015000BB4C3E916BAAAABE000000803F076342E1
:1001600036B79BD8A71A39685618AEBAAB558C1D4E
:100170003CB7CC5763BD6DEDFD753EF6177231BFD0
:10018000000000803F08000000BE922449123EABF0
:10019000AAAA2ABECDCCCC4C3E00000080BEABAAA1
:1001A000AAAA3E00000000BF000000803F0000003F
:1001B0000000084178D3BB4387D1133D190E3CC3DF
:1001C000BD4282AD2B3E68EC8276BED98FE1A93E5E
:1001D0004C80EFFFBE01C4FF7F3F00000000002500
:1001E000730A005854414C5F5452494D3D256400F8
:1001F00025730A0025730A00546573742036202580
:10020000730A005465737420352025730A00546501
:10021000737420342025730A0054657374203320CE
:1002200025730A005465737420322025730A005424
:1002300065737420312025730A006368616E3D2563
:10024000640A0074787077723D25640A0035303096
:100250006B0A003235306B0A003131356B0A0035DC
:10026000366B0A0033386B0A0025730A00765F6C20
:100270006F773D252D332E32660A0025730A0073F1
:10028000656E743D252D75206475703D252D752096
:1002900069676E6F7265643D252D752074746C5F9F
:1002A0007A65726F3D252D750A0025372E3366203D
:1002B00025372E33660025352E32662000457272B2
:1002C0006F72203020566F6C74004E6F74207375FF
:1002D00070706F727465640A004572726F722030BC
:1002E00020566F6C74004572726F72203020566F0A
:1002F0006C740025630074746C3D252D64200074BB
:10030000746C3D252D6420004E65772074746C3D1F
:10031000252D6420002563004D53353631312050A2
:100320003D252D372E326620252D372E32666D0A5B
:1003300000424D5030383520256C6420506120201B
:10034000252D372E32666D00256300545F484541E8
:10035000545F4944583D252D352E32662000545FA8
:100360004445573D252D352E3266200041483D2518
:100370002D352E32662000545F53485432583D25A7
:100380002D352E3266200052485F53485432583D76
:10039000252D352E32662000545F52483D252D34E0
:1003A0002E3166200052483D252D342E3166200026
:1003B0002563002563002563002563002563007223
:1003C00065706F72745F616C6C3D007265706F7206
:1003D000743D00256300256300256300256300202C
:1003E0004F534343414C3D256420002046757365BF
:1003F0003A2065653D253032782068663D253032EB
:1004000078206C663D25303278206C623D25303294
:1004100078004D43553D2530366C780025630074D7
:10042000785F6C656E3D252D6C752C765F6C6F77F3
:100430003D252D6C752C73687432783D252D6C75B7
:100440000A002563004F4B0A002563002563002541
:100450006300256300256300256300256300256391
:100460000064656275675F616C6C3D006465627510
:10047000673D0064656275673D0025730A00646529
:1004800065700A006E6F6E650A00707772733D00CA
:10049000696E74725F7365635F70313D252D372E11
:1004A00033660A00696E74725F70313D252D6C648D
:1004B0000A00696E74725F7365635F70303D252D4D
:1004C000372E33660A00696E74725F70303D252DD9
:1004D0006C640A00765F6D63753D252D352E32669E
:1004E0000A00745F6D63753D252D352E32660A0056
:1004F000707077723D25730A0064656275673D0010
:1005000072636D643D25730A0025730A006175747A
:100510006F0A006C6F675F6D6F64653D0075736295
:100520005F7077723D25730A0072656C61793D25B5
:10053000730A0074746C3D252D640A0052494D45C0
:100540005F616464723D252D642E252D640A006E62
:1005500065696768626F725F7461626C655F736919
:100560007A653D25640A00765F6C6F773D252D33F3
:100570002E32660A00747870773D25640A0063683D
:10058000616E3D25640A006932633D0069643D0087
:100590007478743D25730A0053797374656D205324
:1005A000756D6D6172790A006D61736B3D002C0091
:1005B000696E74657276616C3D252D750023252D5D
:1005C000642C00745F686561745F69647800745FAF
:1005D00064657700616800705F6D73353631310096
:1005E00072685F736874327800745F73687432780D
:1005F0000070610070006164340061643300616404
:100600003200616431006133006132006131007693
:100610005F696E0072680065727200757074696D52
:10062000650070315F6C73740070315F74007031FD
:100630000070305F6C73740070305F740070300055
:10064000765F6D637500745F6D637500743100745F
:100650000069640065363400747874002D002B0046
:100660006175746F006E6F6E6500706F7765725F95
:10067000736176655F6C656472790072656C61792F
:100680005F6C65647900636F6D70617373006163A3
:1006900063656C007072657300705F7077720061E3
:1006A00065730070315F6C6564790070305F6C65F4
:1006B0006472006576656E74006C6564006F770027
:1006C000706B740074785F6C6564790072785F6C2D
:1006D000656472006F706572006E6F6E6500253024
:1006E000327800765F6164343D252D382E36660001
:1006F0002000765F6164333D252D382E366600205C
:1007000000765F6164323D252D382E36660020006C
:10071000765F6164313D252D382E366600200076E7
:100720005F6C696768743D252D382E3666002000A1
:10073000765F61323D252D372E3366002000765FCF
:1007400061313D252D372E3366002000765F696EBE
:100750003D252D352E326600204E657665722D754D
:1007600073656420737461636B203E20256420628E
:10077000797465730A00757074696D653D252D6423
:100780002D646179732D253032643A253032643A14
:10079000253032642D686F7572730A007465737446
:1007A000205B6F66667C317C327C337C347C355DCB
:1007B00020202020202020202D2074657374206D9F
:1007C0006F6465730A0D007478205B706B74207021
:1007D00061796C6F61645D20202020202020202022
:1007E0002020202D2073656E6420726164696F2063
:1007F000706B74206B6579626F6172640A0D0077AB
:100800006474205B6F6E7C6F66667C746573745D68
:1008100020202020202020202020202D20776174DF
:100820006368646F670A0D00765F6C6F77205B7694
:100830005F6C6F775D20202020202020202020204A
:10084000202020202D206C6F7765737420726570D6
:100850006F727420766F6C746167650A0D00757035
:1008600067722020202020202020202020202020EF
:10087000202020202020202020202D207265626F43
:100880006F742076696120626F6F746C6F6164654C
:10089000720A0D0075617274205B33386B7C3536DB
:1008A0006B7C3131356B7C3235306B7C3530306B65
:1008B0005D202D20736574207465726D2F756172D3
:1008C000742073706565640A0D00626F6F74202078
:1008D0002020202020202020202020202020202018
:1008E0002020202020202D207265626F6F740A0D59
:1008F0000070777273205B646565707C6E6F6E65E7
:100900005D2020202020202020202020202D206D50
:10091000637520736C656570206D6F64650A0D00EA
:100920007265737420656570726F6D2020202020C1
:100930002020202020202020202020202D20726513
:1009400073746F726520656570726F6D0A0D00704B
:10095000707772205B6F6E7C6F66665D2020202052
:1009600020202020202020202020202D2070726F89
:100970006772616D6D61626C65207077720A0D003F
:10098000747874205B737472696E675D2020202018
:100990002020202020202020202020202D205365D2
:1009A00074207265706F727420746578742073742B
:1009B00072696E670A0D0074787077205B31352D8F
:1009C000305D2020202020202020202020202020DA
:1009D0002020202D205458205077722E20486967FF
:1009E00068657374203020283364426D290A0D0035
:1009F00074746C205B302D31355D20202020202048
:100A00002020202020202020202020202D2074693C
:100A10006D652D746F2D6C69766520666F72207020
:100A200061636B6574730A0D0073732020202020AE
:100A300020202020202020202020202020202020B6
:100A400020202020202D2073797374656D2073750C
:100A50006D6D6172790A0D007273202020202020B4
:100A60002020202020202020202020202020202086
:100A7000202020202D20726164696F2073746174BE
:100A8000730A0D007269205B236E5D205B696E74D2
:100A90005D20202020202020202020202020202019
:100AA0002D207265706F727420696E746572766144
:100AB0006C0A0D0072636D64205B6F6E7C6F6666FE
:100AC0005D202020202020202020202020202020E9
:100AD0002D20616C6C6F7720636D642066726F6D82
:100AE000206E65746F726B0A0D007265205B236E59
:100AF0005D205B2B7C2D5D205B6D61736B7C617574
:100B0000746F2C6D61736B5D202D206D6F7465208B
:100B10007265706F7274207365742F6D6F6469668F
:100B2000790A0D006F77202020202020202020200F
:100B300020202020202020202020202020202020B5
:100B40002D206F6E652D776972652073656E736FEA
:100B500072730A0D006C6F67205B6175746F7C6F38
:100B60006E7C6F66665D20202020202020202020C3
:100B7000202D206D6F7465732064617461206F6E29
:100B8000205553420A0D006E65205B666C757368D4
:100B90005D20202020202020202020202020202018
:100BA0002020202D206E65696768626F7220746155
:100BB000626C650A0D0065727220202020202020C2
:100BC0002020202020202020202020202020202025
:100BD00020202D206572726F722073746174730A05
:100BE0000D006D6375202020202020202020202053
:100BF00020202020202020202020202020202D20E8
:100C00006D637520696E666F0A0D006964205B7202
:100C1000657365745D202020202020202020202066
:100C2000202020202020202D2069642068616E640F
:100C30006C696E670A0D0068756D202020202020E9
:100C400020202020202020202020202020202020A4
:100C50002020202D2068756D696469747920736582
:100C60006E736F720A0D0072656C6179205B6F6E36
:100C70007C6F66667C73746174735D202020202015
:100C80002020202D2072656C6179206E6574776F4D
:100C9000726B207265706F7274730A0D0064652048
:100CA0005B6D61736B5D20202020202020202020A0
:100CB0002020202020202020202D206465627567C0
:100CC0000A0D006368616E205B31312D32365D2084
:100CD0002020202020202020202020202020202D07
:100CE000206368616E2031312D32362028322E3457
:100CF00030352D32343830204D687A290A0D0063A2
:100D0000616C69205B5B765F696E7C61317C61320E
:100D10005D20766F6C747C72657365747C6E6F6E2B
:100D2000655D202D2063616C6962726174650A0DD6
:100D3000006164632020202020202020202020200B
:100D4000202020202020202020202020202D207343
:100D5000686F7720765F696E2C2061312C206132BC
:100D600020766F6C74616765730A0D007520202012
:100D70002020202020202020202020202020202073
:100D800020202020202020202D20757074696D6582
:100D90000A0D007620202020202020202020202046
:100DA0002020202020202020202020202020202D36
:100DB0002076657273696F6E0A0D0068202020200E
:100DC0002020202020202020202020202020202023
:100DD000202020202020202D2068656C700A0D0026
:100DE000256300756E6B6E6F776E20636D640A000D
:100DF000484D4335383833002573002573002025CE
:100E000073002025362E326620002530327800749B
:100E1000656D705F65787465726E3D252D362E3276
:100E20006600202573002025362E3266204F6E2D59
:100E3000426F61726400253032780074656D705FB6
:100E4000626F6172643D252D362E3266000A0050B5
:100E50003A20256C642050612020252D372E3266E3
:100E6000206D0A002563002563004932433A2000C3
:100E7000452025642E256420636C6F636B20256CF0
:100E8000752063707520256C75206C706D20256C45
:100E9000752069727120256C7520676C656420254A
:100EA0006C7520796C656420256C7520726C6564A6
:100EB00020256C7520747820256C75206C697374FE
:100EC000656E20256C752073656E736F72732025B7
:100ED0006C752073657269616C20256C750A00530E
:100EE0002025642E256420636C6F636B20256C7550
:100EF00020747820256C7520727820256C752072FE
:100F0000747820256C752072727820256C7520729B
:100F100065786D697420256C752061636B74782029
:100F2000256C75206E6F61636B747820256C75205D
:100F300061636B727820256C752074696D65646FD0
:100F4000757420256C752062616461636B72782012
:100F5000256C7520746F6F6C6F6E6720256C752023
:100F6000746F6F73686F727420256C752062616492
:100F700073796E636820256C7520626164637263A7
:100F800020256C7520636F6E74656E74696F6E6476
:100F9000726F7020256C752073656E64696E67646E
:100FA000726F7020256C75206C6C747820256C75C0
:100FB000206C6C727820256C750A00257325730AE5
:100FC000004F6E6C696E650A000A002C206368652C
:100FD000636B207261746520257520487A00257343
:100FE0002025732C206368616E6E656C202575204A
:100FF000706F776572202575000A0025783A004DDC
:1010000041432061646472657373200052616E64B1
:101010006F6D204555493634206164647265737381
:101020002067656E6572617465640A000A2A2A2A5F
:101030002A2A2A2A426F6F74696E672025732A2A2A
:101040002A2A2A2A2A0A00454550524F4D20697300
:1010500020636F72727570742C2072657772697478
:10106000696E6720776974682064656661756C7461
:10107000732E0A006C6F63616C686F737400415467
:101080004D4547413132387266613100020000FF40
:10109000FE0000016E616E00696E660000407A100D
:1010A000F35A00A0724E18090010A5D4E80000E819
:1010B0007648170000E40B54020000CA9A3B000077
:1010C00000E1F505000080969800000040420F0006
:1010D0000000A08601000000102700000000E803C7
:1010E000000000006400000000000A000000000092
:1010F0000100000000002C76D888DC674F0823DF51
:10110000C1DFAE59E1B1B796E5E3E453C63AE65123
:10111000997696E8E6C28426EB898C9B62ED407C4A
:101120006FFCEFBC9C9F40F2BAA56FA5F490055AE6
:101130002AF75C936B6CF9676DC11BFCE0E40D470B
:10114000FEF520E6B500D0ED902E0300943577052E
:101150000080841E080000204E0A000000C80C33E6
:101160003333330F986E12831141EF8D2114893B75
:10117000E65516CFFEE6DB18D1844B381BF77C1DF5
:10118000901DA4BBE424203284725E228100C9F148
:1011900024ECA1E53D274E414E494E495459494E54
:1011A00046CDCCCC3D0AD7233C17B7D13877CC2BD2
:1011B000329595E6241FB14F0A000020410000C877
:1011C0004200401C4620BCBE4CCA1B0E5AAEC59DF8
:1011D000740011241FBECFEFD1E4DEBFCDBF19E0F4
:1011E000A0E0B2E0E4E0F8E201E00BBF02C007904B
:1011F0000D92A83AB107D9F711E3A8EAB9E001C006
:101200001D92AD35B107E1F70E94E2810C94009484
:101210000C9400008AE894E09F938F930E94D990E9
:101220008091540290915502A0915602B0915702BC
:101230000F900F9093FF03C084E894E002C08EE704
:1012400094E09F938F930E94D9900F900F900895F0
:10125000E091611BEF71F0E0EA54F44E80838091DD
:10126000611B8F5F8093611B8091972888608093BA
:1012700097284EE352E061E1CA010E94725280E079
:1012800090E00895CF93DF93EC018091AF099091A6
:10129000B00986FF1DC08E811F928F938D811F9292
:1012A0008F938C811F928F938B811F928F938A8152
:1012B0001F928F9381E693E09F938F930E94C79034
:1012C0008DB79EB70C960FB6F8949EBF0FBE8DBF1C
:1012D000BE0186EE99E00E94A453BE0184E092E034
:1012E000DF91CF910C94195387EE93E0811591050E
:1012F00011F00197F1F708958823B9F052985A98A0
:101300001DBA80916900806280936900EA9A5398BF
:101310005B98EB9A80916900806880936900809166
:1013200068008160809368000895109269005A9A5D
:10133000EA985B9AEB9808951F920F920FB60F925E
:1013400011248F939F93AF93BF938091680080FF88
:1013500020C08091722890917328A0917428B09138
:1013600075280196A11DB11D809372289093732852
:10137000A0937428B09375288091AF099091B0091B
:1013800087FF07C0749882E090E090938102809379
:101390008002BF91AF919F918F910F900FBE0F90E0
:1013A0001F9018951F920F920FB60F9211248F93D2
:1013B0009F93AF93BF938091680080FF20C080917E
:1013C000762890917728A0917828B0917928019675
:1013D000A11DB11D8093762890937728A09378283B
:1013E000B09379288091AF099091B00990FF07C020
:1013F000739882E090E09093810280938002BF9185
:10140000AF919F918F910F900FBE0F901F901895E5
:1014100080937C0080917B00877F80937B0080910C
:101420007C00806C80937C0085E080937A008091C2
:101430007A00806880937A0080917B0087FFFCCFE0
:1014400080917B0085FFFCCF80917A00806480933F
:101450007A0080917A0086FDFCCF1092790010927C
:10146000780084E090E060E070E020917A002064F1
:1014700020937A0020917A0026FDFCCF20917800FD
:1014800030917900620F731F0197009771F71092E6
:101490007C0080917A008F7780937A0076956795AB
:1014A0007695679580E090E00E943887089580E007
:1014B0000E94080A209178023091790240917A02C4
:1014C00050917B020E94188921EE3AE744E95EE3DD
:1014D0000E94D185089580E18093510160E160937D
:1014E00051018091510185FF03C06F5F6F31B9F7E2
:1014F0008BE4689FB0011124882777FD8095982F91
:101500000E943A8720E030E64FE954E40E94D185FA
:1015100020E030E04AE754E40E949B860895CF9390
:10152000DF93EC0188819981009799F08432904192
:1015300021F01982188283E011C0623171F40E9497
:101540006B0A6093092470930A2480930B24909370
:101550000C2484E290E19983888381E0DF91CF912C
:10156000089580917B00886080937B0089EC809354
:101570007C0085E080937A0080917A008068809377
:101580007A0080917B0087FFFCCF80917B0085FFF4
:10159000FCCF80917A00806480937A0080917A00F9
:1015A00086FDFCCF80917A00806480937A008091E0
:1015B0007A0086FDFCCF609178007091790080916F
:1015C0007A008F7780937A0080E090E00E943887DD
:1015D00027ED33EA40E95FE30E94188926E636E604
:1015E00048E853E40E94D0850895BF92CF92DF92DD
:1015F000EF92FF920F931F93CF93DF93CDB7DEB798
:1016000029970FB6F894DEBF0FBECDBF6C011092C4
:10161000A8098FEF898702E71BE1B12C7E0189E0E1
:10162000E80EF11C89858823E9F1E8E0BE16E1F1B6
:10163000BE016F5F7F4FC7010E940D5C89858F3FA0
:1016400011F08E3F19F48093A8092CC0CE010196A9
:10165000C114D10471F40E94265C80939428FE0189
:101660003196ACE8B8E281918D93EE15FF05D9F77C
:101670001DC00E94265CF8018083FE01319620E0A7
:1016800030E0A801485051098191DA01A20FB31F3F
:101690008C932F5F3F4F28303105B1F7B394075F2C
:1016A0001F4FC0CF8B2D03C088E001C081E0299679
:1016B0000FB6F894DEBF0FBECDBFDF91CF911F9163
:1016C0000F91FF90EF90DF90CF90BF9008958DE441
:1016D0009EE09F938F930E94D9900F900F90089552
:1016E0002F923F924F925F926F927F928F929F9232
:1016F000AF92BF92CF92DF92EF92FF920F931F9320
:10170000CF93DF93EC014B01009711F427E004C065
:101710008130910549F426E04AE250E06BE270E046
:1017200089E290E00E94ED5ACE010E94F50A9E01E6
:101730002755364F5901D9018C93CD2B69F092E78B
:10174000C92E9BE1D92ECAE6DBE1E12CF12C2EEF6C
:10175000222E2DE0322EA6C08CE898E20E945B5D1E
:10176000BC01882777FD8095982F0E943A876B01EE
:101770007C01892869F020E030E048EC52E40E94C6
:101780009B869F938F937F936F938BE39EE0ACC078
:10179000CCE8D8E206E31EE089911F928F931F9355
:1017A0000F930E94D9900F900F900F900F90B8E276
:1017B000C439DB0789F720E030E048EC52E4C70188
:1017C000B6010E949B869F938F937F936F9386E2CF
:1017D0009EE09F938F930E94D9900F900F900F904F
:1017E0000F900F900F9080919428882319F080E932
:1017F00093E002C084E094E09F938F9382E29EE0A6
:101800009F938F930E94D9900F900F900F900F90FD
:1018100075C000E010E0FE01E00FF11F80811F9213
:101820008F93AAE0BEE0BF93AF930E94D9900F5F61
:101830001F4F0F900F900F900F900830110559F720
:1018400020E030E048EC52E4C301B2010E949B86E4
:101850009F938F937F936F93A2E0BEE0BF93AF936C
:101860000E94D9900F900F900F900F900F900F90B3
:10187000D6018C91882309F455C080E993E09F93A9
:101880008F933F922F920E94D9900E94670BBFEFD7
:10189000EB1AFB0AE9E0CE0ED11C29960F900F90AF
:1018A0000F900F90D5018C9190E0E816F906ECF5B9
:1018B000CE010E945B5DBC01882777FD8095982F43
:1018C0000E943A872B013C018114910409F4A1CFB5
:1018D00020E030E048EC52E40E949B869F938F9377
:1018E0007F936F938FE09EE09F938F930E94D99098
:1018F0000F900F900F900F900F900F90DF91CF915E
:101900001F910F91FF90EF90DF90CF90BF90AF901D
:101910009F908F907F906F905F904F903F902F900F
:101920000C94670B84E094E0AACFDF91CF911F91D4
:101930000F91FF90EF90DF90CF90BF90AF909F906E
:101940008F907F906F905F904F903F902F90089571
:10195000CF93DF9300D0CDB7DEB780918D288983F8
:10196000809193288A83CE0101960E9466500F9041
:101970000F90DF91CF910895CF93DF93EC012091E9
:101980008C2830918D2840918E2850918F2860911D
:101990009028709191288091922890919328AFEF90
:1019A0000E94488CE1F427E04AE250E06BE270E0EC
:1019B00089E290E00E94ED5A80E090E00E94F50AF2
:1019C000C755D64F888349E050E06AE070E08CE864
:1019D00098E20E944B92DF91CF910C94A80CDF917A
:1019E000CF9108951F920F920FB60F9211240BB64C
:1019F0000F92DF92EF92FF920F931F932F933F93DB
:101A00004F935F936F937F938F939F93AF93BF9306
:101A1000CF93DF93EF93FF93809197288260809319
:101A200097288091540286FD2B9A8091540287FD5D
:101A30002B9A80918002909181021816190614F455
:101A4000749A739A8091AF099091B00985FF02C092
:101A50007498739880910202909103020197909379
:101A6000030280930202892B09F03DC18091BD09D8
:101A70009091BE0901969093BE098093BD09809113
:101A80000D2490910E24A0910F24B0911024019662
:101A9000A11DB11D80930D2490930E24A0930F24BB
:101AA000B093102480E190E09093030280930202AF
:101AB0008091540280FD02C01D9B07C01092AD09A9
:101AC0001092AC0983B7817F09C081E090E09093C8
:101AD000AD098093AC0983B7817F866083BF809115
:101AE000AF099091B00997FF08C08091AC0990911F
:101AF000AD09892B61F0749A739801E11BE1CEE185
:101B0000D4E234E0E32EF12CDD24D3941FC0739A89
:101B10007498F3CF8091BD099091BE0901960E94FF
:101B2000198A892BD1F0F8016085718561157105DD
:101B300009F5F801608571856115710569F5065F24
:101B40001F4F2596FBE109331F07D1F1F80160858E
:101B500071856115710539F3DDCF77988091AF09F3
:101B60009091B00992FFDFCF7498F0928102E092D9
:101B70008002D9CF8091BD099091BE0901960E9443
:101B8000198A892BB1F61C821B82AE0162E186E1C3
:101B900092E00E947252CDCF8091BD099091BE0912
:101BA0000E94198A892B59F6D8821A8309831C82CC
:101BB0001B82AE0162E184E392E00E947252BFCFC9
:101BC00060915A0270915B0261157105A1F18091DB
:101BD000BD099091BE090E94198A892B61F58091F7
:101BE000722890917328A0917428B0917528409123
:101BF000FF1B5091001C6091011C7091021C841B02
:101C0000950BA60BB70B8093391B90933A1BA093AF
:101C10003B1BB0933C1B8091722890917328A0913C
:101C20007428B09175288093FF1B9093001CA0939B
:101C3000011CB093021C6091580270915902611509
:101C40007105A1F18091BD099091BE090E94198A88
:101C5000892B61F58091762890917728A09178283A
:101C6000B09179284091031C5091041C6091051C8F
:101C70007091061C841B950BA60BB70B80933D1B24
:101C800090933E1BA0933F1BB093401B80917628FE
:101C900090917728A0917828B09179288093031C9F
:101CA0009093041CA093051CB093061C80915402D1
:101CB00086FD2B988091540290915502A091560276
:101CC000B091570291FF0FC00E94FD668A3119F052
:101CD000C1E0C80F01C0CBE00E94B7658C2F0E9405
:101CE00015670E94FF6540E050E060E082E892E006
:101CF0000E947252FF91EF91DF91CF91BF91AF910E
:101D00009F918F917F916F915F914F913F912F9113
:101D10001F910F91FF90EF90DF900F900BBE0F90EF
:101D20000FBE0F901F9018958091611B90911D24FC
:101D3000891B08950E94940E882371F0E0911D2460
:101D4000EF71F0E0EA54F44E808190E020911D2480
:101D50002F5F20931D2408958FEF9FEF0895CF9359
:101D6000DF93EC011092DA091092D90988819981E8
:101D70000097C1F08F36934021F01982188283E0DA
:101D8000B6C0613109F0B2C0F89478940E949A0EFE
:101D900099279093D5098093D4098D3009F441C0D7
:101DA0008F3F49F40E94940E8111EECF8FE693E0AD
:101DB000998388839BC08231910509F458C08F377D
:101DC000910509F050C08091D2099091D30918165D
:101DD00019060CF5609157317091583188E090E008
:101DE0000E949590609157317091583180E290E057
:101DF0000E949590609157317091583188E090E041
:101E00000E9495908091D2099091D3090197909367
:101E1000D3098093D2098091D2099091D309CF97A9
:101E200009F610921D241092611B8091D2099091A5
:101E3000D309FC01EE5CFB4D10829093DA0980938C
:101E4000D9091092D3091092D209809195289091C6
:101E50009628009709F4A6CF40E050E06091E81181
:101E60000E9472529FCF8830910571F5ACCF60917E
:101E70005731709158318DE090E00E94959010920A
:101E8000D1091092D0098091D0099091D109209167
:101E9000D2093091D309821793070CF0BCCFFC0113
:101EA000EE5CFB4D8081609157317091583190E02C
:101EB0000E9495908091D0099091D10901969093BC
:101EC000D1098093D009DFCF60915731709158319B
:101ED0000E9495908091D2099091D3092091D409C4
:101EE000FC01EE5CFB4D2083019691CF81E0DF91F8
:101EF000CF9108958091AC099091AD09892BD1F0D3
:101F00008091540290915502A0915602B0915702CF
:101F100093FD10C00E94B76583B7817F866083BF41
:101F2000F89483B7816083BF7894889583B78E7F58
:101F300083BF78940895CF93DF93EC0188819981D2
:101F4000009719F08735904199F40E9474640E94BB
:101F50007A0F40E050E065E88091EC119091ED112E
:101F60000E94725287E590E19983888381E003C0E3
:101F70001982188283E0DF91CF910895CF93DF9388
:101F800000D0CDB7DEB7892B81F05F934F938BEFF5
:101F90009DE09F938F9369837A830E94D9900F90DD
:101FA0000F900F900F907A8169817F936F9388EFE4
:101FB0009DE09F938F930E94D9900F900F900F9068
:101FC0000F900F900F90DF91CF910895FF920F9394
:101FD0001F93CF93DF930E94746480EB0E94D95DBE
:101FE00081111CC00E943D5E8091072090910820C5
:101FF0008160909308208093072089E993E09F9364
:102000008F9388EF9DE09F938F930E94D9900F90BC
:102010000F900F900F90C1E0D0E002C0C0E0D0E080
:10202000FEB08F2D8470F82E729A0E9474648EE434
:102030000E94D95D811116C00E943D5E80910720EB
:1020400090910820826090930820809307208E0151
:102050000F5F1F4F4EE059E061EA73E0CE010E942E
:10206000BE0FE801F11001C072980E9474648EEEF8
:102070000E94D95D811116C00E943D5E80910720AB
:1020800090910820846090930820809307208E010F
:102090000F5F1F4F4EE059E069EA73E0CE010E94E6
:1020A000BE0FE8010E94746486EA0E94D95D811126
:1020B00016C00E943D5E80910720909108208860A4
:1020C00090930820809307208E010F5F1F4F4EE0F2
:1020D00059E060EB73E0CE010E94BE0FE8010E9460
:1020E00074648CE30E94D95D81111EC00E943D5E24
:1020F0008091072090910820806190930820809320
:1021000007208E010F5F1F4F4EE059E068EB73E030
:10211000CE010E94BE0F80EF9DE09F938F930E949F
:10212000D9900F900F90E8010E94746482ED0E9494
:10213000D95D811116C00E943D5E8091072090916B
:102140000820806290930820809307208E010F5F03
:102150001F4F4EE059E060EC73E0CE010E94BE0FCD
:10216000E8010E94746480E80E94D95D811116C064
:102170000E943D5E8091072090910820916090938D
:102180000820809307208E010F5F1F4F4EE059E01B
:1021900069EC73E0CE010E94BE0FE8010E947464F6
:1021A00080ED0E94D95D811116C00E943D5E809134
:1021B0000720909108208068909308208093072042
:1021C0008E010F5F1F4F4EE059E06FEC73E0CE01C0
:1021D0000E94BE0FE8010E9474648CEE0E94D95DDB
:1021E000811116C00E943D5E8091072090910820C9
:1021F000926090930820809307208E010F5F1F4FFD
:102200004EE059E067ED73E0CE010E94BE0FE80199
:1022100007E010E00E9474648CE70E94D95D811190
:1022200013C00E943D5E8091072090910820806439
:1022300090930820809307204EE059E06EED73E004
:10224000CE010E94BE0F05C00150110901151105F4
:1022500009F70E943D5EDF91CF911F910F91FF9092
:102260000C94670BCF93DF9300D0CDB7DEB74A83D2
:1022700069830E94145E6981862F0E94455E4A81AF
:10228000842F0E94455E0F900F90DF91CF910C94A8
:102290003D5EAF92BF92DF92EF92FF920F931F933A
:1022A000CF93DF9300D01F92CDB7DEB7182FD22E79
:1022B0004A835B8369830E94145E6981862F0E9432
:1022C000455E812F81600E943B5E4A81A42E5B8126
:1022D000B52E00E010E0ED2CF12C81E0E81AF108B9
:1022E0000D1580F40E151F0519F40E94605E02C0E2
:1022F0000E94565EF50180830F5F1F4FFFEFAF1AFC
:10230000BF0AEECF0F900F900F90DF91CF911F91EA
:102310000F91FF90EF90DF90BF90AF900C943D5ED7
:10232000AF92BF92CF92DF92EF92FF920F931F93E3
:10233000CF93DF93CDB7DEB760970FB6F894DEBFCB
:102340000FBECDBFB82EA42E6623E9F18E010F5F1C
:102350001F4F80E1F80111928A95E9F728E0A80162
:1023600068E980EB0E944911BB2041F027EE33E081
:102370003F932F930E94C7900F900F906E01F8E04B
:10238000CF0ED11C5EEEE52E53E0F52EF8018191C3
:102390008F011F928F93FF92EF920E94C7900F9030
:1023A0000F900F900F900C151D0581F788851F92D7
:1023B0008F9323E434E03F932F930E94C7900F90B4
:1023C0000F900F900F90AA20E9F18E010F5F1F4F21
:1023D00080E1F80111928A95E9F728E0A80160E808
:1023E00080EB0E944911BB2041F083EF93E09F9363
:1023F0008F930E94C7900F900F906E01F0E1CF0E67
:10240000D11C4EEEE42E43E0F42EF80181918F01B1
:102410001F928F93FF92EF920E94C7900F900F90A0
:102420000F900F900C151D0581F788851F928F93D3
:1024300083E494E09F938F930E94C7900F900F9036
:102440000F900F9060960FB6F894DEBF0FBECDBF11
:10245000DF91CF911F910F91FF90EF90DF90CF9080
:10246000BF90AF900895CF93DF9300D0CDB7DEB784
:102470001A82198222E0AE014F5F5F4F6AEA8EEE48
:102480000E944911898190E0982F88272A81822B08
:102490009093D71B8093D61B22E0AE014F5F5F4F16
:1024A0006CEA8EEE0E944911898190E0982F88276E
:1024B0002A81822B9093D91B8093D81B22E0AE01F6
:1024C0004F5F5F4F6EEA8EEE0E944911898190E066
:1024D000982F88272A81822B9093DB1B8093DA1B0D
:1024E00022E0AE014F5F5F4F60EB8EEE0E9449111C
:1024F000898190E0982F88272A81822B9093E91B6D
:102500008093E81B22E0AE014F5F5F4F62EB8EEEDF
:102510000E944911898190E0982F88272A81822B77
:102520009093EB1B8093EA1B22E0AE014F5F5F4F5D
:1025300064EB8EEE0E944911898190E0982F8827E4
:102540002A81822B9093ED1B8093EC1B22E0AE013D
:102550004F5F5F4F66EB8EEE0E944911898190E0DC
:10256000982F88272A81822B9093DD1B8093DC1B78
:1025700022E0AE014F5F5F4F68EB8EEE0E94491183
:10258000898190E0982F88272A81822B9093DF1BE6
:102590008093DE1B22E0AE014F5F5F4F6AEB8EEE51
:1025A0000E944911898190E0982F88272A81822BE7
:1025B0009093E31B8093E21B22E0AE014F5F5F4FDD
:1025C0006CEB8EEE0E944911898190E0982F88274C
:1025D0002A81822B9093E51B8093E41B22E0AE01BD
:1025E0004F5F5F4F6EEB8EEE0E944911898190E044
:1025F000982F88272A81822B9093E71B8093E61BD4
:102600000F900F90DF91CF9108952F923F924F92AC
:102610005F926F927F928F929F92AF92BF92CF9272
:10262000DF92EF92FF920F931F93CF93DF93CDB77B
:10263000DEB76A970FB6F894DEBF0FBECDBF182F76
:10264000488F298F19821A821B828091FA1B81116F
:1026500007C06A8F0E94331281E08093FA1B6A8D53
:10266000662309F46CC04EE264EF8EEE0E943211D4
:1026700069E07AE180E090E00E94C65D22E0AE0170
:102680004F5F5F4F66EF8EEE0E9449112981822FC6
:1026900090E0A0E0B0E02227382F492F5A2F8A81FE
:1026A000282B8091EC1B9091ED1B281B390B4109C5
:1026B0005109A091EA1BB091EB1B0E94F6896B01B6
:1026C0007C018FE0F594E794D794C7948A95D1F76D
:1026D0006091E41B7091E51B882777FD8095982F0A
:1026E0002BE0660F771F881F991F2A95D1F720913D
:1026F000E61B3091E71B442737FD4095542F2C0DE6
:102700003D1D4E1D5F1D0E94638AC20ED31ED092D6
:10271000E11BC092E01B88E0C80ED11C34E0D594C8
:10272000C7943A95E1F7EE24D7FCE094FE2CC092D2
:10273000EE1BD092EF1BE092F01BF092F11B012FE9
:102740000295000F000F007C0C5CA12FB0E0BD8B48
:10275000AC8BA3E0B0E0012E02C0AA0FBB1F0A940D
:10276000E2F725E335E00E94EF89DC01CB01029618
:10277000A11DB11D8C879D87AE87BF8780E593EC37
:10278000A0E0B0E004C0B595A795979587951A95F8
:10279000D2F7888B998BAA8BBB8B10E01886198691
:1027A0001A861B86A8E02A2E312CAC89BD892A1AEC
:1027B0003B0A988D191709F436C1402F64EF8EEE4D
:1027C0000E9432116C857D858E859F850E94C65D35
:1027D00023E0AE014F5F5F4F66EF8EEE0E9449111E
:1027E000E091E01BF091E11BE05AFF409F01DF0107
:1027F0000E94D8896B017C018091D81B9091D91BD4
:102800009F8B8E8BA090D61BB090D71B2091DA1B8C
:102810003091DB1B0E94D8892B013C013DE075946F
:102820006794579447943A95D1F7A091DC1BB091E7
:10283000DD1BA70196016CE05595479537952795C7
:102840006A95D1F70E94018ABB2797FDB095AB2FFF
:10285000480E591E6A1E7B1E92E0490E511C611CD7
:10286000711CB2E07594679457944794BA95D1F768
:10287000A0E85A0E611C711CA091E81BB091E91BE5
:10288000A30192010E94F689DC01CB012FE0B695ED
:10289000A795979587952A95D1F78C839D83AE83CD
:1028A000BF8329818A8190E0A0E0B0E04424582EC3
:1028B000692E7A2E622A8B81482A022C04C07594D4
:1028C0006794579447940A94D2F74501AA2497FC39
:1028D000A094BA2C42E0880C991CAA1CBB1C4A95F7
:1028E000D1F7A091DE1BB091DF1BA70196010E94DA
:1028F000018A6B017C0157E1F594E794D794C79462
:102900005A95D1F72E893F89DF010E94D889EBE0E3
:102910009595879577956795EA95D1F7C60ED71E59
:10292000E81EF91E8C0C9D1CAE1CBF1C0C8804C03C
:10293000880C991CAA1CBB1C0A94D2F792E0890E41
:10294000911CA11CB11CF2E0B594A79497948794B4
:10295000FA95D1F7481859086A087B08A301920133
:10296000688979898A899B890E94098A97FD0DC0A7
:10297000660F771F881F991F2C813D814E815F81D3
:102980000E94418A49015A010CC02C813D814E812F
:102990005F810E94418A49015A01880C991CAA1C36
:1029A000BB1C9927B7FC9A958B2D7A2D692D9B011D
:1029B000AC010E94098A9B01AC01AEEDBBE00E9414
:1029C000F6896C01FF24D7FCF094EF2CA3E4B3EE5E
:1029D000A50194010E94048ABB2797FDB095AB2FF7
:1029E000C80ED91EEA1EFB1EAFECCA0EAEE0DA1E00
:1029F000E11CF11CA4E0F594E794D794C794AA9540
:102A0000D1F7C80CD91CEA1CFB1C88859985AA85BE
:102A1000BB858C0D9D1DAE1DBF1D88879987AA871C
:102A2000BB871F5FC6CE112391F0212F30E040E01D
:102A300050E0688579858A859B850E94418A20932C
:102A4000F21B3093F31B4093F41B5093F51BA98D9D
:102A5000AA2389F16091F21B7091F31B8091F41B02
:102A60009091F51B611571058105910521F10E9479
:102A70003A8720E836EE45EC57E40E949B8621E039
:102A80003EED42E45EE30E947B899B01AC0160E085
:102A900070E080E89FE30E94D0852BE43AE34DEBA1
:102AA00057E30E949B866093F61B7093F71B8093FD
:102AB000F81B9093F91B6A960FB6F894DEBF0FBE11
:102AC000CDBFDF91CF911F910F91FF90EF90DF90DD
:102AD000CF90BF90AF909F908F907F906F905F90BE
:102AE0004F903F902F9008950F931F93CF93DF93B4
:102AF00000D000D000D0CDB7DEB78E010F5F1F4FE2
:102B000086E0F80111928A95E9F78091081B8111FE
:102B100013C040E061E386EA0E9432114AE06CE2B1
:102B200086EA0E94321181E08093081B6CE77EE305
:102B300080E090E00E94C65D48E06DE286EA0E9477
:102B400032116CE77EE380E090E00E94C65D26E0F3
:102B5000A80162E386EA0E94491147E06DE286EA35
:102B60000E9432118A8190E0982F88272981822B38
:102B70009093031B8093021B2C8130E0322F22277D
:102B80004B81242B3093051B2093041B4E8150E076
:102B9000542F44276D81462B5093071B4093061BEF
:102BA0005F934F933F932F939F938F9387EF93E080
:102BB0009F938F930E94C7900FB6F894DEBF0FBE0D
:102BC000CDBF26960FB6F894DEBF0FBECDBFDF9106
:102BD000CF911F910F910895CF92DF92EF92FF92C4
:102BE0000F931F93CF93DF93CDB7DEB72A970FB61E
:102BF000F894DEBF0FBECDBF8E010F5F1F4F86E082
:102C0000F80111928A95E9F741E062E08CE30E94B5
:102C1000321148E560E08CE30E94321162E174E316
:102C200080E090E00E94C65D26E0A80163E08CE3AE
:102C30000E94491143E062E08CE30E943211098155
:102C400010E0102F00278A81082B1093E31A0093BD
:102C5000E21AEB80F12CFE2CEE248C81E82AF09213
:102C6000E51AE092E41ACD80D12CDC2CCC248E81A4
:102C7000C82AD092E71AC092E61AB801882777FDD1
:102C80008095982F0E943A879B01AC01B701882755
:102C900077FD8095982F2F83388749875A870E9420
:102CA0003A872F81388549855A850E94448620EECF
:102CB0003EE245E652E40E94188920E030E044E319
:102CC00053E40E94D1859F938F937F936F93DF92FC
:102CD000CF92FF92EF921F930F9385E094E09F9322
:102CE0008F930E94C7900FB6F894DEBF0FBECDBF82
:102CF0002A960FB6F894DEBF0FBECDBFDF91CF91FD
:102D00001F910F91FF90EF90DF90CF900895CF9398
:102D1000DF93EC01888199810097F9F0803490412C
:102D200021F01982188283E063C08FEB99E00E9442
:102D30001855892BE1F08091AF099091B00993FD6E
:102D400018C08091AF099091B00994FD43C0809163
:102D5000AF099091B00995FD44C060E870E08FEB39
:102D600099E00E94F15480E490E19983888381E0A6
:102D70003FC08091072082FFE4CF21E048E061E07E
:102D800083E00E9405138091F91B8F938091F81BBB
:102D90008F938091F71B8F938091F61B8F93809177
:102DA000F51B8F938091F41B8F938091F31B8F936E
:102DB0008091F21B8F938FE49EE09F938F930E94EC
:102DC000D9908DB79EB70A960FB6F8949EBF0FBEE6
:102DD0008DBFB7CF8091072083FFB9CF0E947415B4
:102DE000B6CF8091072084FFB8CF0E94EC15B5CFF5
:102DF000DF91CF910895CF93C82F8CEE0E943B5E58
:102E00008C2F0E94455E65E375E080E090E00E94B3
:102E1000C65D8DEE0E943B5E0E94565EC82F0E94EA
:102E2000605E2C2F30E0322F2227A901482BCA01E7
:102E3000CF910895CF93DF93C82F8CEE0E943B5E15
:102E40008C2F0E94455E62E174E380E090E00E9476
:102E5000C65D8CEE0E943B5E80E00E94455E65E3AD
:102E600075E080E090E00E94C65D8DEE0E943B5EC2
:102E70000E94565EC82F0E94565ED82F0E94605E48
:102E80004D2F50E060E070E0762F652F542F4427DF
:102E90006C2B482BCB01BA01DF91CF9108952F9273
:102EA0003F924F925F926F927F928F929F92AF92DA
:102EB000BF92CF92DF92EF92FF920F931F93CF9327
:102EC000DF93CDB7DEB7CD54D1090FB6F894DEBF8E
:102ED0000FBECDBF8091000290910102892BD1F1EC
:102EE00010920102109200028CEE0E943B5E8EE175
:102EF0000E94455E6BE17EE480E090E00E94C65D4A
:102F000082EA0E94FB169093BC098093BB0984EA75
:102F10000E94FB169093BA098093B90986EA0E9431
:102F2000FB169093B8098093B70988EA0E94FB16B4
:102F30009093B6098093B5098AEA0E94FB16909394
:102F4000B4098093B3098CEA0E94FB169093B209EE
:102F50008093B10988E40E941A176FAB78AF89AFEC
:102F60009AAF88E50E941A174B015C018091B30962
:102F70009091B40920E030E040E050E0BA0126969C
:102F80002FAF269727963FAF279728964FAF2897C2
:102F900029965FAF29972A966FAF2A972B967FAF16
:102FA0002B979C0140E050E060E070E080E090E012
:102FB00008E00E94EA8B0E94968B3901B42FA52F5E
:102FC000F62FE72F8C019401A50160E070E080E00E
:102FD00090E05301CB2EDA2EEF2EFE2E0E94218C94
:102FE00029833A832A011B014C01B101C4013150EC
:102FF00041095F4F6F4F7F4F8F4F9F4FA1E0B0E070
:103000002596BFAFAEAF259721153F4F4F4F51408B
:10301000610571058105910509F020F425961FAE23
:103020001EAE259725966EAC7FAC25978091B10991
:103030009091B2095C01C12CD12CE12CF12C00E063
:1030400010E029813A81A201B101C4010E94B98A2C
:10305000D22EE32EF42E052F162FB72FF82FE92F9F
:10306000A0E00E94488C84F42150310940485F4F11
:103070006F4F7F4F8F4F9F4FD22EE32EF42E052F91
:10308000162FB72FF82FE92F2D2D3E2D4F2D502F16
:10309000612F7B2F8F2F9E2F07E10E94038C2B8F98
:1030A0003C8F4D8F5E8F6F8F78A389A39AA3205397
:1030B000384F4F4F5F4F6F4F7F4F8F4F9F4F2B8B2F
:1030C0003C8B4D8B5E8B6F8B788F898F9A8F2056C0
:1030D000304F4F4F5F4F6F4F7F4F8F4F9F4F243D6C
:1030E000304341055105610571058105910541F0A8
:1030F00038F025966EAC7FAC2597FFEF6F1A7F0AEC
:103100008091B9099091BA099C0140E050E060E0DB
:1031100070E080E090E000E10E94EA8B2B833C832A
:103120004D835E836A8779878F8398874091B5093D
:103130005091B609A980BA806201710184019A0197
:1031400040E050E060E070E080E090E00E94B98AEA
:10315000D22EE32EF42E052F162FB72FF82FE92F9E
:10316000A0E00E94488C5CF4AFE70E942A8CD22E2B
:10317000E32EF42E052F162FB72FF82FE92F2D2D24
:103180003E2D4F2D502F612F7B2F8F2F9E2F07E02D
:103190000E94038C59016A017B018C012B813C81C7
:1031A0004D815E816A8579858F8198850E94218C09
:1031B0002B833C834D835E836F8378878F87988BC7
:1031C0002E5F3F4F434051096E4F7F4F8F4F9F4FB0
:1031D00022303105494F5F4F6440710581059105EB
:1031E00021F018F01FEF611A710A8091BB099091CC
:1031F000BC09BC0180E090E020E030E840E050E015
:103200000E94128B29873A874B875C876A8B798B60
:103210008D879E874091B7095091B809A980BA80DF
:103220006201710184019A0140E050E060E070E0C9
:1032300080E090E00E94B98AD22EE32EF42E052F72
:10324000162FB72FF82FE92FA0E00E94488C84F4A6
:1032500021503F4F4F4F5F4F6F4F7F4F8F4F9F4FCB
:10326000D22EE32EF42E052F162FB72FF82FE92F8D
:103270002D2D3E2D4F2D502F612F7B2F8F2F9E2FC9
:1032800008E00E94038C59016A017B018C012985A9
:103290003A854B855C856A8979898D859E850E94F2
:1032A000218C29873A874B875C876D877E87898B3E
:1032B0009A8B2F5F3F4F4140510961097109810984
:1032C0009109213030484C4F5F47614071058105BD
:1032D000910521F018F0BFEF6B1A7B0A2B893C890E
:1032E0004D895E896F89788D898D9A8D2F3C374005
:1032F00041055105610571058105910511F00CF03D
:10330000A5C1A980BA806201710184019501A20161
:10331000B101C4010E94B98AA12CB12CC12C10E8C2
:10332000D12EE12CF12C00E010E00E947C8A2BAF22
:103330003CAF4DAF5EAF6FAF21967FAF2197229626
:103340008FAF229723969FAF2397AB8CBC8CCD8CED
:10335000DE8CEF8CF8A009A11AA19501A601B70196
:10336000C8010E94B98A59016A017B01E82F192F0F
:1033700002E00E94EA8B0E2F0E94218C69017A01E3
:10338000162F272EF82FE92F322E8D2C942EAF2CAE
:10339000B62E072F582EB92FA0E00E94488C5CF45F
:1033A000A1E00E942A8C322E832E942EA52EB62EBA
:1033B000072F582EB92F232D382D492D5A2D6B2D1F
:1033C000702F852D9B2F01E00E94038C2E962FAF2E
:1033D0002E972D963FAF2D9749A75AA76BA77CA78D
:1033E0008DA79EA7522E432E4BA35CA36DA37EA355
:1033F0008FA398A7B22D9601A701612F722D8F2F51
:103400009E2FA0E00E94488C4CF4A3E00E942A8CDE
:1034100069017A01162FB72FF82FE92F9601A7011E
:10342000612F7B2F8F2F9E2F02E00E94038C2FA7EE
:1034300038AB49AB5AAB6BAB7CAB8DAB9EAB1901D8
:103440004A01B62FA72F24968FAF2497F92F2B89E7
:103450003C894D895E896F89788D898D9A8D24325A
:103460003A4F4F4F5F4F6F4F7F4F8F4F9F4F0CF033
:103470008CC02B8D3C8D4D8D5E8D6F8D78A189A17B
:103480009AA12455324F4F4F5F4F6F4F7F4F8F4F51
:103490009F4F59016A017B018C010E94B98A190171
:1034A0004A01B62FA72FFC0103E00E94EA8B5101CD
:1034B0006401EB2EFA2E8F010E94368C59016A01AD
:1034C0007B018C012E962FAD2E972D963FAD2D971B
:1034D00049A55AA56BA57CA58DA59EA50E94218C0A
:1034E000522E432E4BA35CA36DA37EA38FA398A75C
:1034F0009101A4016B2F7A2FCF0102E00E94EA8B89
:1035000051016401EB2EFA2E8F010E94368C02E0ED
:103510000E94EA8B0E2F0E94368CF22E032F142F5E
:10352000D52EE62EB72FF82FE92FA0E00E94488C69
:103530005CF4A1E00E942A8CF22E032F142FD52ECA
:10354000E62EB72FF82FE92F2F2D302F412F5D2D8D
:103550006E2D7B2F8F2F9E2F01E00E94038C59012F
:103560006A017B018C012FA538A949A95AA96BA929
:103570007CA98DA99EA90E94218C19014A01B62F10
:10358000A72F24968FAF2497F92F2B813C814D8153
:103590005E816F8178858F859889A52CB42CCBA00E
:1035A000DCA0EDA0FEA00FA118A50E94368C2B83F5
:1035B0003C834D835E836F8378878F87988B2985C3
:1035C0003A854B855C856D857E8589899A8951010F
:1035D0006401EB2EFA2E24960FAD24971F2F0E9424
:1035E000368C29873A874B875C876D877E87898BE6
:1035F0009A8B2B893C894D895E896F89788D898D5D
:103600009A8DABACBCACCDACDEACEFAC2196FFACD4
:10361000219722960FAD229723961FAD23970E94E4
:10362000368C2056304F4F4F5F4F6F4F7F4F8F4F2D
:103630009F4F243D304341055105610571058105CA
:10364000910521F018F02FEF621A720A6FA978AD78
:1036500089AD9AADAB01BC0180E090E0DC0124961D
:103660004FAF249725965FAF259726966FAF269785
:1036700027967FAF279728968FAF289729969FAFD9
:1036800029972A96AFAF2A972B96BFAF2B97A9847D
:10369000BA84CB84DC84ED84FE8409891A899A017A
:1036A000AB0160E070E080E090E00E94B98AF22E09
:1036B000032F142FD52EE62EB72FF82FE92FA0E0D9
:1036C0000E94488C84F421503109404E5F4F6F4F67
:1036D0007F4F8F4F9F4FF22E032F142FD52EE62EA4
:1036E000B72FF82FE92F2F2D302F412F5D2D6E2D65
:1036F0007B2F8F2F9E2F05E10E94038CAB80BC8017
:10370000CD80DE80EF80F8840F8518890E94368C8A
:10371000F22E032F142FD52EE62EB72FF82FE92FD8
:10372000A0E00E94488C84F4215030484F4F5F4FF6
:103730006F4F7F4F8F4F9F4FF22E032F142FD52E99
:10374000E62EB72FF82FE92F2F2D302F412F5D2D8B
:103750006E2D7B2F8F2F9E2F0FE00E94038C69010F
:103760007A018B018A83998329011A014B015C013B
:10377000285E3340410951096109710981099109A4
:10378000283D304D41405105610571058105910588
:1037900021F018F0BFEF6B1A7B0A0E943D5E67288C
:1037A00059F09601A701B8018A8199810E94968BF0
:1037B00029011A014B015C019201A101B401C5016B
:1037C0000E94348720E030E048EC52E40E949B865F
:1037D000C35BDF4F0FB6F894DEBF0FBECDBFDF91E6
:1037E000CF911F910F91FF90EF90DF90CF90BF90FE
:1037F000AF909F908F907F906F905F904F903F9091
:103800002F9008954F925F926F927F928F929F9226
:10381000AF92BF92CF92DF92EF92FF922B013C01C9
:1038200069017A0123EC35EF4CE851E4C701B60198
:103830000E9418894B015C0128EB3EE143E753E409
:10384000C701B6010E94D1859B01AC01C501B4013D
:103850000E949B860E9408874B015C0120E030E0BB
:1038600048EC52E4C301B2010E949B8621E835E98D
:1038700043EC50E40E941889A50194010E94188924
:103880004B015C0123E333E948E853E4C701B60187
:103890000E94D1859B01AC01C501B4010E949B86A9
:1038A00023E333EB48E553E40E941889FF90EF903F
:1038B000DF90CF90BF90AF909F908F907F906F9050
:1038C0005F904F9008954F925F926F927F928F9288
:1038D0009F92AF92BF92CF92DF92EF92FF926901D7
:1038E0007A010E949A8820E030E040E050E40E9493
:1038F000D08522E93CE54EED5EE30E949B864B01BC
:103900005C0123EC35EF4CE851E4C701B6010E949D
:1039100018892B013C0128EB3EE143E753E4C70142
:10392000B6010E94D1859B01AC01C301B2010E9486
:103930009B869B01AC01C501B4010E94D1856B013E
:103940007C0128EB3EE143E753E40E9418894B01D8
:103950005C01A701960163EC75EF8CE891E40E948D
:10396000D0859B01AC01C501B4010E949B86FF90EC
:10397000EF90DF90CF90BF90AF909F908F907F900F
:103980006F905F904F9008954F925F926F927F92E9
:103990008F929F92AF92BF92CF92DF92EF92FF925F
:1039A0002B013C0169017A0123EC35EF4CE851E42D
:1039B000C701B6010E9418894B015C0128EB3EE16A
:1039C00043E753E4C701B6010E94D1859B01AC01D6
:1039D000C501B4010E949B860E9408874B015C01CF
:1039E00020E030E048EC52E4C301B2010E949B8623
:1039F000A50194010E94188920E030E040E251E4E2
:103A00000E94D08524EE38E34EE05FE30E941889DF
:103A10009B01AC01C701B6010E94D185FF90EF90D8
:103A2000DF90CF90BF90AF909F908F907F906F90DE
:103A30005F904F90089580E80E943B5E81110DC019
:103A40008EEF0E94455E811108C06BE17EE480E04C
:103A500090E00E94C65D0C943D5E0E943D5E8091A8
:103A6000192490911A24A0911B24B0911C24019632
:103A7000A11DB11D8093192490931A24A0931B2497
:103A8000B0931C240895FC01DC0182E020E041E3B6
:103A90009D91292798E0322F330F27FF03C0232F52
:103AA000242701C0232F9150B1F7815089F781E07D
:103AB00090E03281231711F080E090E00895CF92DA
:103AC000DF92EF92FF920F931F93CF93DF930E94A9
:103AD0001B1D80E80E943B5E811172C08AEF0E942C
:103AE000455E81116DC08FE00E94455E811168C006
:103AF00065E375E080E090E00E94C65D81E80E9489
:103B00003B5E81115DC00E94565EC82F0E94565ECA
:103B10000E94565ED82F0E94565E0E94565E182F55
:103B20000E94565E0E94605E082F0E94605E80E8E0
:103B30000E943B5E811144C08CEF0E94455E811162
:103B40003FC089EC0E94455E81113AC065E375E093
:103B500080E090E00E94C65D81E80E943B5E0E948A
:103B6000565ED82E0E94565EC82E0E94565E0E9457
:103B7000565EF82E0E94565EE82E0E94605E1F92EE
:103B8000CF921F92DF921F920F931F921F931F924B
:103B9000DF931F92CF931F92EF921F92FF928AE1C1
:103BA00094E09F938F930E94C7900E943D5E8DB7D3
:103BB0009EB742960FB6F8949EBF0FBE8DBF17C03A
:103BC0000E943D5E8091192490911A24A0911B249B
:103BD000B0911C240196A11DB11D809319249093CE
:103BE0001A24A0931B24B0931C240E941B1D20E0C8
:103BF00030E040E050E060E070E080E090E0DF9195
:103C0000CF911F910F91FF90EF90DF90CF9008958B
:103C1000EF92FF920F931F93CF93DF9300D01F92E9
:103C2000CDB7DEB78C0180E80E943B5E811154C0A5
:103C30000115110551F085EE0E94455E81114CC0C1
:103C400061E077E980E090E009C083EE0E94455E84
:103C5000811142C069E97AEB81E090E00E94C65D83
:103C600081E80E943B5E811137C00E94565EF82EAB
:103C700089830E94565EE82E8A830E94605E8B8351
:103C80000E943D5ECE0101960E94431D892B21F1C9
:103C90006E2D70E07F296C7F80E090E0012B69F051
:103CA0000E94388720E030E04AEF5AE30E941889EA
:103CB00020E030E040EC50E40CC00E94388722E560
:103CC00038EB4FE25BE30E94188926E636E64BE3C9
:103CD00052E40E94D0851BC00E943D5E8091192451
:103CE00090911A24A0911B24B0911C240196A11D2F
:103CF000B11D8093192490931A24A0931B24B09390
:103D00001C240E941B1D60EF7FEF89E794E40F9055
:103D10000F900F90DF91CF911F910F91FF90EF9037
:103D200008950F931F93CF93DF93729A809154025B
:103D300083FF08C08EE40E94D95D811163C0C0E595
:103D4000D0E008C0C0E5D0E00E9474092197209718
:103D5000D9F7F0CF0E94740921972097D9F78FE403
:103D60000E94D95D0E94565E082F0F730E94565E16
:103D7000182F0E94565ED82F0E94605EC82F0E94A6
:103D80003D5E8091540283FF7298602F70E0762F21
:103D90006627610F711D80E090E00E94388720E166
:103DA00034E048EC5BE30E9418896093FB1B70933E
:103DB000FC1B8093FD1B9093FE1B6D2F70E0762FF4
:103DC00066276C0F711D769567957695679580E0EF
:103DD00090E00E94388724EA3CEF44E25CE30E94D2
:103DE000188920E030E040E252E40E94D0856093E0
:103DF00098287093992880939A2890939B2880E024
:103E000090E002C081E090E0DF91CF911F910F918F
:103E100008957298729A8EE40E94D95D80EA0E9499
:103E2000455E80E00E94455E80E00E94455E8FE432
:103E30000E94D95D0E94565E8EE40E94D95D80E8A2
:103E40000E94455E80E00E94455E80E00E94455EE3
:103E50000E943D5E80E090E0089583EE9DE09F9398
:103E60008F930E94D99080916F020F900F908823BA
:103E700061F01F928F9380EE9DE09F938F930E943D
:103E8000D9900F900F900F900F9008958BEB9DE0BD
:103E90009F938F930E94D99083E99DE09F938F9386
:103EA0000E94D9908CE69DE09F938F930E94D990B9
:103EB00081E39DE09F938F930E94D9908FEF9CE0C8
:103EC0009F938F930E94D99083EC9CE09F938F9354
:103ED0000E94D9908DE99CE09F938F930E94D99086
:103EE00087E69CE09F938F930E94D9908091072052
:103EF00090910820827091702DB73EB7205F3F4FA0
:103F00000FB6F8943EBF0FBE2DBF892B41F087E35B
:103F10009CE09F938F930E94D9900F900F908BE01D
:103F20009CE09F938F930E94D99082EE9BE09F9399
:103F30008F930E94D99086EB9BE09F938F930E9472
:103F4000D99087E89BE09F938F930E94D99085E555
:103F50009BE09F938F930E94D99084E29BE09F9374
:103F60008F930E94D9908AEE9AE09F938F930E943C
:103F7000D99084EB9AE09F938F930E94D99084E824
:103F80009AE09F938F930E94D99088E59AE09F933F
:103F90008F930E94D99089E29AE09F938F930E9419
:103FA000D99080EF99E09F938F930E94D99087EBEF
:103FB00099E09F938F930E94D99080E899E09F9316
:103FC0008F930E94D9908FE499E09F938F930E94E2
:103FD000D99080E299E09F938F930E94D9908DB7FA
:103FE0009EB780960FB6F8949EBF0FBE8DBF81EF2F
:103FF00098E09F938F930E94D9908AEC98E09F93CA
:104000008F930E94D99084E998E09F938F930E94A8
:10401000D9908EE598E09F938F930E94D99088E283
:1040200098E09F938F930E94D9908FEF97E09F9392
:104030008F930E94D99087EC97E09F938F930E9473
:10404000D9908CE997E09F938F930E94D9902DB7D8
:104050003EB7205F3F4F0FB6F8943EBF0FBE2DBF57
:10406000089589E494E00C94FD904F925F926F92D2
:104070007F928F929F92AF92BF92CF92DF92EF92F8
:10408000FF92CF93DF93CDB7DEB728970FB6F894A2
:10409000DEBF0FBECDBF80910D2490910E24A09164
:1040A0000F24B091102489839A83AB83BC83409002
:1040B0000D2450900E2460900F2470901024809155
:1040C0000D2490910E24A0910F24B09110248D8383
:1040D0009E83AF83B88760910D2470910E248091E8
:1040E0000F24909110242CE3822E912CA12CB12C22
:1040F000A50194010E94418A7F936F9330E1C32E02
:104100003EE0D32EE12CF12C6D817E818F8198854C
:10411000A70196010E94418AA50194010E94418A4B
:104120003F932F9340E8842E41E5942EAA24A39434
:10413000B12CC301B201A50194010E94418AA701DB
:1041400096010E94418A3F932F9369817A818B81E6
:104150009C81A50194010E94418A3F932F9386E799
:1041600097E09F938F930E94D9900FB6F894DEBF8B
:104170000FBECDBF28960FB6F894DEBF0FBECDBFE1
:10418000DF91CF91FF90EF90DF90CF90BF90AF90F5
:104190009F908F907F906F905F904F900895EDE586
:1041A000F1E3808191818234924479F0ED55F143BD
:1041B000FF93EF9388E597E09F938F930E94D990A8
:1041C0000F900F900F900F9008953A96E53F81E47D
:1041D000F80738F30895CF93DF93EC018C9A0E948F
:1041E000570A9F938F937F936F938CE497E09F93ED
:1041F0008F930E94D9900F900F900F900F900F9077
:104200000F90209719F00E94670B08C08AE497E08E
:104210009F938F930E94D9900F900F9081E00E94FE
:10422000080A2091740230917502409176025091F3
:1042300077020E9418899F938F937F936F938EE3E9
:1042400097E09F938F930E94D9900F900F900F90BB
:104250000F900F900F90209719F00E94670B08C0E5
:104260008CE397E09F938F930E94D9900F900F90CB
:1042700082E00E94080A2091700230917102409100
:104280007202509173020E9418899F938F937F93BB
:104290006F9380E397E09F938F930E94D9900F9044
:1042A0000F900F900F900F900F90209719F00E9491
:1042B000670B08C08EE297E09F938F930E94D9907E
:1042C0000F900F9083E00E94080A9F938F937F9333
:1042D0006F938FE197E09F938F930E94D9908C9872
:1042E0000F900F900F900F900F900F90209719F054
:1042F0000E94670B08C08DE197E09F938F930E9407
:10430000D9900F900F908091072087FF83C021E004
:1043100042E161E080ED0E949D5F9F938F937F93C8
:104320006F9380E197E09F938F930E94D9900F90B5
:104330000F900F900F900F900F90209719F00E9400
:10434000670B08C08EE097E09F938F930E94D990EF
:104350000F900F9021E042E162E080ED0E949D5FAE
:104360009F938F937F936F9381E097E09F938F93B9
:104370000E94D9900F900F900F900F900F900F9078
:10438000209719F00E94670B08C08FEF96E09F936B
:104390008F930E94D9900F900F9021E042E163E04B
:1043A00080ED0E949D5F9F938F937F936F9382EF29
:1043B00096E09F938F930E94D9900F900F900F904B
:1043C0000F900F900F90CD2B19F00E94670B08C033
:1043D00080EF96E09F938F930E94D9900F900F905B
:1043E00021E042E164E080ED0E949D5F9F938F9306
:1043F0007F936F9383EE96E09F938F930E94D99063
:104400000F900F900F900F900F900F90DF91CF9122
:104410000C94670BCD2BD1F3DF91CF9108950F93BF
:104420001F93CF93DF93882389F049E050E06FEF2B
:1044300070E08CE898E20E941B9049E050E06AE04E
:1044400070E08CE898E20E944B9213C0CCE8D8E26E
:104450000EED16E089911F928F931F930F930E9488
:10446000D9900F900F900F900F9088E2C439D80721
:1044700089F7DF91CF911F910F910C94670BCF9229
:10448000DF92EF92FF92CF93DF936B017C0160FF8D
:1044900011C086E894E09F938F9388EF9DE09F93EF
:1044A0008F930E94D9900F900F900F900F9081E002
:1044B00090E002C080E090E0C1FE09C0EC012196CE
:1044C0004EE059E06BE874E00E94BE0FCE01C2FEE0
:1044D00009C0EC0121964EE059E063E974E00E94C6
:1044E000BE0FCE01C3FE09C0EC0121964EE059E09B
:1044F0006BE974E00E94BE0FCE01C4FE09C0EC015E
:1045000021964EE059E06FE974E00E94BE0FCE01A3
:10451000C5FE09C0EC0121964EE059E062EA74E064
:104520000E94BE0FCE01C6FE09C0EC0121964EE0EE
:1045300059E066EA74E00E94BE0FCE01C7FE09C0D2
:10454000EC0121964EE059E06CEA74E00E94BE0F47
:10455000CE01D0FE09C0EC0121964EE059E064EB9B
:1045600074E00E94BE0FCE01D1FE09C0EC0121967D
:104570004EE059E06CEB74E00E94BE0FCE01D2FE1B
:1045800009C0EC0121964EE059E060EC74E00E9415
:10459000BE0FCE0120910720309108202470327088
:1045A000232B59F0D3FE09C0EC0121964EE059E0CF
:1045B00066EC74E00E94BE0FCE012091072023FF1D
:1045C0000BC0D4FE09C0EC0121964EE059E06BEC23
:1045D00074E00E94BE0FCE012091072024FF0BC083
:1045E000D5FE09C0EC0121964EE059E061ED74E082
:1045F0000E94BE0FCE01D6FE09C0EC0121964EE00E
:1046000059E069ED74E00E94BE0FCE01B701A6012A
:1046100044275078452B462B472B61F04EE059E05C
:1046200064EE74E0DF91CF91FF90EF90DF90CF9038
:104630000C94BE0FCD28CE28CF2841F489ED96E00A
:104640009F938F930E94D9900F900F90DF91CF91FD
:10465000FF90EF90DF90CF9008950F931F93CF932B
:10466000DF938C01C0E0D0E00115110509F48AC088
:1046700064ED76E0C8010E94FA8F892B09F4C160CD
:104680006CEC76E0C8010E94FA8F892B09F4C260B5
:1046900064EC76E0C8010E94FA8F892B09F4C460AB
:1046A00060EC76E0C8010E94FA8F892B09F4C8609B
:1046B0006DEB76E0C8010E94FA8F892B09F4C06186
:1046C00069EB76E0C8010E94FA8F892B09F4C06279
:1046D00063EB76E0C8010E94FA8F892B09F4C0646D
:1046E0006BEA76E0C8010E94FA8F892B09F4C06852
:1046F00063EA76E0C8010E94FA8F892B09F4D16041
:104700006FE976E0C8010E94FA8F892B09F4D26024
:1047100069E976E0C8010E94FA8F892B09F4D46018
:1047200064E976E0C8010E94FA8F892B09F4D86009
:104730006EE876E0C8010E94FA8F892B09F4D061F7
:1047400066E876E0C8010E94FA8F892B09F4D062EE
:104750006BE776E0C8010E94FA8F892B09F4D064D8
:104760006AE676E0C8010E94FA8F892B09F4D068C6
:1047700060916D0270916E0280E090E00E940E9058
:104780008C0172CFCE01DF91CF911F910F910895CF
:10479000AF92BF92CF92DF92EF92FF920F931F934F
:1047A000CF93DF93F22E032F142FE52ED62EA72EB4
:1047B000B82EC92E217030E040E050E060E070E09B
:1047C00080E090E0A0E00E94488C89F0E5EFF4E002
:1047D000FF93EF93E8EFFDE0FF93EF930E94D990F2
:1047E0000F900F900F900F90E1E0F0E002C0E0E03A
:1047F000F0E08091072080FF17C02F2D247030E05B
:1048000040E050E060E070E080E090E0A0E00E94D6
:10481000488C51F0EF0121964EE059E069EF74E0C9
:10482000CF010E94BE0FFE012F2D227030E040E02C
:1048300050E060E070E080E090E0A0E00E94488CF2
:1048400051F0EF0121964EE059E06DEF74E0CF0199
:104850000E94BE0FFE012F2D287030E040E050E096
:1048600060E070E080E090E0A0E00E94488C51F0B1
:10487000EF0121964EE059E065E175E0CF010E941D
:10488000BE0FFE012F2D207130E040E050E060E0CF
:1048900070E080E090E0A0E00E94488C51F0EF01D1
:1048A00021964EE059E060E075E0CF010E94BE0F16
:1048B000FE012F2D207230E040E050E060E070E01B
:1048C00080E090E0A0E00E94488C51F0EF0121963A
:1048D0004EE059E063E075E0CF010E94BE0FFE019B
:1048E0002F2D207430E040E050E060E070E080E088
:1048F00090E0A0E00E94488C51F0EF0121964EE03C
:1049000059E069E075E0CF010E94BE0FFE012F2D36
:10491000207830E040E050E060E070E080E090E03F
:10492000A0E00E94488C51F0EF0121964EE059E042
:104930006FE075E0CF010E94BE0FFE0120E0302F36
:10494000317040E050E060E070E080E090E0A0E096
:104950000E94488C51F0EF0121964EE059E062E14F
:1049600075E0CF010E94BE0FFE0120E0302F3270B3
:1049700040E050E060E070E080E090E0A0E00E9465
:10498000488C51F0EF0121964EE059E067E175E067
:10499000CF010E94BE0FFE0120E0302F347040E0B6
:1049A00050E060E070E080E090E0A0E00E94488C81
:1049B00051F0EF0121964EE059E06EE175E0CF0134
:1049C0000E94BE0FFE0120E0302F387040E050E022
:1049D00060E070E080E090E0A0E00E94488C51F040
:1049E000EF0121964EE059E061E275E0CF010E94AF
:1049F000BE0FFE0120E0302F307140E050E060E05B
:104A000070E080E090E0A0E00E94488C51F0EF015F
:104A100021964EE059E066E275E0CF010E94BE0F9C
:104A2000FE0120E0302F307240E050E060E070E0A6
:104A300080E090E0A0E00E94488C51F0EF012196C8
:104A40004EE059E06DE275E0CF010E94BE0FFE011D
:104A500020E030E040E050E06D2D647070E080E0D8
:104A600090E0A0E00E94488C51F0EF0121964EE0CA
:104A700059E064E375E0CF010E94BE0FFE01809112
:104A8000072081FF17C020E0302F307440E050E055
:104A900060E070E080E090E0A0E00E94488C51F07F
:104AA000EF0121964EE059E068E375E0CF010E94E6
:104AB000BE0FFE01809107209091082090FF17C043
:104AC00020E030E040E05E2D507160E070E080E07A
:104AD00090E0A0E00E94488C51F0EF0121964EE05A
:104AE00059E06BE375E0CF010E94BE0FFE0180919B
:104AF00007209091082090FF17C020E030E040E0B0
:104B00005E2D507260E070E080E090E0A0E00E94D6
:104B1000488C51F0EF0121964EE059E06EE375E0CC
:104B2000CF010E94BE0FFE018091072090910820C6
:104B300090FF17C020E030E040E05E2D507460E050
:104B400070E080E090E0A0E00E94488C51F0EF011E
:104B500021964EE059E064E475E0CF010E94BE0F5B
:104B6000FE0120E0302F307840E050E060E070E05F
:104B700080E090E0A0E00E94488C51F0EF01219687
:104B80004EE059E06FE475E0CF010E94BE0FFE01D8
:104B900020E030E0412F417050E060E070E080E0C4
:104BA00090E0A0E00E94488C51F0EF0121964EE089
:104BB00059E064E575E0CF010E94BE0FFE0120E0E0
:104BC00030E0412F427050E060E070E080E090E023
:104BD000A0E00E94488C51F0EF0121964EE059E090
:104BE00067E575E0CF010E94BE0FFE0120E030E0D6
:104BF000412F447050E060E070E080E090E0A0E081
:104C00000E94488C51F0EF0121964EE059E06AE590
:104C100075E0CF010E94BE0FFE018091072087FF43
:104C200017C020E030E0412F487050E060E070E0B5
:104C300080E090E0A0E00E94488C51F0EF012196C6
:104C40004EE059E06DE575E0CF010E94BE0FFE0118
:104C50008091072087FF17C020E030E0412F40718E
:104C600050E060E070E080E090E0A0E00E94488CBE
:104C700051F0EF0121964EE059E061E675E0CF0179
:104C80000E94BE0FFE018091072087FF17C020E021
:104C900030E0412F407250E060E070E080E090E052
:104CA000A0E00E94488C51F0EF0121964EE059E0BF
:104CB00065E675E0CF010E94BE0FFE0180910720DE
:104CC00087FF17C020E030E0412F407450E060E0E3
:104CD00070E080E090E0A0E00E94488C51F0EF018D
:104CE00021964EE059E069E675E0CF010E94BE0FC3
:104CF000FE018091072082FF17C020E030E0412FA5
:104D0000407850E060E070E080E090E0A0E00E9439
:104D1000488C51F0EF0121964EE059E068E276E0D0
:104D2000CF010E94BE0FFE018091072082FF17C0B5
:104D300020E030E040E05E2D517060E070E080E007
:104D400090E0A0E00E94488C51F0EF0121964EE0E7
:104D500059E06DE675E0CF010E94BE0FFE01809123
:104D600007209091082090FF17C020E030E040E03D
:104D70005E2D527060E070E080E090E0A0E00E9464
:104D8000488C51F0EF0121964EE059E060E775E064
:104D9000CF010E94BE0FFE01809107209091082054
:104DA00090FF17C020E030E040E05E2D547060E0DE
:104DB00070E080E090E0A0E00E94488C51F0EF01AC
:104DC00021964EE059E068E775E0CF010E94BE0FE2
:104DD000FE01809107209091082091FF1EC020E0E5
:104DE00030E040E05E2D587060E070E080E090E0E0
:104DF000A0E00E94488C89F04EE059E061E875E03F
:104E0000CF01DF91CF911F910F91FF90EF90DF9035
:104E1000CF90BF90AF900C94BE0F2F2D302F412F0D
:104E20005E2D6D2D7A2D8B2D9C2DA0E00E94488C3F
:104E300041F485E696E09F938F930E94D9900F905E
:104E40000F90DF91CF911F910F91FF90EF90DF9026
:104E5000CF90BF90AF9008958F929F92BF92DF92B4
:104E6000EF920F931F93CF93DF93EC014B01FB0164
:104E7000108260E676E00E94FA8F892B61F58091BE
:104E800007207DE4D72EE0E8EE2E82FD02C004E08C
:104E900001C004E810E0B12C81FF02C060ECE62EF6
:104EA00026E04AE250E06BE270E089E290E00E9486
:104EB000ED5A81E090E00E94F50A882311F05DE54B
:104EC000D52E809107209091082090FD16E091FF4B
:104ED00007C0186005C0D12CE12C00E010E0B12C17
:104EE0006EE576E0CE010E94FA8F892B61F481E0B5
:104EF000F401808360916D0270916E0280E090E019
:104F00000E940E90EC016CE576E0CE010E94FA8FD3
:104F1000892B61F48FEFF401808360916D027091B1
:104F20006E0280E090E00E940E90EC01209709F460
:104F300024C168E576E0CE010E94FA8F892B19F42E
:104F4000FD2DF160DF2E64E576E0CE010E94FA8F40
:104F5000892B19F48D2D8460D82E61E576E0CE0181
:104F60000E94FA8F892B19F4ED2DE260DE2E6FE49A
:104F700076E0CE010E94FA8F892B19F4FD2DF8609E
:104F8000DF2E6CE476E0CE010E94FA8F892B19F4B3
:104F90008D2D8061D82E66E476E0CE010E94FA8FD6
:104FA000892B19F4ED2DE062DE2E60E476E0CE016F
:104FB0000E94FA8F892B19F4FD2DF064DF2E6DE32A
:104FC00076E0CE010E94FA8F892B19F48D2D80682E
:104FD000D82E68E376E0CE010E94FA8F892B19F46F
:104FE000EE2DE160EE2E61E376E0CE010E94FA8FB5
:104FF000892B19F4FE2DF260EF2E6EE276E0CE01E1
:105000000E94FA8F892B19F48E2D8460E82E69E2B4
:1050100076E0CE010E94FA8F892B19F4EE2DE8601C
:10502000EE2E62E276E0CE010E94FA8F892B19F40F
:10503000FE2DF061EF2E6BE176E0CE010E94FA8F3B
:10504000892B19F48E2D8062E82E67E176E0CE017F
:105050000E94FA8F892B19F4EB2DE460BE2E64E1D7
:1050600076E0CE010E94FA8F892B19F4FE2DF064B0
:10507000EF2E6FE076E0CE010E94FA8F892B19F4B3
:105080008E2D8068E82E6CE076E0CE010E94FA8FCB
:10509000892B09F4016069E076E0CE010E94FA8F65
:1050A000892B09F4026066E076E0CE010E94FA8F57
:1050B000892B09F4046062E076E0CE010E94FA8F49
:1050C000892B09F408606EEF75E0CE010E94FA8F1B
:1050D000892B09F400616AEF75E0CE010E94FA8F16
:1050E000892B09F4006266EF75E0CE010E94FA8F09
:1050F000892B09F4006464EF75E0CE010E94FA8FF9
:10510000892B09F4006861EF75E0CE010E94FA8FE7
:10511000892B09F4116069EE75E0CE010E94FA8FC7
:10512000892B09F4126060EE75E0CE010E94FA8FBF
:10513000892B09F4146067ED75E0CE010E94FA8FA7
:10514000892B09F4186064ED75E0CE010E94FA8F96
:10515000892B09F410616EEC75E0CE010E94FA8F84
:10516000892B09F4106263EC75E0CE010E94FA8F7E
:10517000892B09F0D2CE1064D0CE2D2D3E2DA80162
:105180006B2D70E080E090E0DF91CF911F910F9147
:10519000EF90DF90BF909F908F9008955F926F92F5
:1051A0007F928F929F92AF92BF92CF92DF92EF92B7
:1051B000FF920F931F93CF93DF93782EC1E1DBE132
:1051C00000E010E0FDEBEF2EF5E0FF2E8170582E91
:1051D000872D8270682EA8EACA2EA5E0DA2EB0EBE1
:1051E000AB2EB5E0BB2E8EEA882E85E0982E772078
:1051F00051F01F930F93FF92EF920E94D9900F905E
:105200000F900F900F905520A1F089858F9388857E
:105210008F93BF92AF920E94D9900F900F900F90F2
:105220000F906620C1F09F928F920E94D9900F90AC
:105230000F90662081F0DF92CF920E94D990288152
:1052400039814A815B816C817D818E819F810E9441
:10525000C8230F900F900E94670B0F5F1F4F2A9675
:105260000430110521F6DF91CF911F910F91FF902E
:10527000EF90DF90CF90BF90AF909F908F907F90F6
:105280006F905F90089588E995E09F938F930E94B7
:10529000D9900E94312088EF9AE19F938F9380E903
:1052A00095E09F938F930E94D9908CE895E09F930F
:1052B0008F930E94D99080E00E940F2287E895E0AA
:1052C0009F938F930E94D9900E94E60F80910720B0
:1052D0002DB73EB7265F3F4F0FB6F8943EBF0FBEC7
:1052E0002DBF80FF05C041E061E081E00E94901188
:1052F0000E943520809153021F928F938EE795E094
:105300009F938F930E94D9908091AB091F928F93A6
:1053100085E795E09F938F930E94D99080917F02BB
:105320008F9380917E028F9380917D028F938091E5
:105330007C028F9387E695E09F938F930E94D9908C
:105340001F9280E48F938FE495E09F938F930E9448
:10535000D99080919D281F928F9380919C281F92B5
:105360008F938CE395E09F938F930E94D9908091C7
:1053700052021F928F9383E395E09F938F930E9435
:10538000D9908091540290915502A0915602B0910B
:1053900057022DB73EB7245E3F4F0FB6F8943EBF7D
:1053A0000FBE2DBF96FF03C08AE895E002C08DE8CE
:1053B00095E09F938F9389E295E09F938F930E944E
:1053C000D99083E00E94CE280F900F900F900F90FD
:1053D0001D9B03C08AE895E002C08DE895E09F938D
:1053E0008F938DE195E09F938F930E94D99083E1F5
:1053F00095E09F938F930E94D990809154020F90D3
:105400000F900F900F900F900F9081FF09C08DE0CB
:1054100095E09F938F930E94D9900F900F9013C0A7
:1054200080FF03C08AE895E002C08DE895E09F9375
:105430008F9389E095E09F938F930E94D9900F906E
:105440000F900F900F908091540290915502A0916F
:105450005602B091570288279078892B8A2B8B2B84
:1054600019F08AE895E002C08DE895E09F938F934C
:1054700080E095E09F938F930E94D99089EF94E00C
:105480009F938F930E94D9906091AF097091B0095A
:1054900080E090E00E943F220E94670B0F900F90E7
:1054A0000F900F900F900F90779903C08AE895E0C6
:1054B00002C08DE895E09F938F9380EF94E09F93D7
:1054C0008F930E94D9900E940A090E94B10A9F936B
:1054D0008F937F936F9382EE94E09F938F930E94BC
:1054E000D9900E946B0A9F938F937F936F9384ED63
:1054F00094E09F938F930E94D99081E090E00E9466
:10550000EB208091722890917328A0917428B0911B
:105510007528BF93AF939F938F9386EC94E09F93EE
:105520008F930E94D990809187288F9380918628AD
:105530008F93809185288F93809184288F9382EB1D
:1055400094E09F938F930E94D990809176289091B8
:105550007728A0917828B0917928BF93AF939F9333
:105560008F9384EA94E09F938F930E94D9908DB794
:105570009EB782960FB6F8949EBF0FBE8DBF8091E6
:105580008B288F9380918A288F93809189288F937D
:10559000809188288F9380E994E09F938F930E9455
:1055A000D99061E070E080E090E00E94700B0F9075
:1055B0000F900F900F900F900F9061E070E081E0DE
:1055C00090E00C94700BF894E0E0F0E081E28093BE
:1055D00057008491E2E0F0E041E2409357004491AB
:1055E000E4E0F0E091E290935700E49190E0A0E0D5
:1055F000B0E0DC019927882750E060E070E0762F6A
:10560000652F542F4427840F951FA61FB71F8E0F99
:10561000911DA11DB11D8093B21B9093B31BA0934C
:10562000B41BB093B51B78940895CF93DF93CDB797
:10563000DEB761970FB6F894DEBF0FBECDBF48E26C
:1056400050E06AE170E081E19BE10E942D9220919F
:10565000111B3091121B4091131B5091141B609130
:10566000151B7091161B8091171B9091181BAFEFA3
:105670000E94488C09F05DC08DE48093111B80E886
:105680008093121B84E08093131B1092141B1092C2
:10569000151B1092161B1092171B1092181B8CE3EF
:1056A00090E090931A1B8093191B10921B1B109271
:1056B0001C1B10921D1B10921E1B10921F1B109280
:1056C000201B1092211B1092221B1092241B10925F
:1056D000231B1092251B1092261B1092271B109241
:1056E000281B1092291B10922A1B10922B1B109220
:1056F0002C1B10922E1B10922D1B10922F1B109200
:10570000301B1092311B1092321B1092331B1092DF
:10571000341B1092351B1092361B1092381B1092BE
:10572000371B48E250E06AE170E081E19BE10E94B2
:105730004B9242E050E066E170E0CE010F960E948D
:105740002D928F8598898F3F2FEF9207A9F48AE0D9
:1057500090E4A0E0B0E08093540290935502A093AF
:105760005602B093570242E050E066E170E084E5F3
:1057700092E00E944B920AC0A0E0B0E080935402F5
:1057800090935502A0935602B093570242E050E026
:1057900062E570E0CE010F960E942D928F85988968
:1057A0008F3F2FEF920769F41092B0091092AF0962
:1057B00042E050E062E570E08FEA99E00E944B928F
:1057C00004C09093B0098093AF0949E050E06AE0CB
:1057D00070E08CE898E20E942D920E94A80C44E0B0
:1057E00050E066E470E0CE010B960E942D928B850E
:1057F0009C85AD85BE8544E050E066E470E08F3F57
:105800009F4FAF4FBF4F29F484E792E00E944B9225
:1058100004C084E792E00E942D9244E050E062E4EC
:1058200070E0CE010B960E942D928B859C85AD85F4
:10583000BE8544E050E062E470E08F3F9F4FAF4F81
:10584000BF4F29F480E792E00E944B9204C080E7AA
:1058500092E00E942D9244E050E06AE470E0CE01B4
:105860000B960E942D928B859C85AD85BE8544E06C
:1058700050E06AE470E08F3F9F4FAF4FBF4F29F475
:1058800088E792E00E944B9204C088E792E00E9471
:105890002D9241E050E065E170E0CE0141960E941A
:1058A0002D92898941E050E065E170E08F3F29F455
:1058B0008BEA99E00E944B9204C08BEA99E00E9427
:1058C0002D9241E050E064E170E0CE0141960E94EB
:1058D0002D92898941E050E064E170E08F3F29F426
:1058E00083E592E00E944B9204C083E592E00E941F
:1058F0002D9241E050E063E170E0CE0141960E94BC
:105900002D92898941E050E063E170E08F3F29F4F6
:1059100082E592E00E944B9204C082E592E00E94F0
:105920002D924AE050E060E070E0CE0101960E94C6
:105930002D9289814AE050E060E070E08F3F29F4C9
:1059400088EF9AE10E944B9204C088EF9AE10E948E
:105950002D9244E050E06EE470E0CE010B960E9480
:105960002D928B859C85AD85BE8544E050E06EE42C
:1059700070E08F3F9F4FAF4FBF4F29F48CE792E00D
:105980000E944B9204C08CE792E00E942D92619697
:105990000FB6F894DEBF0FBECDBFDF91CF91089553
:1059A000CF92DF92EF92FF9260916D0270916E0242
:1059B00080E090E00E940E9061E975E00E942290E4
:1059C000892B09F00BC18DE48093111B80E8809333
:1059D000121B84E08093131B1092141B1092151B52
:1059E0001092161B1092171B1092181B8CE390E05C
:1059F00090931A1B8093191B10921B1B10921C1B57
:105A000010921D1B10921E1B10921F1B1092201B28
:105A10001092211B1092221B1092241B1092231B08
:105A20001092251B1092261B1092271B1092281BE8
:105A30001092291B10922A1B10922B1B10922C1BC8
:105A400010922E1B10922D1B10922F1B1092301BA8
:105A50001092311B1092321B1092331B1092341B88
:105A60001092351B1092361B1092381B1092371B68
:105A700048E250E06AE170E081E19BE10E944B92D4
:105A80008AE090E4A0E0B0E0809354029093550245
:105A9000A0935602B093570242E050E066E170E0F6
:105AA00084E592E00E944B921092B0091092AF09E7
:105AB00042E050E062E570E08FEA99E00E944B928C
:105AC00042E2C42EDD24DA944CECE42E4BE3F42EB7
:105AD000C0927402D0927502E0927602F092770240
:105AE00044E050E066E470E084E792E00E944B926C
:105AF000C0927002D0927102E0927202F092730230
:105B000044E050E062E470E080E792E00E944B9253
:105B100087ED94E3AFEEBCE3809378029093790233
:105B2000A0937A02B0937B0244E050E06AE470E014
:105B300088E792E00E944B928AE999E9A9E1B0E4F2
:105B400080937C0290937D02A0937E02B0937F02AB
:105B500044E050E06EE470E08CE792E00E944B92EB
:105B60001092AB0980E00E94596841E050E065E185
:105B700070E08BEA99E00E944B928AE18093530295
:105B80000E94006741E050E064E170E083E592E04C
:105B90000E944B928FE08093520241E050E063E11B
:105BA00070E082E592E00E944B928AE0E8EFFAE131
:105BB000DF011D928A95E9F74AE050E060E070E06D
:105BC000CF010E944B9281E00E940F2280E090E082
:105BD000FF90EF90DF90CF900C94BC0CFF90EF9073
:105BE000DF90CF9008952F923F924F925F926F92E5
:105BF0007F928F929F92AF92BF92CF92DF92EF925D
:105C0000FF920F931F93CF93DF93CDB7DEB72B9700
:105C10000FB6F894DEBF0FBECDBF9B878A874A01BF
:105C2000FC0180819181892B11F00C94C23F60911D
:105C30006D0270916E02CA010E940E9060E470E0E5
:105C4000C4010E944190009759F4609157317091BE
:105C500058318AE090E00E94959081E00C94C73F13
:105C60008130910561F4F401B0801B2D110F110BEF
:105C7000012F412E512E612E712EA12EBCC08230DB
:105C80009105B9F4F4018081992787FD9095982FAB
:105C900088272181820F911D27FD9A95B82E192FF3
:105CA000092F000F000B402E502E602E702EA02EBC
:105CB000A2C083309105B1F5F4012081922F990F94
:105CC000990B392F492F592F692F792F892F00E1EF
:105CD0000E94EA8B19012A013B01B82FA92F2181CB
:105CE000922F990F990B392F492F592F692F792FFF
:105CF000892F08E00E94EA8B59016A017B018C011F
:105D00009101A201B3018B2F9A2F0E94218CA280B6
:105D10001A2D110F110BB12EC12ED12EE12EF12E05
:105D2000012F55C004970CF45DC0F4012081922F1F
:105D3000990F990B392F492F592F692F792F892FB7
:105D400008E10E94EA8B19012A013B01B82FA92F13
:105D50002181922F990F990B392F492F592F692F94
:105D6000792F892F00E10E94EA8B59016A017B019A
:105D70008C019101A201B3018B2F9A2F0E94218CDB
:105D8000A3801A2D110F110BB12EC12ED12EE12E91
:105D9000F12E012F0E94218C19012A013B01B82FFD
:105DA000A92F2281922F990F990B392F492F592F03
:105DB000692F792F892F08E00E94EA8B59016A0127
:105DC0007B018C019101A201B3018B2F9A2F0E94BC
:105DD000218CB22E132F042F452E562E672E782E8F
:105DE000A92E09C07AE0B72E10E000E0412C512C1A
:105DF000612C712CA12C0E94670B2B2D312F402F71
:105E0000542D652D762D872D9A2D2736FFE63F07D9
:105E1000FCE64F075105610571058105910511F4F7
:105E20000C94CF392736EFE63E07ECE64E075105D6
:105E3000610571058105910511F008F093C12936BE
:105E4000F2E73F074105510561057105810591059F
:105E500011F40C94EC3C2936E2E73E07410551056C
:105E6000610571058105910511F008F0A3C0253683
:105E7000F4E63F074105510561057105810591056E
:105E800009F480C52536E4E63E0741055105610564
:105E900071058105910509F0A8F5A6E70E94488CD7
:105EA00009F4F1C70E94488C09F060F4A8E60E944A
:105EB000488C09F4ADC5A5E70E94488C09F4CDC70C
:105EC0000C94C03F2B2D312F402F542D652D762D56
:105ED000872D9A2D2A33F6E23F07410551056105CA
:105EE00071058105910509F41EC32436314641052B
:105EF0005105610571058105910511F40C94653D0D
:105F00000C94C03F2B2D312F402F542D652D762D15
:105F1000872D9A2D2737FFE63F074105510561057B
:105F200071058105910511F40C94103B2737EFE6BC
:105F30003E0741055105610571058105910509F08F
:105F4000C0F42436F9E63F074105510561057105A6
:105F50008105910509F45AC725363E46410551058C
:105F6000610571058105910511F40C94443B0C9475
:105F7000C03F2B2D312F402F542D652D762D872D91
:105F80009A2D2333F1E73F0741055105610571055E
:105F90008105910511F40C94653D25363247410584
:105FA0005105610571058105910511F40C940E3CB4
:105FB0000C94C03F2B2D312F402F542D652D762D65
:105FC000872D9A2D2837F4E63F07F1E64F07510554
:105FD000610571058105910509F4B5C22837E4E62C
:105FE0003E07E1E64E075105610571058105910502
:105FF00011F008F050C02837F4E73F07410551057C
:10600000610571058105910509F48DC22837E4E722
:106010003E0741055105610571058105910509F0AE
:10602000C8F42337F2E73F074105510561057105C3
:106030008105910511F40C943D3D2337334741050B
:106040005105610571058105910511F40C94513DCF
:106050000C94C03F2B2D312F402F542D652D762DC4
:10606000872D9A2D2133F4E63F07F1E64F075105BE
:10607000610571058105910509F469C2233634462D
:1060800041465105610571058105910511F40C9496
:10609000653D0C94C03F2B2D312F402F542D652D85
:1060A000762D872D9A2D2336FDE63F07F8E64F071C
:1060B0005105610571058105910509F46CC223360E
:1060C000EDE63E07E8E64E075105610571058105DD
:1060D000910509F0C8F42236F5E63F07F4E64F07CC
:1060E0005105610571058105910509F44BC42237FD
:1060F000324745465105610571058105910511F449
:106100000C94693A0C94C03F2B2D312F402F542D05
:10611000652D762D872D9A2D2336F2E33F07F9E67C
:106120004F075105610571058105910509F42FC2DD
:106130002436E3E63E07ECE64E075105610571059E
:106140008105910511F40C94CC392D36354748461C
:106150005105610571058105910511F00C94C03F51
:106160000C947B3D2B2D312F402F542D652D762DFA
:10617000872D9A2D2136EDE63E07E5E74E07E8E646
:106180005E07610571058105910511F40C942E3BA4
:106190002136FDE63F07F5E74F07F8E65F076105A3
:1061A00071058105910511F008F0DAC02437E8E7A0
:1061B0003E07E4E74E07510561057105810591052C
:1061C00009F4CDC62437F8E73F07F4E74F07510538
:1061D000610571058105910511F008F055C0213365
:1061E000E1E33E07E1E74E075105610571058105D1
:1061F000910511F40C94AA3A2133F1E33F07F1E73A
:106200004F075105610571058105910509F0D0F42D
:106210002537E3E63E07EDE64E07510561057105BA
:106220008105910511F40C94AA3A2033314341477A
:106230005105610571058105910511F40C94693AC8
:106240000C94C03F2B2D312F402F542D652D762DD2
:10625000872D9A2D2037E5E63E07E2E74E075105E8
:10626000610571058105910511F40C940E3C2C36E5
:10627000344744475105610571058105910511F4C5
:106280000C94E93E0C94C03F2B2D312F402F542D00
:10629000652D762D872D9A2D2936ECE63E07E1E611
:1062A0004E07E3E65E07610571058105910509F476
:1062B000A7C12936FCE63F07F1E64F07F3E65F0783
:1062C000610571058105910509F0E0F42437E4E6E4
:1062D0003E07E7E74E075105610571058105910508
:1062E00011F40C94373F24373F464F465246610520
:1062F00071058105910511F00C94C03F0C940000CC
:106300000C94C23F2B2D312F402F542D652D762D0F
:10631000872D9A2D2633E9E63E07E5E74E07E5E6A9
:106320005E07610571058105910509F475C3203784
:10633000FCE63F07F5E64F07F8E65F0761057105E4
:106340008105910509F464C32E363146484653460B
:10635000610571058105910509F4D5C50C94C03F0F
:106360002B2D312F402F542D652D762D872D9A2DD5
:106370002437F3E73F07F5E64F07F2E75F076105CC
:1063800071058105910511F40C94BE3B2437E3E7B8
:106390003E07E5E64E07E2E75E0761057105810508
:1063A000910511F008F055C02337F2E73F07F7E7F2
:1063B0004F07F0E75F07610571058105910511F44D
:1063C0000C94C13B2337E2E73E07E7E74E07E0E7DF
:1063D0005E07610571058105910509F0C8F4223752
:1063E000F7E73F07F0E74F075F0761057105810594
:1063F000910509F4D4C0233735464247504761051B
:1064000071058105910511F40C942B3E0C94C03F4D
:106410002B2D312F402F542D652D762D872D9A2D24
:106420002436FDE63F07F3E64F07F2E75F07610515
:1064300071058105910509F4FAC321363C464546AC
:106440005247610571058105910509F402C30C9459
:10645000C03F2B2D312F402F542D652D762D872DAC
:106460009A2D2437F2E73F07F1E64F07F5E75F077C
:10647000610571058105910509F43EC42437E2E701
:106480003E07E1E64E07E5E75E0761057105810518
:10649000910509F0C8F42437F3E73F07F5E64F0705
:1064A000F4E75F07610571058105910509F482C56F
:1064B00027373047484754476105710581059105E5
:1064C00009F4F7C40C94C03F2B2D312F402F542DCD
:1064D000652D762D872D9A2D2F36FCE63F07FFE59B
:1064E0004F07F6E75F07610571058105910509F41E
:1064F00049C32C36E1E63E07E4E74E07E8E75E07CE
:10650000610571058105910511F40C94B33E2237A4
:10651000374640475547610571058105910511F0E2
:106520000C94C03F16C783E080937A2810927C2891
:1065300010927B284AE758E262E184E392E00E94ED
:1065400072520C94C23F0E9474150C94C23F21E019
:1065500042E161E080ED0E949D5F21E042E161E067
:1065600080ED0E949D5F21E042E161E080ED0E94AC
:106570009D5F21E042E161E080ED0E949D5F21E0AE
:1065800042E161E080ED0E949D5F0C94C23F0E9459
:10659000E60F0C94C23F0E94EC150C94C23F609130
:1065A0006D0270916E0280E090E00E940E908C016E
:1065B0006AE875E00E942290892B19F477980C9470
:1065C000C23F6DE875E0C8010E942290892B19F442
:1065D000779A0C94C23F779903C08AE895E002C08D
:1065E0008DE895E09F938F938AE794E09F938F9334
:1065F0000E94D9900F900F900F900F900C94C23F73
:1066000060916D0270916E0280E090E00E940E90A9
:106610008C0164E575E00E942290892B09F077C017
:1066200060916D0270916E0280E090E00E940E9089
:106630008C01009711F40C94C23F68E975E00E9448
:106640002290892BB1F482E29FEFACECBBE3809304
:10665000740290937502A0937602B093770244E09F
:1066600050E066E470E084E792E00E944B920C9464
:10667000C23F6EE975E0C8010E942290892BB1F4F7
:1066800082E29FEFACECBAE38093740290937502C0
:10669000A0937602B093770244E050E066E470E0A5
:1066A00084E792E00E944B920C94C23FC8010E9482
:1066B000F88E2B013C0120E030E0A9010E94978672
:1066C0008823D9F081E00E94080A9B01AC01C30134
:1066D000B2010E949B86609374027093750280934E
:1066E00076029093770244E050E066E470E084E73D
:1066F00092E00E944B920C94C23F86EE92E09F93F0
:106700008F930E94D9900F900F900C94C23F67E531
:1067100075E0C8010E942290892B09F077C0609132
:106720006D0270916E0280E090E00E940E908C01EC
:10673000009711F40C94C23F68E975E00E94229022
:10674000892BB1F482E29FEFACECBBE38093700243
:1067500090937102A0937202B093730244E050E0F0
:1067600062E470E080E792E00E944B920C94C23F9A
:106770006EE975E0C8010E942290892BB1F482E293
:106780009FEFACECBAE38093700290937102A093F8
:106790007202B093730244E050E062E470E080E77C
:1067A00092E00E944B920C94C23FC8010E94F88E66
:1067B0002B013C0120E030E0A9010E94978688234C
:1067C000D9F082E00E94080A9B01AC01C301B2012A
:1067D0000E949B8660937002709371028093720294
:1067E0009093730244E050E062E470E080E792E04E
:1067F0000E944B920C94C23F89ED92E09F938F933D
:106800000E94D9900F900F900C94C23F6FE475E0F6
:10681000C8010E942290892B09F073C060916D021B
:1068200070916E0280E090E00E940E908C010097C3
:1068300011F40C94C23F68E975E00E942290892B04
:10684000B1F487ED94E3AFEEBCE3809378029093CC
:106850007902A0937A02B0937B0244E050E06AE4AC
:1068600070E088E792E00E944B920C94C23F6EE980
:1068700075E0C8010E942290892B51F48AEC92E0C5
:106880009F938F930E94D9900F900F900C94C23FCA
:10689000C8010E94F88E2B013C0120E030E0A901E4
:1068A0000E949786882319F180E00E94080A4B0114
:1068B0005C0121EE3AE744E95EE3C301B2010E94C4
:1068C000D085A50194010E949B8660937802709305
:1068D000790280937A0290937B0244E050E06AE46C
:1068E00070E088E792E00E944B920C94C23F8DEBDF
:1068F00092E09F938F930E94D9900F900F900C94E9
:10690000C23F0E94570A9F938F937F936F9386EBAA
:1069100092E09F938F930E94D99082E00E94080A90
:106920002091700230917102409172025091730275
:106930000E941889162F072FF82EE92E81E00E9459
:10694000080AEF92FF920F931F93209174023091E7
:10695000750240917602509177020E9418899F93A8
:106960008F937F936F938AEA92E09F938F930E9415
:10697000D9900E94670B0FB6F894DEBF0FBECDBF53
:106980000C94C23F60916D0270916E0280E090E0C5
:106990000E940E900097C1F00E942D232091AF0914
:1069A0003091B0098217930709F19093B009809351
:1069B000AF0942E050E062E570E08FEA99E00E94A2
:1069C0004B9283E794E002C08CE694E09F938F9310
:1069D0000E94D9906091AF097091B00980E090E079
:1069E0000E943F220E94670B0F900F9081E694E077
:1069F0009F938F930E94D9906FEF7FEF80E090E09C
:106A00000E943F220E94670B0F900F900C94C23F90
:106A10000E94461F0C94C23FF4018481843329F400
:106A200040E061E080E00E94901180916F02882335
:106A300011F40C94C23F1F928F938EE594E09F93C4
:106A40008F930E94D9900F900F900F900F900C94FD
:106A5000C23FF4018481893709F080C060916D02E2
:106A600070916E0280E090E00E940E908C016AE8C6
:106A700075E00E942290892B51F4809154029091EC
:106A80005502A0915602B0915702906410C06DE873
:106A900075E0C8010E942290892BD1F480915402A4
:106AA00090915502A0915602B09157029F7B80931E
:106AB000540290935502A0935602B093570242E0BD
:106AC00050E066E170E084E592E00E944B9246C09F
:106AD00063EA75E0C8010E942290892B21F580911C
:106AE000101B8F9380910F1B8F9380910E1B8F93A0
:106AF00080910D1B8F9380910C1B8F9380910B1BAA
:106B00008F9380910A1B8F938091091B8F938FE73E
:106B100092E09F938F930E94D9900FB6F894DEBFB6
:106B20000FBECDBF1BC08091540290915502A09121
:106B30005602B091570296FF03C08AE895E002C062
:106B40008DE895E09F938F938BE792E09F938F93CF
:106B50000E94D9900F900F900F900F9080916F022C
:106B6000882311F40C94C23F1F928F938BE594E01D
:106B70009F938F930E94D9900F900F900F900F903A
:106B80000C94C23FF40184818737E9F560916D026E
:106B900070916E0280E090E00E940E900097D9F014
:106BA0000E94F88E2B013C0120E030E0A9010E94F8
:106BB0009786882381F040927C0250927D026092F9
:106BC0007E0270927F0244E050E06EE470E08CE759
:106BD00092E00E944B9280917F028F9380917E027F
:106BE0008F9380917D028F9380917C028F938DE6AD
:106BF00092E09F938F930E94D9900F900F900F90E7
:106C00000F900F900F9080916F02882311F40C94D5
:106C1000C23F1F928F9388E594E09F938F930E94C9
:106C2000D9900F900F900F900F900C94C23F6091ED
:106C30006D0270916E0280E090E00E940E908C01D7
:106C40006AE875E00E9422904090540250905502EC
:106C50006090560270905702892B31F4689457F86F
:106C600066246A94762C0BC06DE875E0C8010E941A
:106C70002290892BA9F4E89457F86624772440924F
:106C8000540250925502609256027092570242E0AE
:106C900050E066E170E084E592E00E944B9218C0FB
:106CA0004424F0E85F2245284628472819F08AE85E
:106CB00095E002C08DE895E09F938F9389E692E07E
:106CC0009F938F930E94D9900F900F900F900F90E9
:106CD00080916F02882311F40C94C23F1F928F930E
:106CE00085E594E09F938F930E94D9900F900F9029
:106CF0000F900F900C94C23F60916D0270916E02E4
:106D000080E090E00E940E905C0169EA75E00E94CC
:106D10002290892B11F489E108C06DEA75E0C50164
:106D20000E942290892B49F480E18093C400109244
:106D3000C50082E08093C00055C061EB75E0C501DD
:106D40000E942290892B11F488E0EFCF66EB75E06A
:106D5000C5010E942290892B39F06BEB75E0C501CB
:106D60000E942290892B11F483E0DFCF8091C40030
:106D7000893141F484E692E09F938F930E94D990E9
:106D80000F900F908091C400803141F48FE592E024
:106D90009F938F930E94D9900F900F908091C40081
:106DA000883041F489E592E09F938F930E94D990B7
:106DB0000F900F908091C400833041F483E592E0FE
:106DC0009F938F930E94D9900F900F908091C40051
:106DD000883041F48DE492E09F938F930E94D99084
:106DE0000F900F9080916F02882311F40C94C23F92
:106DF0001F928F9382E594E09F938F930E94D99086
:106E00000F900F900F900F900C94C23F60916D0205
:106E100070916E0280E090E00E940E9068E975E04B
:106E20000E942290892B11F481E001C080E00E9431
:106E30000F2280916F02882311F40C94C23F1F929D
:106E40008F938FE494E09F938F930E94D9900F903B
:106E50000F900F900F900C94C23F0E9435208091AC
:106E60006F02882311F40C94C23F1F928F938CE41D
:106E700094E09F938F930E94D9900F900F900F9062
:106E80000F900C94C23F0E94312080916F028823A2
:106E900011F40C94C23F1F928F9389E494E09F9366
:106EA0008F930E94D9900F900F900F900F900C9499
:106EB000C23F60916D0270916E0280E090E00E948E
:106EC0000E900E94FC8E803170F48093AB090E947A
:106ED000596841E050E065E170E08BEA99E00E947A
:106EE0004B920C94C23F8091AB091F928F9383E425
:106EF00092E09F938F930E94D9900F900F900F90E4
:106F00000F900C94C23F60916D0270916E0280E010
:106F100090E00E940E900E94FC8E95EF980F9031A9
:106F200070F4809353020E94006741E050E064E1F6
:106F300070E083E592E00E944B920C94C23F8091F6
:106F400053021F928F938AE392E09F938F930E9444
:106F5000D9900F900F900F900F900C94C23F6091BA
:106F60006D0270916E0280E090E00E940E9000979A
:106F700089F04AE050E0BC0188EF9AE10E9432902B
:106F80004AE050E060E070E088EF9AE10E944B92A6
:106F90000C94C23F88EF9AE19F938F9380EC95E029
:106FA0009F938F930E94C7900F900F900F900F9018
:106FB0000C94C23F60916D0270916E0280E090E08F
:106FC0000E940E905C016CED73E00E942290892B70
:106FD000D9F4219A8091540290915502A0915602C1
:106FE000B091570280618093540290935502A09310
:106FF0005602B093570242E050E066E170E084E54B
:1070000092E00E944B92BEC768E575E0C5010E9400
:107010002290892BD9F4229A8091540290915502A2
:10702000A0915602B09157028062809354029093CF
:107030005502A0935602B093570242E050E066E139
:1070400070E084E592E00E944B929CC76EEB73E087
:10705000C5010E942290892BD9F4239A8091540271
:1070600090915502A0915602B0915702806480938E
:10707000540290935502A0935602B093570242E0F7
:1070800050E066E170E084E592E00E944B927AC79E
:107090006BEF74E0C5010E942290892BD9F4239AEA
:1070A0008091540290915502A0915602B0915702DE
:1070B00080688093540290935502A0935602B09337
:1070C000570242E050E066E170E084E592E00E9401
:1070D0004B9258C767E579E0C5010E942290892B41
:1070E00071F581E080931E2481E19BE1909320243F
:1070F00080931F2410922224109221248091540204
:1071000090915502A0915602B091570291608093E0
:10711000540290935502A0935602B093570242E056
:1071200050E066E170E084E592E00E944B924EE10F
:1071300054E262E184E392E00E94725223C765EE5A
:1071400073E0C5010E942290892B11F5E1E4FBE177
:10715000119211922BE1E136F207D1F7809154029E
:1071600090915502A0915602B0915702926080937F
:10717000540290935502A0935602B093570242E0F6
:1071800050E066E170E084E592E00E944B92FAC61E
:107190006DE875E0C5010E94229040915402509123
:1071A00055026091560270915702892BC1F44F70BD
:1071B0005C7F409354025093550260935602709343
:1071C00057022B9A42E050E066E170E084E592E0DD
:1071D0000E944B92809183280E941567D3C644FF7A
:1071E00003C08AE895E002C08DE895E09F938F93F5
:1071F0008FE292E09F938F930E94D99080915402E6
:107200000F900F900F900F9085FF03C08AE895E0D4
:1072100002C08DE895E09F938F9384E292E09F9364
:107220008F930E94D990809154020F900F900F90ED
:107230000F9086FF03C08AE895E002C08DE895E0D4
:107240009F938F9389E192E09F938F930E94D990AF
:10725000809154020F900F900F900F9087FF03C002
:107260008AE895E002C08DE895E09F938F938EE0C9
:1072700092E09F938F930E94D990809154029091B5
:107280005502A0915602B09157020F900F900F90A7
:107290000F9090FF03C08AE895E002C08DE895E06A
:1072A0009F938F9383E092E09F938F930E94D99056
:1072B0008091540290915502A0915602B0915702CC
:1072C0000F900F900F900F9091FF03C08AE895E008
:1072D00002C08DE895E09F938F9388EF91E09F9394
:1072E0008F930E94D9908091540290915502A09161
:1072F0005602B09157020F900F900F900F9091FF90
:1073000041C688EC95E00E94FD9051E4A52E5BE11A
:10731000B52E0BE010E060ED862E65E0962EF501AF
:1073200080819181F2E0AF0EB11C9F938F931F93E8
:107330000F939F928F920E94C7900F5F1F4F0F90E5
:107340000F900F900F900F900F900B31110539F7A0
:1073500019C685E494E09F938F930E94D990809101
:107360006F020F900F90882361F01F928F9382E439
:1073700094E09F938F930E94D9900F900F900F905D
:107380000F9088E10FB6F89480936000109260002F
:107390000FBE0C94007CF6C50E944E5FF3C5609151
:1073A0006D0270916E0280E090E00E940E908C0160
:1073B0006AE875E00E942290892BE9F40E94FF653B
:1073C0008091540290915502A0915602B0915702BB
:1073D0008D7F81608093540290935502A093560252
:1073E000B093570242E050E066E170E084E592E03D
:1073F0000E944B92C7C56DE875E0C8010E942290BB
:10740000892BE1F40E94B765809154029091550256
:10741000A0915602B09157028C7F809354029093B2
:107420005502A0935602B093570242E050E066E145
:1074300070E084E592E00E944B92A4C56BED75E08C
:10744000C8010E942290892BE9F40E94B7658091BF
:10745000540290915502A0915602B09157028E7F2E
:1074600082608093540290935502A0935602B09389
:10747000570242E050E066E170E084E592E00E944D
:107480004B9280C58091540281FF0FC08BED95E037
:107490009F938F9384EF91E09F938F930E94D99055
:1074A0000F900F900F900F906DC580FF03C08AE87A
:1074B00095E002C08DE895E09F938F9380EF91E077
:1074C0009F938F930E94D9900F900F900F900F90E1
:1074D00059C580911C248F9380911B248F93809198
:1074E0001A248F93809119248F93809118248F935D
:1074F000809117248F93809116248F938091152467
:107500008F93809114248F93809113248F93809173
:1075100012248F93809111248F938FE194E09F9395
:107520008F930E94D99080916F020FB6F894DEBFBE
:107530000FBECDBF882309F425C51F928F938CE120
:1075400094E09F938F930E94D9900F900F900F908B
:107550000F9018C5F89481E090E029E0FC01209399
:107560005700C895E02C80E090E0FC012093570084
:10757000C895F02C7894F89483E090E0FC01209377
:107580005700C895002D82E090E0FC012093570041
:10759000C895102D78948091B51B8F938091B41B62
:1075A0008F938091B31B8F938091B21B8F9322E1B5
:1075B00034E03F932F930E94D9901F92EF921F9235
:1075C000FF921F920F931F921F938BEE93E09F9356
:1075D0008F930E94D9900E94CF20809166001F92C5
:1075E0008F938FED93E09F938F930E94D9900E9489
:1075F000670B80916F020FB6F894DEBF0FBECDBF50
:10760000882309F4BFC41F928F938CED93E09F935E
:107610008F930E94D9900F900F900F900F90B2C44B
:1076200060E070E080E090E00E94700B60E070E04D
:1076300081E090E00E94700B80916F02882309F432
:10764000A1C41F928F9389ED93E09F938F930E9423
:10765000D9900F900F900F900F9094C40E94091F23
:107660000E94670B80916F02882309F48BC41F92DC
:107670008F9386ED93E09F938F930E94D9900F9004
:107680000F900F900F907EC460916D0270916E020A
:1076900080E090E00E940E9060EE75E00E942290E3
:1076A000892B31F5F89486EE99E00E945F535C01D6
:1076B000009769F0C5010F960E946356B50184E0FA
:1076C00092E00E941953C5010E940754F0CF86EE44
:1076D00099E00E94EC53892B29F086EE99E00E94F4
:1076E0009853F5CF86EE99E00E945B53789434C0AE
:1076F00086EE99E00E945F535C0106EE15E0A1144E
:10770000B10451F1F50186811F928F9380851F92FC
:107710008F9385811F928F9381851F928F9387818D
:107720001F928F9384811F928F9383811F928F93D7
:1077300082811F928F9382851F928F931F930F9345
:107740000E94C790C5010E9407545C010FB6F894CF
:10775000DEBF0FBECDBFD3CF80916F02882309F467
:1077600011C41F928F9383ED93E09F938F930E9498
:10777000D9900F900F900F900F9004C40E94D02CBE
:1077800001C460916D0270916E0280E090E00E94F1
:107790000E908C0165E276E00E942290892BD1F454
:1077A0008091540290915502A0915602B0915702D7
:1077B000977F8093540290935502A0935602B09302
:1077C000570242E050E066E170E084E592E00E94FA
:1077D0004B92D8C36EE975E0C8010E942290892BB4
:1077E000D1F48091540290915502A0915602B0912B
:1077F000570298608093540290935502A0935602CA
:10780000B093570242E050E066E170E084E592E018
:107810000E944B92B7C30E940A09B4C360916D02E3
:1078200070916E0280E090E00E940E90FC01208139
:107830002332B1F44AE050E060E070E001960E942B
:10784000B08C1B0160916D0270916E0280E090E03F
:107850000E940E90F4E02F1631040CF094C002C088
:10786000212C312C009709F48EC01982BE016F5F64
:107870007F4F0E942C2729013A014B01B82FA92FD5
:107880008AE0829DF001839DF00D1124EF5EF44E9D
:1078900020812A8331813B8382818C8393819D83E4
:1078A00024812E8335813F838681888797819987BC
:1078B0009201A301B4018B2F9A2FAA80BB80CC80A8
:1078C000DD80EE80FF80088519850E943F8C09F4D9
:1078D0005DC08981882351F18CF02A81422A3B8145
:1078E000532A8C81682A9D81792A2E81822A3F81A0
:1078F000932A8885B82B9985A92B18C04094509459
:107900006094709480949094B095A0952A814222BE
:107910003B8153228C8168229D8179222E81822293
:107920003F8193228885B8239985A923408251827B
:107930006282738284829582B683A78348E250E094
:107940006AE170E081E19BE10E944B928BEC93E055
:107950009F938F930E94D9908AE0829DF001839D2E
:10796000F00D1124EF5EF44E20813181428153816C
:1079700064817581868197810E94C8230E94670B6C
:107980000F900F9003C082E00E94CE288FEB93E00F
:107990009F938F930E94D9902FEF3FEF4FEF5FEFB0
:1079A0006FEF7FEF8FEF9FEF0E94C8230E94670B5E
:1079B00080916F020F900F90882309F4E3C21F9209
:1079C0008F938CEB93E09F938F930E94D9900F90AD
:1079D0000F900F900F90D6C260916D0270916E0261
:1079E00080E090E00E940E90FC0120812332A1F4FF
:1079F0004AE050E060E070E001960E94B08C8B019C
:107A000060916D0270916E0280E090E00E940E9095
:107A100004301105ECF402C000E010E00097C1F062
:107A20004AE050E060E070E00E94E48D2AE0209F90
:107A3000F001219FF00D1124EF5EF44E71876087F5
:107A400048E250E06AE170E081E19BE10E944B92E4
:107A500081E00E94CE2880916F02882309F492C2AF
:107A60001F928F9389EB93E09F938F930E94D990FD
:107A70000F900F900F900F9085C20E949C5680919E
:107A80006F02882309F47EC21F928F9386EB93E0E6
:107A90009F938F930E94D9900F900F900F900F900B
:107AA00071C20E94432980916F02882309F46AC23F
:107AB0001F928F9383EB93E09F938F930E94D990B3
:107AC0000F900F900F900F905DC280E090E00E94A9
:107AD000EB2080916F02882309F454C21F928F9388
:107AE00080EB93E09F938F930E94D9900F900F901B
:107AF0000F900F9047C28091072081FF2DC00E94F8
:107B0000911E892B49F58091FE1B8F938091FD1B5F
:107B10008F938091FC1B8F938091FB1B8F9385EA41
:107B200093E09F938F930E94D99080919B288F938D
:107B300080919A288F93809199288F93809198288B
:107B40008F9388E993E09F938F930E94D9900FB60B
:107B5000F894DEBF0FBECDBF0E94670B8091072057
:107B60009091082090FF63C081E090E00E94081E81
:107B70003B014C0180E090E00E94081E1B012C019B
:107B80000E945F1D9F928F927F926F9287E893E091
:107B90009F938F930E94D9905F924F923F922F9222
:107BA00087E793E09F938F930E94D990222D332DE6
:107BB000442D552D662D772D882D992D0E94021C60
:107BC0009F938F937F936F938CE693E09F938F9314
:107BD0000E94D990222D332D442D552D662D772DC1
:107BE000882D992D0E94631C9F938F937F936F9391
:107BF0008EE593E09F938F930E94D990222D332D91
:107C0000442D552D662D772D882D992D0E94C41C4D
:107C10009F938F937F936F938BE493E09F938F93C6
:107C20000E94D9900FB6F894DEBF0FBECDBF0E9460
:107C3000670B80916F02882309F4A4C11F928F9370
:107C400088E493E09F938F930E94D9900F900F90B8
:107C50000F900F9097C18091072082FF2BC021E0E9
:107C600048E061E083E00E9405138091F91B8F9347
:107C70008091F81B8F938091F71B8F938091F61B57
:107C80008F938091F51B8F938091F41B8F9380913C
:107C9000F31B8F938091F21B8F9381E393E09F936B
:107CA0008F930E94D9900E94670B0FB6F894DEBFA5
:107CB0000FBECDBF809107209091082091FF41C059
:107CC0000E944F17B62EA72E982E892E20E030E066
:107CD00048EC52E4D501F4016B2F7A2F8F2F9E2FA1
:107CE0000E94188920E836EE45EC57E40E949B86F6
:107CF00021E03EED42E45EE30E947B899B01AC0102
:107D000060E070E080E89FE30E94D0852BE43AE3D6
:107D10004DEB57E30E949B869F938F937F936F93C6
:107D20008F929F92AF92BF9288E193E09F938F933F
:107D30000E94D9900E94670B0FB6F894DEBF0FBE69
:107D4000CDBF80916F02882309F41CC11F928F93CD
:107D500085E193E09F938F930E94D9900F900F90AD
:107D60000F900F900FC160916D0270916E0280E0D4
:107D700090E00E940E906AE276E00E942290892BA9
:107D8000B1F460916D0270916E0280E090E00E940B
:107D90000E90009709F4F6C00E94FC8E803108F026
:107DA000F1C090915201982B90935201EBC08091B9
:107DB00052018F701F928F9383EE91E09F938F9368
:107DC0000E94D9900E94670B0F900F900F900F9018
:107DD000D9C060916D0270916E0280E090E00E94C7
:107DE0000E90009711F14AE050E060E070E00E94D0
:107DF000B08C603198F4609352021F926F9388E0C8
:107E000093E09F938F930E94D99041E050E063E10B
:107E100070E082E592E00E944B9211C08091520284
:107E20001F928F938FEF92E006C0809152021F92B3
:107E30008F9386EF92E09F938F930E94D9900F903B
:107E40000F900F900F900E94670B80916F02882314
:107E500009F498C01F928F9383EF92E09F938F93C2
:107E60000E94D9900F900F900F900F908BC060914F
:107E70006D0270916E0280E090E00E940E908C0185
:107E80006AE875E00E942290892BE1F40E94686400
:107E90008091540290915502A0915602B0915702E0
:107EA00090618093540290935502A0935602B09330
:107EB000570242E050E066E170E084E592E00E9403
:107EC0004B9260C06DE875E0C8010E942290892B3A
:107ED00081F5F8940E94766488E10FB6F894809357
:107EE0006000109260000FBE84B7877F84BF8091CE
:107EF00060008861809360001092600078948091A7
:107F0000540290915502A0915602B09157029F7E63
:107F10008093540290935502A0935602B093570257
:107F200042E050E066E170E084E592E00E944B920E
:107F300029C06FE276E0C8010E942290409154026D
:107F4000509155026091560270915702892B21F48D
:107F500054FF18C0F894FFCF54FF03C08AE895E09F
:107F600002C08DE895E09F938F938FED91E09F93F2
:107F70008F930E94D9900F900F900F900F9002C096
:107F80000E942D1FEA85FB851182108283E02B96CB
:107F90000FB6F894DEBF0FBECDBFDF91CF911F911A
:107FA0000F91FF90EF90DF90CF90BF90AF909F9098
:107FB0008F907F906F905F904F903F902F9008959B
:107FC0000F931F93CF93DF93EC018A0188819981EE
:107FD000009711F18E32904121F01982188283E0CE
:107FE00020C06231E9F4A80162E170E087ED99E018
:107FF0000E94F32D84E080937A2810927C281092BE
:108000007B2810937E2800937D284AE758E262E19E
:1080100084E392E00E9472528EE290E19983888319
:1080200081E0DF91CF911F910F9108950E945C64D0
:108030006C9A6B9A6A9A6F9A729A749A739A779AF0
:10804000809880B3897F80BB8398849887E08093F1
:108050007E00549A0E94E32A0E94152B81E00E9420
:108060007C0980E090E00E94BC0C0E94D35D0E94DD
:108070006B0A6093092470930A2480930B249093D5
:108080000C248091540286FD239A0895CF93DF93A8
:10809000EC0188819981009741F08931904109F480
:1080A0008CC01982188283E093C00E941640809190
:1080B000540280FD05C081FF01C01D9B0E94B76571
:1080C000809170008C7F809370008091B6008062F8
:1080D0008093B6001092B20082E08093B10080914C
:1080E000B6008770E1F78091700081608093700026
:1080F00068E279E080E090E00E9446640E943120CE
:1081000080E00E940F228AE69EE09F938F930E9458
:10811000D9900E94E60F809107200F900F9086FD66
:108120000E94FA5E809107209091082090FD0E94A5
:108130001B1D8091072087FF06C021E04CE061E015
:1081400080ED0E949D5F8091AB090E9459688091EB
:1081500053020E9400670E94FD668093D6098091B9
:1081600053020E9400678091AB091F928F93809108
:10817000D6091F928F9384E396E09F938F930E947A
:10818000C7901092D8091092D7090F900F900F90B6
:108190000F900F900F9088E492E090939628809330
:1081A000952883E290E09093E9118093E81189E1AA
:1081B00090E19983888381E00BC06332E1F742E369
:1081C00054E260E070E087ED99E00E94F32DE3CF88
:1081D000DF91CF9108958436910514F19F938F9389
:1081E00086E496E09F938F930E94C790809111241C
:1081F00090911224A0911324B09114240196A11DF2
:10820000B11D8093112490931224A0931324B09352
:1082100014240F900F900F900F9081E090E008953C
:1082200080E090E008952F923F924F925F926F927C
:108230007F928F929F92AF92BF92CF92DF92EF92F6
:10824000FF920F931F93CF93DF93CDB7DEB7C8593B
:10825000D1090FB6F894DEBF0FBECDBFC157DF4FB7
:1082600099838883CF58D0408A01633871F48BEDAD
:1082700099E0C956DF4F6883C759D0400E94B55076
:10828000C956DF4F6881C759D040C157DF4FA88119
:10829000B981CF58D0402D913C91273CBFE03B079E
:1082A00009F49DC340F42115310581F029303E4089
:1082B00009F4DBC3CFC3283D4FE0340709F4ABC357
:1082C0002F3D3F4011F40C94B84DC4C346EE52E02C
:1082D00061E870E08BED99E00E949B5089E09EE0A0
:1082E00075C3E3E0F0E0EC0FFD1FE00FF11F10821B
:1082F000C8010E94EB40892B89F720E030E040E084
:1083000050E0652D627070E080E090E0A0E00E9497
:10831000488C09F0FEC5C257DF4F2881CE58D040A7
:10832000287030E040E050E060E070E080E090E0F5
:10833000A0E00E94488CA1F127E04AE250E06BE205
:1083400070E089E290E00E94ED5A8CE898E20E9489
:108350005B5DBC01882777FD8095982F0E943A8746
:1083600020E030E048EC52E40E949B869F938F937C
:108370007F936F938AE796E09F938F931F9287E78F
:108380008F93CE01800F911F03969F938F930E942E
:108390002A91080F191F0FB6F894DEBF0FBECDBF8C
:1083A000C257DF4F2881CE58D040207130E040E0E6
:1083B00050E060E070E080E090E0A0E00E94488C37
:1083C000F1F126E04AE250E06BE270E089E290E0F1
:1083D0000E94ED5A81E090E00E94F50A8093AA097C
:1083E0008AE69BE10E945B5DBC01882777FD809552
:1083F000982F0E943A8720E030E048EC52E40E9437
:108400009B869F938F937F936F9384E896E09F93CF
:108410008F931F9287E78F93C8010296E1E0F0E007
:10842000EC0FFD1F8E0F9F1F9F938F930E942A9129
:10843000080F191F0FB6F894DEBF0FBECDBFC65789
:10844000DF4F2881CA58D04030E040E050E060E083
:1084500070E080E090E0A0E00E94488C01F10E9472
:10846000B10A9F938F937F936F938FE896E09F93CA
:108470008F931F9287E78F93C801029641E050E0E7
:108480004C0F5D1F840F951F9F938F930E942A911D
:10849000080F191F0FB6F894DEBF0FBECDBFC2572D
:1084A000DF4F2881CE58D040207430E040E050E0CB
:1084B00060E070E080E090E0A0E00E94488C31F144
:1084C00080910C248F9380910B248F9380910A24A8
:1084D0008F93809109248F938DE996E09F938F93DA
:1084E0001F9287E78F93C8010296A1E0B0E0AC0F1E
:1084F000BD1F8A0F9B1F9F938F930E942A91080F85
:10850000191F0FB6F894DEBF0FBECDBFC257DF4FA5
:108510002881CE58D040207830E040E050E060E044
:1085200070E080E090E0A0E00E94488C41F1F89477
:108530008091722890917328A0917428B091752829
:108540007894BF93AF939F938F938BEA96E09F931A
:108550008F931F9287E78F93C801029621E030E046
:108560002C0F3D1F820F931F9F938F930E942A9180
:10857000080F191F0FB6F894DEBF0FBECDBF20E065
:10858000372D317040E050E060E070E080E090E036
:10859000A0E00E94488C09F0CDC420E0372D327055
:1085A00040E050E060E070E080E090E0A0E00E94F9
:1085B000488C09F047C520E0372D347040E050E08A
:1085C00060E070E080E090E0A0E00E94488C09F05C
:1085D0006AC520E0372D387040E050E060E070E080
:1085E00080E090E0A0E00E94488C09F08BC520E07C
:1085F000372D307140E050E060E070E080E090E0C6
:10860000A0E00E94488C09F005C620E0372D3072AA
:1086100040E050E060E070E080E090E0A0E00E9488
:10862000488C09F027C620E030E040E050E0652D9E
:10863000647070E080E090E0A0E00E94488C09F057
:1086400047C620E0CD56DF4F3881C359D04040E0C7
:1086500050E060E070E080E090E0A0E00E94488C94
:1086600009F0A3C620E0CC56DF4F3881C459D04072
:1086700040E050E060E070E080E090E0A0E00E9428
:10868000488C09F0C0C620E030E0482D417050E031
:1086900060E070E080E090E0A0E00E94488C09F08B
:1086A000E0C620E030E0482D427050E060E070E02D
:1086B00080E090E0A0E00E94488C09F005C720E02F
:1086C00030E0CE56DF4F4881C259D04050E060E0E4
:1086D00070E080E090E0A0E00E94488C09F027C79D
:1086E00020E030E0482D487050E060E070E080E02D
:1086F00090E0A0E00E94488C09F043C720E030E001
:10870000482D407150E060E070E080E090E0A0E033
:108710000E94488C09F065C720E030E0482D407287
:1087200050E060E070E080E090E0A0E00E94488CC3
:1087300009F087C720E030E0482D407450E060E049
:1087400070E080E090E0A0E00E94488C09F0A9C7AA
:10875000B82DB078EB2E20E030E04B2F50E060E0F9
:1087600070E080E090E0A0E00E94488C09F0C9C76A
:10877000E92DE170FE2E20E030E040E05E2F60E069
:1087800070E080E090E0A0E00E94488C09F0C3C750
:1087900020E030E04E2D50E060E070E080E090E0BE
:1087A000A0E00E94488C09F0C1C720E030E040E022
:1087B0005F2D60E070E080E090E0A0E00E94488CD7
:1087C00009F0E6C720E030E040E0592D527060E04B
:1087D00070E080E090E0A0E00E94488C11F00C94E2
:1087E000FB4B20E030E040E0592D547060E070E039
:1087F00080E090E0A0E00E94488C11F00C942E4C98
:1088000020E030E040E0592D507160E070E080E001
:1088100090E0A0E00E94488C11F00C94614C20E0A4
:1088200030E040E0592D507260E070E080E090E070
:10883000A0E00E94488C11F00C94A04C20E030E0A5
:1088400040E0592D507460E070E080E090E0A0E0DE
:108850000E94488C11F00C94DF4C20E030E040E0A6
:10886000592D587060E070E080E090E0A0E00E9438
:10887000488C11F00C941E4D20E030E040E0CB56C7
:10888000DF4F5881C559D04060E070E080E090E053
:10889000A0E00E94488C11F00C944F4D779A809183
:1088A000AF099091B00992FD749AC257DF4F2881A9
:1088B000CE58D040372DA401652DCF56DF4F78819B
:1088C000C159D040842D962DA0E0FE0133967F0142
:1088D0000E94488C11F00C94864D80915202806168
:1088E00089838091CF098A83F701E00FF11F1082FD
:1088F0008091AF099091B00998012D5F3F4F7901A8
:1089000080FF0CC0FF922F9382E498E09F938F9397
:108910000E94C7900F900F900F900F90B701CE015B
:1089200001960E94E4598091540282FF0AC022E716
:1089300034E2A701BE016F5F7F4F8DE592E00E9498
:108940006A5E8091AF099091B00982FD73980E9490
:10895000FF658BED99E00E94B75080915402909191
:108960005502A0915602B091570290FF3FC00F5F91
:108970001F4F0E94FD66F82E89E10E941567409105
:10898000540250915502609156027091570250FF67
:1089900029C073988091CF098F5F8093CF098A8314
:1089A000B8016F5F7F4FCE0101960E94E4598BEDB5
:1089B00099E00E94B75040E050E065E88091EC11EA
:1089C0009091ED110E94725287EC9FE0C157DF4FEA
:1089D000A881B981CF58D0408D939C9338C000E0D6
:1089E00010E0CDCF8F2D0E941567739A8091AC094E
:1089F0009091AD09892B11F00E94B7658091CF0944
:108A00008F5F8093CF098091AF099091B00982FF69
:108A100065CC739A63CC87EC99E00E941855892B3A
:108A2000B1F00E94FF658091540287FD2B9860E4AD
:108A300070E087EC99E00E94F1548FED9FE0C15700
:108A4000DF4FE881F981CF58D0409183808381E066
:108A50000C94CB4DC157DF4FA881B981CF58D0407E
:108A60001D921C9283E00C94CB4D623181F7809172
:108A7000540290915502A0915602B091570291FD77
:108A80002DCCF80180818130D1F40180F281E02D7C
:108A90002081C257DF4F2883CE58D040718082801A
:108AA000938054803581CF56DF4F3883C159D040F1
:108AB0004680678020843184A12CB12C3DC0823057
:108AC00081F4A380B480212C312CB1E0C257DF4F58
:108AD000B883CE58D040712C812C50E8952E512C63
:108AE00024C0833099F0843009F0F8CB212C312C4C
:108AF000A12CB12CE5E0C257DF4FE883CE58D0401F
:108B0000712C812C912C42E0542E0FC0212C312C41
:108B1000A12CB12CF5E0C257DF4FF883CE58D040DE
:108B2000712C812C912C55245394CF56DF4F1882F1
:108B3000C159D040412C612C20917C0230917D02A2
:108B400040917E0250917F026091092470910A2425
:108B500080910B2490910C240E94978687FF26C059
:108B60008091152490911624A0911724B091182477
:108B70000196A11DB11D8093152490931624A093F6
:108B80001724B093182425E0C257DF4F2883CE580E
:108B9000D04020E2722E812C912C34E0532ECF56FF
:108BA000DF4F1882C159D040412C612C382D3470D0
:108BB000CE56DF4F3883C259D04020E030E0CE5649
:108BC000DF4F4881C259D04050E060E070E080E063
:108BD00090E0A0E00E94488C09F08C9AC257DF4FC9
:108BE0004881CE58D0404072C657DF4F4883CA589C
:108BF000D040242F30E040E050E060E070E080E0C2
:108C000090E0A0E00E94488C11F00E94B10A572D1C
:108C10005074CD56DF4F5883C359D04020E0352FD4
:108C200040E050E060E070E080E090E0A0E00E9472
:108C3000488C11F00E94911E672D6078CC56DF4F52
:108C40006883C459D04020E0362F40E050E060E017
:108C500070E080E090E0A0E00E94488C51F00E941B
:108C6000570A60937F28709380288093812890937F
:108C70008228C257DF4F2881CE58D040217030E083
:108C800040E050E060E070E080E090E0A0E00E9412
:108C9000488CF1F088EF9AE19F938F938AE596E0F4
:108CA0009F938F931F9287E78F93CE0103969F9395
:108CB0008F930E942A917C010E94EB400FB6F8949A
:108CC000DEBF0FBECDBF892B09F008CB870102C0E4
:108CD00000E010E0C257DF4F2881CE58D04022700C
:108CE00030E040E050E060E070E080E090E0A0E044
:108CF0000E94488C09F442C0C801029662E676E000
:108D0000E1E0F0E0EC0FFD1F8E0F9F1F0E942B9003
:108D10000D5F1F4F8CE8C82E88E2D82E9EEEE92EFC
:108D200093E0F92E27E7D6018D916D011F928F9365
:108D3000FF92EF921F922F93C8010296E1E0F0E0BC
:108D4000EC0FFD1F8E0F9F1F9F938F93C856DF4F11
:108D50002883C859D0400E942A91080F191F0FB6C6
:108D6000F894DEBF0FBECDBFC856DF4F2881C8596B
:108D7000D04054E9C51658E2D506A9F6C257DF4FD0
:108D80002881CE58D040247030E040E050E060E0D0
:108D900070E080E090E0A0E00E94488C09F461C09F
:108DA000C801029666E676E0A1E0B0E0AC0FBD1F18
:108DB0008A0F9B1F0E942B900C5F1F4F7E01BAE70A
:108DC000EB0EF11C80E1F70111928A95E9F728E09A
:108DD000A70168E980EB0E9449116701F8E0CF0E16
:108DE000D11C4EEE53E027E7D7018D917D011F92F4
:108DF0008F935F934F931F922F93C8010296E1E0E8
:108E0000F0E0EC0FFD1F8E0F9F1F9F938F93C856AE
:108E1000DF4F2883C859D040CA56DF4F4883C65910
:108E2000D040C956DF4F5883C759D0400E942A917D
:108E3000080F191F0FB6F894DEBF0FBECDBFC8567E
:108E4000DF4F2881C859D040CA56DF4F4881C659E4
:108E5000D040C956DF4F5881C759D040EC14FD04AB
:108E600019F6792D7078CB56DF4F7883C559D040ED
:108E700020E030E040E0572F60E070E080E090E0DC
:108E8000A0E00E94488CE1F48091AC099091AD097A
:108E90009F938F938BE696E09F938F931F9287E724
:108EA0008F93CE01800F911F03969F938F930E9403
:108EB0002A91080F191F0FB6F894DEBF0FBECDBF61
:108EC00020E030E040E050E0652D617070E080E02F
:108ED00090E0A0E00E94488C09F40FCAE3E0F0E0C3
:108EE000EC0FFD1FE00FF11F80E28083E5E3F4E269
:108EF00080810F5F1F4F882309F4F3C98081A1E0AF
:108F0000B0E0AC0FBD1FA00FB11F12968C9331962D
:108F1000EFCFCE01800F911F62E776E003960E94AB
:108F20002B90095F1F4FC8010E94EB40892B09F06D
:108F3000D5C9F1C92114310409F42FCBF8946091FB
:108F40007228709173288091742890917528C65763
:108F5000DF4F688379838A839B83CA58D040789493
:108F60008091621B9091631BA091641BB091651B63
:108F7000C657DF4F288139814A815B81CA58D0406A
:108F8000281B390B4A0B5B0BCA01B9010E943887B9
:108F90006B017C01B10180E090E00E9438879B0169
:108FA000AC01C701B6010E949B867C01FF928F93A2
:108FB0007F936F9386EB96E09F938F931F9287E743
:108FC0008F939E01200F311F2D5F3F4F3F932F93B3
:108FD000C956DF4F6883C759D040CA56DF4F7883E0
:108FE000C659D0400E942A91080F191FC956DF4F59
:108FF0006881C759D040CA56DF4F7881C659D040E2
:10900000862F972FAE2DBF2D80938428909385288F
:10901000A0938628B0938728C657DF4F488159818F
:109020006A817B81CA58D0404093621B5093631B76
:109030006093641B7093651B0FB6F894DEBF0FBE80
:10904000CDBFABCA2114310409F4B5CAF89480919C
:10905000391B90913A1BA0913B1BB0913C1B78941B
:109060009F938F9380915B028F9380915A028F938D
:1090700083EC96E09F938F931F9287E78F93C801AD
:109080000296A1E0B0E0AC0FBD1F8A0F9B1F9F931B
:109090008F930E942A91080F191F0FB6F894DEBF14
:1090A0000FBECDBF88CAF89480917628909177281A
:1090B000A0917828B09179287894BF93AF939F932B
:1090C0008F9383ED96E09F938F931F9287E78F9303
:1090D000C801029621E030E02C0F3D1F820F931F44
:1090E0009F938F930E942A91080F191FC8010E9415
:1090F000EB400FB6F894DEBF0FBECDBF892B09F051
:10910000EDC867CA2114310409F471CAF89460915A
:109110007628709177288091782890917928C65781
:10912000DF4F688379838A839B83CA58D0407894C1
:109130008091661B9091671BA091681BB091691B81
:10914000C657DF4F288139814A815B81CA58D04098
:10915000281B390B4A0B5B0BCA01B9010E943887E7
:109160006B017C01B10180E090E00E9438879B0197
:10917000AC01C701B6010E949B867C01FF928F93D0
:109180007F936F938EED96E09F938F931F9287E767
:109190008F939E01200F311F2D5F3F4F3F932F93E1
:1091A000C956DF4F6883C759D040CA56DF4F78830E
:1091B000C659D0400E942A91080F191FC956DF4F87
:1091C0006881C759D040CA56DF4F7881C659D04010
:1091D000862F972FAE2DBF2D8093882890938928B6
:1091E000A0938A28B0938B28C657DF4F48815981B6
:1091F0006A817B81CA58D0404093661B5093671B9D
:109200006093681B7093691B0FB6F894DEBF0FBEA6
:10921000CDBFEDC9232809F4F8C9F89480913D1B0E
:1092200090913E1BA0913F1BB091401B78949F935F
:109230008F93809159028F93809158028F938BEE78
:1092400096E09F938F931F9287E78F93C8010296B2
:10925000A1E0B0E0AC0FBD1F8A0F9B1F9F938F93BF
:109260000E942A91080F191F0FB6F894DEBF0FBE97
:10927000CDBFCBC980910D2490910E24A0910F24D5
:10928000B0911024BF93AF939F938F938BEF96E091
:109290009F938F931F9287E78F93C801029621E0D7
:1092A00030E02C0F3D1F820F931F9F938F930E94DE
:1092B0002A91080F191FC8010E94EB400FB6F894BD
:1092C000DEBF0FBECDBF892B11F00C946E41ABC930
:1092D000809118248F93809117248F938091162466
:1092E0008F93809115248F93809114248F93809174
:1092F00013248F93809112248F93809111248F9344
:1093000086E097E09F938F931F92B7E7FB2EFF9223
:10931000C801029661E070E06C0F7D1F860F971FF9
:109320009F938F930E942A91080F191FC8010E94D2
:10933000EB400FB6F894DEBF0FBECDBF892B11F006
:109340000C946E41809107209091082090FF79C97C
:1093500080911C248F9380911B248F9380911A24D9
:109360008F93809119248F938AE297E09F938F9334
:109370001F92FF92C8010296E1E0F0E0EC0FFD1FA2
:109380008E0F9F1F9F938F930E942A91080F191F82
:10939000C8010E94EB400FB6F894DEBF0FBECDBFF0
:1093A000892B11F00C946E414CC98091FE1B8F9358
:1093B0008091FD1B8F938091FC1B8F938091FB1BF1
:1093C0008F938CE397E09F938F931F9287E78F9300
:1093D000C801029641E050E04C0F5D1F840F951FBD
:1093E0009F938F930E942A91080F191FC8010E9412
:1093F000EB400FB6F894DEBF0FBECDBF892B11F046
:109400000C946E412FC9809182288F93809181287E
:109410008F93809180288F9380917F288F9387E40A
:1094200097E09F938F931F9287E78F93C8010296CF
:10943000A1E0B0E0AC0FBD1F8A0F9B1F9F938F93DD
:109440000E942A91080F191FC8010E94EB400FB615
:10945000F894DEBF0FBECDBF892B11F00C946E4186
:1094600012C981E00E94080A2091740230917502AD
:1094700040917602509177020E9418899F938F93B2
:109480007F936F9384E597E09F938F931F9287E775
:109490008F93C801029621E030E02C0F3D1F820F10
:1094A000931F9F938F930E942A91080F191FC80141
:1094B0000E94EB400FB6F894DEBF0FBECDBF892BE4
:1094C00011F00C946E41EDC882E00E94080A2091D0
:1094D00070023091710240917202509173020E94A9
:1094E00018899F938F937F936F9381E697E09F9363
:1094F0008F931F9287E78F93C801029661E070E017
:109500006C0F7D1F860F971F9F938F930E942A9148
:10951000080F191FC8010E94EB400FB6F894DEBF78
:109520000FBECDBF892B11F00C946E41C8C883E0EB
:109530000E94080A9F938F937F936F938EE697E024
:109540009F938F931F9287E78F93C8010296E1E064
:10955000F0E0EC0FFD1F8E0F9F1F9F938F930E94D3
:109560002A91080F191F8C98C8010E94EB400FB672
:10957000F894DEBF0FBECDBF892B11F00C946E4165
:10958000AFC88091072087FFB9C821E042E161E0C0
:1095900080ED0E949D5F9F938F937F936F938BE7E6
:1095A00097E09F938F931F9287E78F93C80102964E
:1095B00041E050E04C0F5D1F840F951F9F938F93E8
:1095C0000E942A91080F191FC8010E94EB400FB694
:1095D000F894DEBF0FBECDBF892B11F00C946E4105
:1095E0008DC88091072087FF97C821E042E162E0A3
:1095F00080ED0E949D5F9F938F937F936F9389E887
:1096000097E09F938F931F9287E78F93C8010296ED
:10961000A1E0B0E0AC0FBD1F8A0F9B1F9F938F93FB
:109620000E942A91080F191FC8010E94EB400FB633
:10963000F894DEBF0FBECDBF892B11F00C946E41A4
:109640006BC88091072087FF75C821E042E163E085
:1096500080ED0E949D5F9F938F937F936F9387E927
:1096600097E09F938F931F9287E78F93C80102968D
:1096700021E030E02C0F3D1F820F931F9F938F93AB
:109680000E942A91080F191FC8010E94EB400FB6D3
:10969000F894DEBF0FBECDBF892B11F00C946E4144
:1096A00049C88091072087FF53C821E042E164E068
:1096B00080ED0E949D5F9F938F937F936F9385EAC8
:1096C00097E09F938F931F9287E78F93C80102962D
:1096D00061E070E06C0F7D1F860F971F9F938F9343
:1096E0000E942A91080F191FC8010E94EB400FB673
:1096F000F894DEBF0FBECDBF892B11F00C946E41E4
:1097000027C88091072082FF33C846E061E083E0EC
:109710000E9405132DC88091072082FF39C821E0DF
:1097200046E061E083E00E94051332C88091072083
:1097300082FF3BC88091F51B8F938091F41B8F9320
:109740008091F31B8F938091F21B8F9383EB97E0B3
:109750009F938F931F9287E78F93C801029621E012
:1097600030E02C0F3D1F820F931F9F938F930E9419
:109770002A91080F191FC8010E94EB400FB6F894F8
:10978000DEBF0FBECDBF892B11F00C946E410DC80A
:109790008091072082FF16C88091F91B8F938091DA
:1097A000F81B8F938091F71B8F938091F61B8F93FB
:1097B0008BEB97E09F938F931F9287E78F93C8015E
:1097C000029661E070E06C0F7D1F860F971F9F93DC
:1097D0008F930E942A91080F191FC8010E94EB4025
:1097E0000FB6F894DEBF0FBECDBF892B11F00C94DD
:1097F0006E410C94E243809107209091082090FDE7
:1098000002C00C94F14380E090E00E94081E9F93F8
:109810008F937F936F9386EC97E09F938F931F9224
:1098200087E78F93C8010296E1E0F0E0EC0FFD1F9F
:109830008E0F9F1F9F938F930E942A91080F191FCD
:10984000C8010E94EB400FB6F894DEBF0FBECDBF3B
:10985000892B11F00C946E410C94F14380910720F8
:109860009091082090FD02C00C94004481E090E0AB
:109870000E94081E9F938F937F936F9386ED97E0CE
:109880009F938F931F9287E78F93C801029641E0C1
:1098900050E04C0F5D1F840F951F9F938F930E9484
:1098A0002A91080F191FC8010E94EB400FB6F894C7
:1098B000DEBF0FBECDBF892B11F00C946E410C940E
:1098C0000044809107209091082090FD02C00C94E4
:1098D0000F4481E090E00E94081E6B017C0180E053
:1098E00090E00E94081E9B01AC01C701B6010E94D6
:1098F000021C9F938F937F936F9387EE97E09F93C4
:109900008F931F9287E78F93C8010296A1E0B0E082
:10991000AC0FBD1F8A0F9B1F9F938F930E942A91AC
:10992000080F191FC8010E94EB400FB6F894DEBF64
:109930000FBECDBF892B11F00C946E410C940F44D7
:10994000809107209091082090FD02C00C941E4445
:1099500081E090E00E94081E6B017C0180E090E0B5
:109960000E94081E9B01AC01C701B6010E94631C46
:109970009F938F937F936F9382EF97E09F938F9343
:109980001F9287E78F93C801029621E030E02C0FE9
:109990003D1F820F931F9F938F930E942A91080F60
:1099A000191FC8010E94EB400FB6F894DEBF0FBE2E
:1099B000CDBF892B11F00C946E410C941E44809104
:1099C00007209091082090FD02C00C942D4481E066
:1099D00090E00E94081E6B017C0180E090E00E94F4
:1099E000081E9B01AC01C701B6010E94C41C9F93D5
:1099F0008F937F936F9380E098E09F938F931F9254
:109A000087E78F93C801029661E070E06C0F7D1FBD
:109A1000860F971F9F938F930E942A91080F191FFB
:109A2000C8010E94EB400FB6F894DEBF0FBECDBF59
:109A3000892B11F00C946E410C942D4480910720D9
:109A40009091082091FD02C00C943C440E944F1755
:109A50009F938F937F936F9383E198E09F938F936E
:109A60001F9287E78F93C8010296E1E0F0E0EC0FC8
:109A7000FD1F8E0F9F1F9F938F930E942A91080FA7
:109A8000191FC8010E94EB400FB6F894DEBF0FBE4D
:109A9000CDBF892B11F00C946E410C943C44D50140
:109AA00016968C9116971F928F9315968C911597F9
:109AB0001F928F9313968C9113971F928F931296E8
:109AC0008C911F928F9384E298E09F938F931F92C3
:109AD00087E78F93C8010296E1E0F0E0EC0FFD1FED
:109AE0008E0F9F1F9F938F930E942A91080F191F1B
:109AF000C8010E94EB400FB6F894DEBF0FBECDBF89
:109B0000892B11F00C946E410C944E448091AF0956
:109B10009091B00982FD0CC08091540280FD08C074
:109B200081FD02C00C946D441D9902C00C946D44DB
:109B3000FF92EF928BE398E09F938F930E94C790E0
:109B400080916F020F900F900F900F90882311F467
:109B50000C946D441F928F9387E69EE09F938F93A2
:109B60000E94D9900F900F900F900F900C946D441D
:109B700087EC99E00E941855892B11F40C94274525
:109B80000E94B7658091540287FD02C00C946E411B
:109B90002B9A0C946E41C856DF4F0FB6F894DEBF77
:109BA0000FBECDBFDF91CF911F910F91FF90EF902E
:109BB000DF90CF90BF90AF909F908F907F906F90ED
:109BC0005F904F903F902F9008950C94DE504F92ED
:109BD0005F926F927F928F929F92AF92BF92CF923D
:109BE000DF92EF92FF920F931F93CF93DF93CDB746
:109BF000DEB760970FB6F894DEBF0FBECDBF6B0126
:109C00000E94FD66E82FF0E0EE0FFF1FE55DF44EC9
:109C1000808191810196918380838091AF09909199
:109C2000B00981FD74988090540290905502A090E4
:109C30005602B09057020E9438597C01FC01808185
:109C4000982F92959F70913099F48F7051F4809174
:109C50000F1B9091101B01969093101B80930F1B6C
:109C60000CC1B6018CE998E20E945450892B51F046
:109C700080910D1B90910E1B019690930E1B80936B
:109C80000D1BFBC0D501C4011EE0B695A7959795A5
:109C900087951A95D1F7F82FF1708F2E86EE99E0FF
:109CA0000E945F538C01009709F448C0B601C801B7
:109CB00002960E945450892BE9F1980142E459E040
:109CC00060E074E6C8010F960E94DF55F7019181AC
:109CD000F8018481981321C082858F5F82878091EB
:109CE0000B1B90910C1B019690930C1B80930B1BEC
:109CF00084E00E94555AF801208530E02817390782
:109D000008F0AEC184E00E94555AF8018087F7013F
:109D100080818F70F8018187B0C0F801128684E0DD
:109D20000E94555AF8018087F70180818F70F801F1
:109D3000818797C1C8010E940754B4CF84E092E0A4
:109D40000E94F4528C01009709F497C0B601C80133
:109D500002960E944B50F70181818150F801848363
:109D600080E091E0A0E0B0E083879487A587B68784
:109D7000128684E00E94555AF8018087F70180819D
:109D80008F70F8018187B80186EE99E00E94BF5379
:109D9000980142E459E060E074E6C8010F960E9421
:109DA000DF5599249394F7018181F8018483F701A9
:109DB00080818F70F801878384E00E94555AF801F2
:109DC000858383E00E94555A5C01F8018683878170
:109DD0008F3009F0912CF7014180F8018481481AF5
:109DE000512C612C712CA6E0440C551C661C771C70
:109DF000AA95D1F72385348545855685A0ECB0E03A
:109E00000E94F689BB27A92F982F872F480E591E2D
:109E10006A1E7B1E43865486658676868091AF09CE
:109E20009091B00981FD33C08091540280FD2FC014
:109E300081FD2BC08091540290915502A091560251
:109E4000B091570288279078892B8A2B8B2B09F0A9
:109E5000D2C0992091F082E080931E241092202499
:109E600010921F2410932224009321244EE154E2E7
:109E700062E184E392E00E9472528091AF09909176
:109E8000B00981FFF0C0749AEEC01D9BD3CFA4E649
:109E9000B0E0A30192010E94F689672F782F892FE5
:109EA000992724E630E040E050E00E94418A7F9309
:109EB0006F93452C562C672C77245F924F92BB24CE
:109EC000BF92AF92F80185811F928F93F701808135
:109ED0008F701F928F9381811F928F93F6018181E2
:109EE0001F928F9380811F928F93C70102969F9339
:109EF0008F9383E598E09F938F930E94C790809102
:109F00006F020FB6F894DEBF0FBECDBF882361F09D
:109F10001F928F9384E69EE09F938F930E94D99027
:109F20000F900F900F900F908091540290915502D6
:109F3000A0915602B091570296FF2DC0882059F18A
:109F4000F7012081322F3F70832F90E00297D4F0E9
:109F50008FEF830F207F822B80838BED99E00E940F
:109F6000E54D8091091B90910A1B019690930A1B65
:109F70008093091B8091AF099091B00996FF0BC0A7
:109F8000739809C080910F1B9091101B01969093BC
:109F9000101B80930F1B8091072086FF4BCF0E94E0
:109FA000EC5EC70105960E94B85EF70181811F92A1
:109FB0008F93F80186811F928F9385811F928F93D3
:109FC00087E998E09F938F931F9280E18F939E0182
:109FD0002F5F3F4F6901DF922F930E942A9182E009
:109FE0000E94D25EC6010E94B85E0FB6F894DEBF32
:109FF0000FBECDBF1FCF88EF9AE12091F81A222320
:10A0000009F427CF9F938F938AEA98E09F938F93C9
:10A01000FE0131966F01DF92EF930E9467915C0120
:10A02000B601C70102960E944C900F900F900F90BE
:10A030000F900F900F90009709F40BCF95012F5FB1
:10A040003F4F280F391FA9012F5F3F4FFA01808131
:10A050008032C9F362E18CE092E00E947252F9CE44
:10A06000812C912CA0CE60960FB6F894DEBF0FBE67
:10A07000CDBFDF91CF911F910F91FF90EF90DF90B7
:10A08000CF90BF90AF909F908F907F906F905F9098
:10A090004F9008950895FB012081FC012083FB016E
:10A0A0002181FC0121830895FC019081DB018C91C9
:10A0B000981309C081E090E0318111962C913217FC
:10A0C00021F080E0089580E090E00895BC018CE9E3
:10A0D00098E20C944B50DC011996ED91FC911A9783
:10A0E0000280F381E02D309709F0099408950F93D1
:10A0F0001F93CF93DF9300D0CDB7DEB78C0188E1FB
:10A100000E94685ABC01CE0101960E944B50D801B2
:10A110001996ED91FC911A970190F081E02DBE0106
:10A120006F5F7F4FC80109950F900F90DF91CF911E
:10A130001F910F910895EF92FF920F931F93CF936A
:10A14000DF93EC018B017A014EEF52E00E94C45084
:10A15000FA86E98662E073E0C801DF91CF911F9132
:10A160000F91FF90EF900C941D510C94DC50CF9305
:10A17000DF93EC016CE978E288E10E945E5ACE013F
:10A18000DF91CF910C94DE50EF92FF920F931F93CB
:10A19000CF93DF93EC018B017A010E94F950F8868E
:10A1A000EF8266E073E0C801DF91CF911F910F91BC
:10A1B000FF90EF900C941D510C9401510C94796B0D
:10A1C000DC011796ED91FC9118970190F081E02D3C
:10A1D0000994DC011796ED91FC9118970280F381A8
:10A1E000E02D309709F0099408958AEE91E10C94DE
:10A1F0005B53FC0173836283BC018AEE91E10C9492
:10A20000BF53BC018AEE91E10C94A453CF93DF932A
:10A21000EC018AEE91E10E945F53009749F0FC0146
:10A22000228133812C173D0729F00E940754F5CF76
:10A2300080E090E0DF91CF9108950F931F93CF932B
:10A24000DF938B010E940651EC01009731F01D83D2
:10A250000C83C8010E94AA6D8E83DF91CF911F915C
:10A260000F9108951F93CF93DF93EC01162FEC818C
:10A27000FD813097D1F09093ED118093EC1182E045
:10A280008887CE0106960995992787FD90950297B4
:10A29000029710F0133839F4BE01CE01DF91CF914F
:10A2A0001F910C945F5181E08887DF91CF911F91BE
:10A2B0000895FC01208520FD0C9432510895CF9221
:10A2C000DF92EF92FF920F931F93CF93DF93EC01F6
:10A2D0006B01E090EC11F090ED110091EE111091F6
:10A2E000EF11F801EC17FD0739F0309709F44AC077
:10A2F0000190F081E02DF6CF209709F443C08885C6
:10A30000882309F118860115110561F0C017D107DE
:10A3100029F0AE0167E8C8010E945951F801008197
:10A320001181F1CFEC81FD81309769F0CC15DD050D
:10A3300051F0D093ED11C093EC1140E050E063E890
:10A34000CE0106960995E091EE11F091EF11CE172E
:10A35000DF0769F4888199819093EF118093EE1162
:10A360000DC0808191818C179D0721F0FC013097F1
:10A37000C1F704C08881998191838083F092ED11A7
:10A38000E092EC11DF91CF911F910F91FF90EF9030
:10A39000DF90CF9008951F93CF93DF931092F81121
:10A3A000C091EE11D091EF1111E0209779F08985DD
:10A3B000882341F01887198640E050E062E8CE011A
:10A3C0000E9432510990D881C02DEFCFDF91CF91FB
:10A3D0001F91089580919B1291E0980F90939B128A
:10A3E00008956091EC117091ED110C945F518AE821
:10A3F00080939B121092991210929A121092EF1160
:10A400001092EE111092ED111092EC1108958091BE
:10A41000F81181110E94CB5170919A12772309F49F
:10A4200051C0E09199122E2F30E085E0E89FF001B5
:10A430001124E750FE4E60816093F71141815281F3
:10A440005093F6114093F511838194819093F41108
:10A450008093F3112F5F3F4F2F7133272093991271
:10A46000715070939A12009731F58091EE1190918E
:10A47000EF119093F2118093F1118091F11190916D
:10A48000F211892BF9F08091F81181110E94CB51C2
:10A490004091F5115091F6116091F7118091F111F1
:10A4A0009091F2110E945951E091F111F091F21145
:10A4B00080819181DECF613819F421E0FC01208791
:10A4C0000E9459518091F81120919A1290E0820FC8
:10A4D000911D08958091F81120919A1290E0820FB9
:10A4E000911D089520919A122032B9F0E0919912AD
:10A4F000E20FEF71E093F01135E0E39FF0011124DA
:10A50000E750FE4E608352834183948383832F5FA1
:10A5100020939A1280E090E0089581E090E0089501
:10A52000CF93DF93C091EC11D091ED110E9459515E
:10A53000D093ED11C093EC11DF91CF910895AB0151
:10A540003091EE112091EF11E32FF22FE817F90768
:10A55000B1F0309721F00190F081E02DF7CF009716
:10A5600071F0FC01308321839093EF118093EE1101
:10A5700021E020871782168261E80C94905208959A
:10A58000009749F0FC0120852150223020F421E081
:10A5900021872093F811089521E030E0FC018085A7
:10A5A000811102C020E030E0C9010895CF93DF930C
:10A5B000EC014A815B8160E070E08C819D810E94AA
:10A5C0001B902A813B8188819981289FA001299F26
:10A5D000500D389F500D112460E070E08E819F81F6
:10A5E000DF91CF910C941B90FC018281938120E03C
:10A5F00030E028173907D1F0A481B581A20FB31F2D
:10A600004C91411110C081E08C9380819181289FF1
:10A61000A001299F500D389F500D112486819781EC
:10A62000840F951F08952F5F3F4FE3CF80E090E0A8
:10A630000895FC01268137814281538180E090E0BA
:10A6400084179507C9F02617370781F4A481B581CF
:10A65000A80FB91F2C91121614F421502C930480CA
:10A66000F581E02DE80FF91F80810895A081B18167
:10A670002A0F3B1F0196E4CF8FEF0895FC018681DE
:10A68000978168177907A0F0A081B1814281538139
:10A69000A49F9001A59F300DB49F300D1124280F69
:10A6A000391F81E090E06217730720F080E0089581
:10A6B00080E090E00895FC01118210820895FC0171
:10A6C000808191810895FB0120813181FC013183DA
:10A6D00020830895DC01ED91FC91309731F0808169
:10A6E0009181009729F0FC01FACF80E090E0089575
:10A6F000CF010895DC01ED91FC9111973097A9F0FD
:10A7000020813181232B21F41D921C92CF010895C9
:10A71000A081B1818D919C911197892B11F0FD0140
:10A72000F7CF11821082CD01089580E090E0089566
:10A73000DC01ED91FC911197309721F0208131815E
:10A740002D933C93CF010895DC01ED91FC9130975E
:10A75000A9F0A0E0B0E020813181E617F70741F4CD
:10A76000109709F4DC012D933C9311821082089517
:10A770002115310519F0DF01F901EDCF08950F938F
:10A780001F93CF93DF938C01EB010E94A453198296
:10A790001882C8010E946A53009711F4F80101C0A1
:10A7A000FC01D183C083DF91CF911F910F91089558
:10A7B0000F931F93CF93DF93EC018B010E94A4535F
:10A7C00088819981F8019183808319830883DF91BF
:10A7D000CF911F910F910895DC01ED91FC9180E0E4
:10A7E00090E0309729F001960190F081E02DF9CFAB
:10A7F0000895FB01309719F4BA010C94D853808165
:10A800009181DA018D939C93518340830895009741
:10A8100021F0FC0180819181089580E090E008950D
:10A8200080919E1290919F12892B29F410929D1273
:10A8300010929C1208950E940463E0919E12F09180
:10A840009F122281338140815181240F351F281BA3
:10A85000390B0480F581E02D309769F042815381F6
:10A8600060817181460F571F481B590B42175307D0
:10A8700080F79A01EECF280F391F30939D12209355
:10A880009C12089582E892E00C94C052EF92FF92DD
:10A890000F931F93CF93DF938C01FC0180819181F3
:10A8A000009799F08A359105D9F0F801118210824C
:10A8B00083E068C0868197818417950709F049C0B5
:10A8C0000480F581E02D3097A9F710929F12109225
:10A8D0009E128AE590E0F8019183808381E052C066
:10A8E000673891F16238A9F7C0919E12D0919F12FA
:10A8F000E12CF12C209769F3CE010E947B71892B0A
:10A90000F1F0AE0168E88E819F810E947252892B1E
:10A91000A1F41F821E828C819D81E114F10421F03B
:10A92000F7019583848304C090939F1280939E12B5
:10A930001D821C820E941054D7CF0E9442547E0177
:10A940000C80DD81C02DD6CFE0919E12F0919F1238
:10A95000BACFF0939F12E0939E12A481B581109715
:10A9600009F4B7CF16968D919C9117978417950788
:10A9700011F0FD01F2CF14968D919C91159795835E
:10A980008483EBCFDF91CF911F910F91FF90EF90D8
:10A990000895CF93DF93EC010E9442548E819F81F2
:10A9A00030919E1220919F12892B59F0E32FF22FA4
:10A9B000309739F0EC17FD0781F00480F581E02D28
:10A9C000F7CF8091EC119091ED119F838E833C83A2
:10A9D0002D83D0939F12C0939E12DF91CF910C9440
:10A9E0001054CF93DF93EC010E945B71CE01DF9195
:10A9F000CF910C94C954CF93DF93EC010E946771FF
:10AA0000CE01DF91CF910C94C954CF93DF93EC0129
:10AA10000E947171CE01DF91CF910C94C954FC0159
:10AA200020813181260F371F318320830C941054ED
:10AA300021E030E0FC0186819781892B11F020E034
:10AA400030E0C9010895FC01228133818081918128
:10AA5000820F931F0895FC0180819181089581E008
:10AA600090E020919E1230919F12232B11F480E0F0
:10AA700090E0089580919E1290919F12892B29F069
:10AA800080919C1290919D12089580E090E008952D
:10AA9000CF93DF93EC01E0919E12F0919F128E17FD
:10AAA0009F0769F48C819D8190939F1280939E12E1
:10AAB0000DC0848195818C179D0721F0FC01309792
:10AAC000C1F706C08C819D81958384830E941054B8
:10AAD0001D821C821F821E82DF91CF910895EF920A
:10AAE000FF920F931F93CF93DF938C017A01FC01A8
:10AAF00080819181009741F08B34910501F1F8013B
:10AB00001182108283E048C081EA92E10E945F5383
:10AB1000EC01209751F06C817D81CE0102960E945C
:10AB2000F1540990D881C02DF4CF81E08093A01218
:10AB30008BE490E0F8019183808381E02DC0683838
:10AB4000E1F781EA92E10E945F53EC01209781F3E3
:10AB5000CE010296E816F906D9F4BE0181EA92E127
:10AB60000E94A453E090EC11F090ED118A859B8532
:10AB70009093ED118093EC11EC85FD85309719F0E1
:10AB80008E859F850995F092ED11E092EC11D0CF62
:10AB90000990D881C02DDACFDF91CF911F910F910D
:10ABA000FF90EF9008951092A01281EA92E10E9426
:10ABB0005B5360E070E08CE892E00C949F520F933E
:10ABC0001F93CF93DF93EC010091EC111091ED11E5
:10ABD0001B870A875D874C873F872E878091A0124D
:10ABE000882379F08CE892E09093ED118093EC113A
:10ABF000CE0102960E94F1541093ED110093EC11D6
:10AC000002C07D836C83BE0181EA92E10E94A4535D
:10AC1000BE0181EA92E1DF91CF911F910F910C94D7
:10AC2000BF530F931F93CF93DF93EC018091A0123A
:10AC3000882391F00091EC111091ED118CE892E0D5
:10AC40009093ED118093EC11CE0102960E94FB547B
:10AC50001093ED110093EC11BE0181EA92E10E9484
:10AC6000A453BE0181EA92E1DF91CF911F910F9130
:10AC70000C94BF530F931F93CF93DF93EC018091FC
:10AC8000A012882391F00091EC111091ED118CE845
:10AC900092E09093ED118093EC11CE0102960E9408
:10ACA00005551093ED110093EC11BE0181EA92E17C
:10ACB0000E94A453BE0181EA92E1DF91CF911F91DE
:10ACC0000F910C94BF53CF93DF93EC018091A012AE
:10ACD000882329F0CE0102960E94485504C01F82A5
:10ACE0001E8219861886BE0181EA92E1DF91CF911A
:10ACF0000C94A453CF93DF93EC018091A01288238E
:10AD000031F0CE010296DF91CF910C94185581EA73
:10AD100092E10E945F53009739F08C179D0739F03C
:10AD2000FC0180819181F7CF81E090E002C080E05A
:10AD300090E0DF91CF9108952F923F924F925F92D2
:10AD40006F927F928F929F92AF92BF92CF92DF923B
:10AD5000EF92FF920F931F93CF93DF93CDB7DEB7A0
:10AD6000E8970FB6F894DEBF0FBECDBFE3EDFAE271
:10AD70002081318142815381EFECFAE250804180A1
:10AD800032802380EBECFAE28081898391819A837F
:10AD9000A281AB836380E7ECFAE2B081BC8381815E
:10ADA0008D8392819E83A381AF83E3ECFAE2B0812D
:10ADB000B8878181898792819A87A381AB87EFEBDE
:10ADC000FAE2B081BC8781818D8792819E87A381C1
:10ADD000AF87EBEBFAE2B081B88B8181898B9281EE
:10ADE0009A8BA381AB8BE7EBFAE2B081BC8B8181BC
:10ADF0008D8B92819E8BA381AF8BE3EBFAE2B081C6
:10AE0000B88F8181898F92819A8FA381AB8FEFEA6E
:10AE1000FAE2B081BC8F81818D8F92819E8FA38158
:10AE2000AF8FEBEAFAE2B081B8A3818189A3928166
:10AE30009AA3A381ABA3E7EAFAE2B081BCA3818124
:10AE40008DA392819EA3A381AFA3E3EAFAE2B0812E
:10AE5000B8A7818189A792819AA7A381ABA7EFE9BF
:10AE6000FAE2B081BCA781818DA792819EA7A381C0
:10AE7000AFA7EBE9FAE2B081B8AB818189AB9281EF
:10AE80009AAB7380E7E9FAE2B080A1809280838078
:10AE9000E3E9FAE2F080E180D280C380EFE8FAE2F1
:10AEA000A081AFABB181B8AF128103812BAB3CABBA
:10AEB0004DAB5EAB0E9432635EA95F934DA94F9389
:10AEC0003CA93F932BA92F932F923F924F925F92D1
:10AED0006F922B812F932A812F9329812F932F817A
:10AEE0002F932E812F932D812F932C812F932B85A0
:10AEF0002F932A852F9329852F9328852F932F858C
:10AF00002F932E852F932D852F932C852F932B896F
:10AF10002F932A892F9329892F9328892F932F895B
:10AF20002F932E892F932D892F932C892F932B8D3F
:10AF30002F932A8D2F93298D2F93288D2F932F8D2B
:10AF40002F932E8D2F932D8D2F932C8D2F932BA1FF
:10AF50002F932AA12F9329A12F9328A12F932FA1BB
:10AF60002F932EA12F932DA12F932CA12F932BA59F
:10AF70002F932AA52F9329A52F9328A52F932FA58B
:10AF80002F932EA52F932DA52F932CA52F937F9232
:10AF90002AA92F9329A92F9328A92F938F929F92A3
:10AFA000AF92BF92CF92DF92EF92FF920F931F93D7
:10AFB00028AD2F932FA92F939F938F937F936F93F8
:10AFC000ADE9B8E28C911F928F93ECE9F8E28081B1
:10AFD0001F928F938FED9EE09F938F930E94D99045
:10AFE000E3E0FBE22081318142815381EFEFFAE21D
:10AFF0005080418032802380E3EFFAE290808180AC
:10B0000072806380EFEEFAE28081898391819A8376
:10B01000A281AB83B381BC83EBEEFAE280818D83A6
:10B0200091819E83A281AF83B381B887E7EEFAE274
:10B030008081898791819A87A281AB87B381BC8700
:10B04000E3EEFAE280818D8791819E87A281AF87AE
:10B05000B381B88BEFEDFAE28081898B91819A8B75
:10B06000B280A380EBEDFAE2F080E180D280C38071
:10B07000E7EDFAE2A081AB8BB181BC8B1281038139
:10B080000FB6F894DEBF0FBECDBF2BAB3CAB4DABC4
:10B090005EAB0E9432635EA95F934DA94F933CA9BA
:10B0A0003F932BA92F932F923F924F925F926F92D3
:10B0B0007F928F929F922C812F932B812F932A81A5
:10B0C0002F9329812F9328852F932F812F932E81C2
:10B0D0002F932D812F932C852F932B852F932A85AA
:10B0E0002F9329852F9328892F932F852F932E8592
:10B0F0002F932D852F93AF92BF922A892F93298961
:10B100002F93CF92DF92EF92FF920F931F932C8990
:10B110002F932B892F939F938F937F936F93ADE9F9
:10B12000B8E28C911F928F93ECE9F8E280811F9234
:10B130008F9380E79EE09F938F930E94D9900FB6E4
:10B14000F894DEBF0FBECDBFE8960FB6F894DEBF11
:10B150000FBECDBFDF91CF911F910F91FF90EF9068
:10B16000DF90CF90BF90AF909F908F907F906F9027
:10B170005F904F903F902F90089580E380935713F6
:10B180000895CF93DF936091571370E0C0E3D0E050
:10B19000C61BD70B6B557D4EAE010E941290CE019F
:10B1A000DF91CF910895CF92DF92EF92FF920F93AC
:10B1B0001F93CF93DF937C01C0905A13D0905B1301
:10B1C0006091571370E0E601E096C61BD70BC138BB
:10B1D000D105D8F400E310E0061B170B6B557D4E2C
:10B1E000A8010E9412906091A3127091A412809104
:10B1F000581390915913680F791FA601C701800F4A
:10B20000911F0E941290CE0102C080E090E0DF9179
:10B21000CF911F910F91FF90EF90DF90CF90089505
:10B2200090915713980F90935713089540915A1384
:10B2300050915B134817590798F02091581330919B
:10B240005913280F391F3093591320935813481B53
:10B25000590B50935B1340935A1381E090E008958B
:10B2600080E090E0089590935B1380935A130895C3
:10B2700080915813909159138B529D4E089580914F
:10B28000571390E08B559D4E089581E090E02091FA
:10B29000A3123091A412255D324111F480E090E0B8
:10B2A00008950E944559892B61F06091A312709115
:10B2B000A41240915A1350915B1385ED92E10C94C6
:10B2C0001290209158133091591321153105B9F07E
:10B2D00080915A1390915B13C096E5EDF2E1AF01B6
:10B2E000455A52414817590734F4DF01A20FB31FE2
:10B2F0004C914193F4CF1092591310925813089522
:10B300008091A3129091A412089580915A13909164
:10B310005B1308959091571380E3891B089520E3F0
:10B3200080915713281B80915A1390915B13820FC1
:10B33000911D08951F93CF93DF93EC011091571344
:10B34000812F90E08C179D076CF00E948F598C0F15
:10B350009D1F8138910530F41C1B1093571381E019
:10B3600090E002C080E090E0DF91CF911F910895BE
:10B37000CF93DF93E6EAF8E21192119288E2E63D7C
:10B38000F807D1F7CEE9D8E26CEF72E0CE010E9467
:10B390004B50229688E2C63AD807B1F7DF91CF9199
:10B3A0000895109259131092581310925B13109233
:10B3B0005A1380E38093571385ED92E19093A41282
:10B3C0008093A3120C94B859EF92FF920F931F939E
:10B3D000CF93DF9300D0CDB7DEB78C0169837A833A
:10B3E0000E94D1596981E62E7A81F72E81E8E8160C
:10B3F000F10418F080E8E82EF12CA701B801809143
:10B40000A3129091A4120E941290F0925B13E0920A
:10B410005A13C7010F900F90DF91CF911F910F9199
:10B42000FF90EF9008950F931F93CF93DF938C01BC
:10B43000EB010E94D1591093A4120093A312D09350
:10B440005B13C0935A13DF91CF911F910F91089511
:10B4500020E3E6EAF8E2DC0101900D922A95E1F79B
:10B4600088E0EEE9F8E2DB0101900D928A95E1F7C0
:10B47000089520E3FC01A6EAB8E201900D922A9516
:10B48000E1F788E0FB01AEE9B8E201900D928A9500
:10B49000E1F70895E82FF0E0EE0FFF1FEA55F74DB2
:10B4A0007183608381E090E00895E82FF0E0EE0F73
:10B4B000FF1FEA55F74D80819181089590E0880F34
:10B4C000991F8259974D0E944B5081E090E008955A
:10B4D00090E0880F991F8259974D08958115910525
:10B4E00011F00197F1F70895E091D928F091DA2849
:10B4F00090818091D82889230895E091D628F091F1
:10B50000D72880819091D828892B8083E091DB28EF
:10B51000F091DC2880819091D828892B8083089530
:10B52000E091D628F091D72890818091D8288095F5
:10B5300089238083E091DB28F091DC289081809141
:10B54000D82880958923808308951F93CF93DF9314
:10B55000E091D628F091D72890818091D8288095C5
:10B5600089238083E091DB28F091DC288081909111
:10B57000D828892B80838FEB93E00E946E5A1FB7E7
:10B58000F894E091DB28F091DC2890818091D82814
:10B5900080958923808383E890E00E946E5AE09131
:10B5A000D928F091DA28D081C091D8281FBF78948B
:10B5B0008BE393E00E946E5AE091D928F091DA284B
:10B5C00090818091D828982319F08D2F8C2301C069
:10B5D00081E0DF91CF911F9108955093DC28409333
:10B5E000DB287093D7286093D6289093DA2880932D
:10B5F000D92881E001C0880F2A95EAF78093D828DE
:10B600000C94A55ACF93DF93C82FDFB7F894E0913D
:10B61000DB28F091DC2880819091D828892B8083C9
:10B6200083E090E00E946E5ACC2351F0E091DB2839
:10B63000F091DC2880819091D82890959823908370
:10B6400087E190E00E946E5AE091D928F091DA28C3
:10B6500080819091D828892309F4C0E089E590E0A1
:10B660000E946E5AE091DB28F091DC288081909155
:10B67000D828909598239083DFBF8BE390E00E94B9
:10B680006E5A8C2FDF91CF910895CF93DF93C82FFF
:10B69000D8E08C2F81700E94025BC6958111C06832
:10B6A000D150B9F78C2FDF91CF9108958FEF0C9483
:10B6B000455BDF92EF92FF920F931F93CF93DF933F
:10B6C000E82EEB010E94A55A81112FC080EF0E9445
:10B6D000455BF12C10E488EFD82ED10E81E00E945A
:10B6E000025B082F81E00E94025B882319F000238F
:10B6F00061F01DC0011109C01E1528F0888180FF6E
:10B7000004C0E11611F0F12E01E0802F0E94025BCF
:10B710009881969501119068988311501D11DECF84
:10B7200021961111D8CF8F2D03C08FEF01C08EEF5E
:10B73000DF91CF911F910F91FF90EF90DF900895CF
:10B74000FF920F931F93CF93DF93F82EEB010E948C
:10B75000A55A209769F085E50E94455B8E01085F38
:10B760001F4F89910E94455BC017D107D1F703C0D5
:10B770008CEC0E94455B8F2DDF91CF911F910F9133
:10B78000FF900C94455B0F931F93CF93DF93DB01E6
:10B79000EC9111969C911197F0E0F92B803181F496
:10B7A000BF016E7FE3E0660F771FEA95E1F716961B
:10B7B0009C911697ECE0F0E0E91BF109E60FF71F0A
:10B7C000F7FF07C091E0EA019883F195E195F1094F
:10B7D00002C0EA011882883279F414968C91982F6D
:10B7E0009076903649F086FF02C0EE7F05C085FF57
:10B7F00002C0EC7F01C0E87FCF0144E096958795B9
:10B800004A95E1F7D9018C93EF70E801E88380E075
:10B81000DF91CF911F910F9108950F931F93CF93B5
:10B82000DF93EC018B01B80188810E94595B88830A
:10B8300081508D3F30F4F8018081883211F08031E1
:10B8400091F7DF91CF911F910F910895CF93DF93DF
:10B85000EC010E94A55ABE0184EB0E94A05B81E02E
:10B860000E94025BC82F0E94A55A81E0C11101C04D
:10B8700080E0DF91CF9108951F93CF93DF9300D0A5
:10B88000CDB7DEB7182F69837A830E94A55A0E942C
:10B89000745A69817A81882341F084E40E94A05B14
:10B8A000113029F00E947D5A02C082E001C080E080
:10B8B0000F900F90DF91CF911F9108954F925F925B
:10B8C0006F927F928F929F92AF92BF92CF92DF92B0
:10B8D000EF92FF920F931F93CF93DF93CDB7DEB715
:10B8E00029970FB6F894DEBF0FBECDBF6C015B0188
:10B8F0004A0189010E94A55AB6018EEB0E94A05B05
:10B90000CE0101967C013E019AE0690E711C27016F
:10B910000E94565BF70181937F01E615F705C1F799
:10B9200069E070E0C2010E94EC75811109C09401C8
:10B93000A501B201F60180810E94C35B80E001C0D5
:10B9400083E029960FB6F894DEBF0FBECDBFDF911E
:10B95000CF911F910F91FF90EF90DF90CF90BF900C
:10B96000AF909F908F907F906F905F904F900895D1
:10B970005F926F927F928F929F92AF92BF92CF927F
:10B98000DF92EF92FF920F931F93CF93DF93CDB788
:10B99000DEB729970FB6F894DEBF0FBECDBF582E85
:10B9A0006B015A01890160E070E08EEB0E94A05BA0
:10B9B000CE0101967C014E019AE0890E911C37015F
:10B9C0000E94565BF70181937F01E815F905C1F7E5
:10B9D00069E070E0C3010E94EC75811108C0950117
:10B9E000A601B301852D0E94C35B80E001C083E006
:10B9F00029960FB6F894DEBF0FBECDBFDF91CF9171
:10BA00001F910F91FF90EF90DF90CF90BF90AF907C
:10BA10009F908F907F906F905F9008950F931F93EA
:10BA2000CF93DF93CDB7DEB728970FB6F894DEBF7C
:10BA30000FBECDBF182F062F98E0E8E0F3E0DE013F
:10BA4000119601900D929A95E1F7242F332727FD47
:10BA5000309541E752E0249FC001259F900D349F0F
:10BA6000900D112464E670E00E942D8ACB0144E61B
:10BA7000049F800D911D1124FE013196AE01475F98
:10BA80005F4F619170E02617370711F4019603C0EC
:10BA9000E417F507B1F7112319F0919581959109F4
:10BAA00028960FB6F894DEBF0FBECDBFDF91CF91C1
:10BAB0001F910F910895EF92FF920F931F93CF93D1
:10BAC000DF93CDB7DEB72B970FB6F894DEBF0FBE6E
:10BAD000CDBFF82EE92E682F792F88E08F0D0E94B8
:10BAE0003C5C882319F084E391E243C066E471E48E
:10BAF0008FE090E00E94C65D8E01075F1F4F9801A6
:10BB0000AE01465F5F4FBE01655F7F4F8F2D9E2D5B
:10BB10000E945E5C8111E7CF88E0E8E0F3E0DE019F
:10BB2000119601900D928A95E1F7498521E732E05F
:10BB3000429FC001439F900D112464E670E00E9473
:10BB40002D8A8A8594E6899F600D711D1124FE015E
:10BB500031968191481303C06F5F7F4F03C0E01798
:10BB6000F107B9F78B85882319F0719561957109F3
:10BB7000CB012B960FB6F894DEBF0FBECDBFDF9181
:10BB8000CF911F910F91FF90EF900895DC01CB01B1
:10BB900081159105A105B10529F081509040A04083
:10BBA000B040D9F708951092B90080E28093B800B0
:10BBB000089594EA9093BC0040EA56E861E070E092
:10BBC0009091BC0097FD0BC041505109610971096A
:10BBD000411551056105710599F781E0089590912E
:10BBE000B900987F983011F09031B9F78093BB007D
:10BBF00084E88093BC0080EA96E8A1E0B0E0209160
:10BC0000BC0027FD08C00197A109B1090097A10553
:10BC1000B105A9F7E2CF8091B900887F883111F092
:10BC20008034D9F680E0089524EA34E844E920938A
:10BC3000BC009091BC0097FFFCCF9091B900987F19
:10BC4000983011F0903199F78093BB003093BC008D
:10BC50009091BC0097FFFCCF9091B900987F9032F3
:10BC600011F0983539F44093BC009091BC0094FDDC
:10BC7000FCCFDDCF08950C94D95D84E98093BC009E
:10BC80008091BC0084FDFCCF08958093BB0084E8C4
:10BC90008093BC008091BC0087FFFCCF9091B900DD
:10BCA000987F81E0983209F480E0089584EC8093D5
:10BCB000BC008091BC0087FFFCCF8091BB00089541
:10BCC00084E88093BC008091BC0087FFFCCF80910A
:10BCD000BB000895E0E1DC01FD91CD01F0933F014F
:10BCE000E150C9F780913C018F7D80933C018091A8
:10BCF0003C01877F80933C01FB0180E1919190930F
:10BD00003E018150D9F780913C01806880933C01CD
:10BD100080913D0180FFFCCF4051510980913C0151
:10BD2000806280933C0180913C01877F80933C013D
:10BD3000141615069CF4FB0180E1919190933E014D
:10BD40008150D9F780913C01806880933C018091BB
:10BD50003D0180FFFCCF40515109EACFF90180E15C
:10BD600090913E0191938150D9F781E090E0089540
:10BD70000F931F93CF93DF93EC018CE70E94145E27
:10BD80008CE70E94455E8E01005F1F4F89910E94E3
:10BD9000455EC017D107D1F7DF91CF911F910F9169
:10BDA0000C943D5E813019F440E050E002C040EC5C
:10BDB00050E060E070E08CE790E00C94321181304C
:10BDC00019F44EE050E002C048E050E060E070E05E
:10BDD0008CE790E00C94321141E050E060E070E0BC
:10BDE0008CE790E00E9432116AE67AE080E090E011
:10BDF0000C94C65D48E350E060E070E08CE790E0B2
:10BE00000E94321149E350E060E070E08CE790E07E
:10BE10000E94321144E150E060E070E08CE790E075
:10BE20000E94321148E750E060E070E08CE790E05B
:10BE30000E9432114EE550E060E070E08CE790E047
:10BE40000E9432114DE650E060E070E08CE790E037
:10BE50000E9432116CE17AE186E090E00E94C65DBA
:10BE60004CE050E060E070E08CE790E00E9432111E
:10BE700041E050E060E070E08CE790E00E94321119
:10BE800046E050E060E070E08CE790E00E94321104
:10BE90006AE67AE080E090E00C94C65DCF93DF9391
:10BEA000CDB7DEB7A2970FB6F894DEBF0FBECDBFF9
:10BEB00081E1EBE2F9E0DE01529601900D928A9564
:10BEC000E1F781E1ECE3F9E0DE01119601900D92DA
:10BED0008A95E1F70E94FA5ECE0142960E94B85E12
:10BEE00082E00E94D25E6AE67AE080E090E00E9402
:10BEF000C65DCE0101960E94B85E60E17EEA88E2EE
:10BF000090E00E94C65D80E00E94DF5E60E17EEA14
:10BF100088E290E00E94C65D4EE050E060E070E094
:10BF20008CE790E00E943211A2960FB6F894DEBF23
:10BF30000FBECDBFDF91CF910895CF92DF92EF92E8
:10BF4000FF920F931F93CF93DF9300D01F92CDB733
:10BF5000DEB7F82E042F122F213031F0223031F0CD
:10BF6000243031F0283031F090E005C091E003C07A
:10BF700092E001C093E00C3059F00E3011F494605F
:10BF800007C0003111F4986003C0023109F49C60CD
:10BF9000613059F0623011F4906207C0633011F4DF
:10BFA000906403C0643009F490669068692F70E073
:10BFB00023E030E0AE014F5F5F4F8F2D90E00E9495
:10BFC000491169E07AE180E090E00E94C65D8F2D22
:10BFD0008160F82E0E94D95D0E94565E89830E947E
:10BFE000565E8A83023119F40E94565E8B830E944A
:10BFF000565E87FDF1CF0E94605E0E943D5E69E063
:10C000007AE180E090E00E94C65D8F2D0E94D95DAC
:10C010000E94565E89830E94565E8A83023119F41B
:10C020000E94605E8B830E94605E0E943D5E39814B
:10C030002A81023149F5832F90E0A0E0B0E04B81E6
:10C040007727662731FF0EC030E0322F2227620F9C
:10C05000731F811D911D640F711D811D911D8C6FBA
:10C060009F6F0BC030E0322F2227620F731F811D9C
:10C07000911D640F711D811D911D0E943A8720E85A
:10C080003FEF4FEF57E420C0632F70E0762F662715
:10C09000620F711D882777FD8095982F0E943A873F
:10C0A0000C3029F420E030EE4FEF54E40DC00E3098
:10C0B00029F420E038EF4FEF55E406C0003131F4A9
:10C0C00020E03EEF4FEF56E40E949B862FE632E1E0
:10C0D00043E050E40E9418896B017C01612F70E0FD
:10C0E00080E090E00E943A879B01AC01C701B60155
:10C0F0000E949B860F900F900F90DF91CF911F9120
:10C100000F91FF90EF90DF90CF900895E6E4F1E07B
:10C11000808120819081308182958695869583707B
:10C1200022952F70822B832B92959F70892B0895D7
:10C130000F931F93CF93DF9300D0CDB7DEB746E0C8
:10C140006CE080E00E94C86389E18093C400109293
:10C15000C50082E08093C00080E00E9453640E948A
:10C16000F46284B784B784B784B784B7EDE5F1E3AC
:10C1700022E432E4318320833A968DB79EB70A9742
:10C18000E817F907B8F38DE499E09F938F938CE259
:10C1900090E19F938F930E94D9900E942F720E94EA
:10C1A000F75160E070E082E892E00E949F520E94A6
:10C1B000D355E0911003F091110309950E94866018
:10C1C00090E00E946B72CE0101960E9429620F904E
:10C1D0000F900F900F90882341F08CE090E19F9397
:10C1E0008F930E94D9900F900F90CE0101960E94DC
:10C1F00066500E9437628C010E943362AE014F5F2D
:10C200005F4FB8010E941F670E94A3610E940067F0
:10C210000E943B620E9459688FEF9FE09F938F932B
:10C220000E94D9908A811F928F930BEF1FE01F937A
:10C230000F930E94D99089811F928F931F930F9320
:10C240000E94D99089EF9FE09F938F930E94D9908D
:10C250000E946F72E0914D03F0914E030995E091B9
:10C260003F03F09140030995E0912603F0912703E5
:10C2700009950E946068182F0E94FD661F921F9307
:10C280001F928F9380914C038F9380914B038F93D8
:10C2900080913E038F9380913D038F938EED9FE0BD
:10C2A0009F938F930E94D990E0915703F091580388
:10C2B0000FB6F894DEBF0FBECDBF309791F0099551
:10C2C000BC0180E890E00E94198A7F936F938BEC09
:10C2D0009FE09F938F930E94D9900F900F900F90A3
:10C2E0000F9089EC9FE09F938F930E94D99060E01C
:10C2F00070E088ED92E00E949F528CEE92E00E94E6
:10C300003F7181EC9FE09F938F930E94D9900F9093
:10C310000F900F900F900F900F90DF91CF911F9182
:10C320000F9108957F936F939F938F938BEB9FE073
:10C330009F938F930E94D9900F900F900F900F9022
:10C340000F900F9008951F93CF93DF93CDB7DEB773
:10C35000A0970FB6F894DEBF0FBECDBF89E590E081
:10C360000E944592182F282F35EF380F303108F0F2
:10C37000982F9095291709F461C087E490E19F9365
:10C380008F930E94D990ECE8F0E10F900F90DE01BE
:10C39000119684918D93319680E1E439F807C9F7BD
:10C3A000F89448E050E065E770E0CE0101960E9405
:10C3B0004B92EEE7F0E1DE01119684918D93319678
:10C3C00080E1EC38F807C9F74EE050E067E670E02E
:10C3D000CE0101960E944B92E4E7F0E1DE01119656
:10C3E00084918D93319680E1EE37F807C9F74AE0E2
:10C3F00050E06DE570E0CE0101960E944B926DEC2D
:10C400007BEA87E590E00E94639260E070E085E55A
:10C4100090E00E94639260E084E590E00E94559273
:10C4200060E070E08BE590E00E9463921AE16AE1BF
:10C4300075EE89E590E00E9463927894812FA09632
:10C440000FB6F894DEBF0FBECDBFDF91CF911F9125
:10C450000895F89442E050E065E770E00E942D9264
:10C46000789480E0089587E590E00C94459285E506
:10C4700090E00C94459284E590E00C943D924091BC
:10C48000EB285091EC286091ED287091EE2890E017
:10C49000A0E0B0E0480F591F6A1F7B1F4093EB28B4
:10C4A0005093EC286093ED287093EE284091E72894
:10C4B0005091E8286091E9287091EA28480F591FA7
:10C4C0006A1F7B1F4093E7285093E8286093E92870
:10C4D0007093EA2820918B2A2223A1F04091E3282F
:10C4E0005091E4286091E5287091E628480F591F83
:10C4F0006A1F7B1F4093E3285093E4286093E5284C
:10C500007093E62808951F920F920FB60F92112490
:10C510000BB60F922F933F934F935F936F937F933D
:10C520008F939F93AF93BF93EF93FF9380915E138D
:10C5300090915F13019690935F1380935E138091A7
:10C540005D138F5F80935D138038A9F410925D13A3
:10C550008091EB289091EC28A091ED28B091EE28E5
:10C560000196A11DB11D8093EB289093EC28A09318
:10C57000ED28B093EE2880918B2A8823E1F08091FA
:10C580005C138F5F80935C138038A9F410925C1366
:10C590008091E3289091E428A091E528B091E628C5
:10C5A0000196A11DB11D8093E3289093E428A093E8
:10C5B000E528B093E6280E942F55892B11F00E94A0
:10C5C0004254FF91EF91BF91AF919F918F917F91D5
:10C5D0006F915F914F913F912F910F900BBE0F90F4
:10C5E0000FBE0F901F901895F8941092B60016BCCD
:10C5F00083EF87BD82E084BD94E095BD95B395BB84
:10C6000080936E007894089580915E1390915F13EB
:10C6100020915E1330915F1382179307A9F7089555
:10C62000009751F022E330E000002150310921153C
:10C630003105D1F70197F4CF08950F931F93CF934E
:10C64000DF93EC010E9404638C010E940463801B51
:10C65000910B8C179D07C8F3DF91CF911F910F911C
:10C66000089508950F931F936091EB287091EC2823
:10C670008091ED289091EE280091EB281091EC2804
:10C680002091ED283091EE286017710782079307FB
:10C6900059F71F910F9108951F920F920FB60F92A5
:10C6A00011241092AE020F900FBE0F901F9018959C
:10C6B0001F920F920FB60F9211240BB60F922F9369
:10C6C0003F934F935F936F937F938F939F93AF931A
:10C6D000BF93EF93FF93E091A402F091A5028081B4
:10C6E000E091AF02F091B002309709F00995FF9107
:10C6F000EF91BF91AF919F918F917F916F915F91DA
:10C700004F913F912F910F900BBE0F900FBE0F9046
:10C710001F9018951F920F920FB60F92112410922E
:10C72000BB020F900FBE0F901F9018951F920F9293
:10C730000FB60F9211240BB60F922F933F934F9386
:10C740005F936F937F938F939F93AF93BF93EF9379
:10C75000FF93E091B102F091B2028081E091BC02BE
:10C76000F091BD02309709F00995FF91EF91BF91CB
:10C77000AF919F918F917F916F915F914F913F9179
:10C780002F910F900BBE0F900FBE0F901F9018951A
:10C790009DE0899FF0011124EC55FD4FA281B381EA
:10C7A0001C92A481B5816C93A681B78188ED8C938E
:10C7B000A085B1854C9312861486138608959DE05A
:10C7C000899FF0011124EC55FD4F81E08287A08103
:10C7D000B1816C933A9680818111FDCF08951F93AA
:10C7E000CF93DF93182FEB01FE016491662329F0AC
:10C7F000812F0E94DF632196F7CFDF91CF911F91A8
:10C8000008951F93CF93DF93182FEB01888188231E
:10C8100069F08A3021F46DE0812F0E94DF63699115
:10C820006D30A1F3812F0E94DF63F0CFDF91CF91B4
:10C830001F910895CF93DF93CDB7DEB79E01285F98
:10C840003F4F4E815F8160E470E080E693E10E949B
:10C85000969160E673E18D810E940164DF91CF9132
:10C860000895CF93C82F8A3031F46DE08091A013E2
:10C870000E94DF6302C08D3029F06C2F8091A013DD
:10C880000E94DF6380E090E0CF9108959DE0899F52
:10C89000F0011124EC55FD4F748763870895682FCC
:10C8A00080E00C94DF638093A01386E992E090937C
:10C8B000583180935731089584B7877F84BF88E1CA
:10C8C0000FB6F89480936000109260000FBE089538
:10C8D0002FE088E190E00FB6F894A895809360006F
:10C8E0000FBE209360000895A895089588E10FB6C3
:10C8F000F89480936000109260000FBE0895F89441
:10C9000028E088E190E00FB6F894A8958093600045
:10C910000FBE20936000FFCF8091F6288091F6280B
:10C9200090E0089540E06FE181E491E00C94F569B6
:10C93000E9E3F1E0808180818D7F80838DE090E06C
:10C940000197F1F723E040E06FE182E491E00E947B
:10C95000FF6983E090E00197F1F708959091390124
:10C9600091FD0AC0282F803108F02FE040E06FE0F1
:10C9700085E491E00C94FF6908958091390181FD6F
:10C980000EC040E06FE181E491E00E94F569282F3C
:10C990002F7E81E090E0213021F080E0089580E05A
:10C9A00090E008958091390181FD10C040E06FE171
:10C9B00081E491E00E94F5698F3131F0982F9F7EDC
:10C9C000915081E0923018F480E0089581E008955C
:10C9D0000E94D2648823E1F30895CF93DF93C82F98
:10C9E0000E94E8640E949264D82FC81789F1C83069
:10C9F00019F40E94986425C0C93121F4863189F464
:10CA000029E005C0C63169F4893159F426E040E0D7
:10CA10006FE182E491E00E94FF69E3E0F0E031978A
:10CA2000F1F72C2F40E06FE182E491E00E94FF6972
:10CA3000D83019F4E9E6F1E002C0E3E0F0E0319724
:10CA4000F1F70E9492648C1719F083E490E002C021
:10CA500080E490E0DF91CF9108950E94E864109205
:10CA60008B2A0E94986480913901826080933901F9
:10CA700080910E2B8823D9F180919400909195009C
:10CA800040911F2B5091202B84179507A0F4809183
:10CA9000EB2A9091EC2AA091ED2AB091EE2A8C57C6
:10CAA000914EAF4FBF4F8093EB2A9093EC2AA09307
:10CAB000ED2AB093EE2A2091940030919500241B2A
:10CAC000350B8091EB2A9091EC2AA091ED2AB09140
:10CAD000EE2A820F931FA11DB11D8093EB2A909324
:10CAE000EC2AA093ED2AB093EE2A10920E2B80919F
:10CAF000102B8823D9F1809194009091950040915A
:10CB0000232B5091242B84179507A0F48091F32AAE
:10CB10009091F42AA091F52AB091F62A8C57914E63
:10CB2000AF4FBF4F8093F32A9093F42AA093F52A36
:10CB3000B093F62A2091940030919500241B350B78
:10CB40008091F32A9091F42AA091F52AB091F62AC7
:10CB5000820F931FA11DB11D8093F32A9093F42A95
:10CB6000A093F52AB093F62A1092102B0895809185
:10CB70008B2A882381F080912414811104C00E94A3
:10CB8000D264811106C081E08093221481E090E09C
:10CB900008950E942D6580E090E0089580919400B2
:10CBA000909195009093242B8093232B21E0209348
:10CBB000102B8091390181FD08C08091390181FDE0
:10CBC0001AC086E10E94ED6416C020938A2A8091E3
:10CBD0009400909195009093202B80931F2B20938D
:10CBE0000E2B809139018D7F8093390180918A2AA3
:10CBF0008111FCCFE2CF81E080938B2A0895809150
:10CC00008B2A81110AC080912414882321F081E0AD
:10CC10008093231402C00E94CE6581E090E00895C5
:10CC20001F93CF93DF931F92CDB7DEB78FB7898362
:10CC300080912414811126C0F89480918B2A882336
:10CC400051F08091390181FD1BC00E94D26488237C
:10CC5000B9F080E003C00E94FF6581E020914701A8
:10CC600091E02E3008F090E0192F119581110E946B
:10CC7000B765107429F089818FBF81E090E004C00E
:10CC800089818FBF80E090E00F90DF91CF911F915D
:10CC9000089580912314882321F00E94CE6510927C
:10CCA000231480912214882321F00E942D65109274
:10CCB00022141092241408950F931F93AB0121E0C6
:10CCC000209324140091CF2A1091D02A2091D12AA8
:10CCD0003091D22A0F5F1F4F2F4F3F4F0093CF2A23
:10CCE0001093D02A2093D12A3093D22A22E0260F03
:10CCF00027FF0CC08091882A9091892A01969093F1
:10CD0000892A8093882A0FEF1FEF07C0BC0181EAB0
:10CD100093E10E94129000E010E00E944966C80171
:10CD20001F910F9108958093261408950E94926494
:10CD3000823011F0823111F480E0089581E008958D
:10CD400008958FEF80934E0122E044E060EF8CE67F
:10CD500091E00E94FF6925E041E06EE08CE290E006
:10CD60000E94FF6980E880936F0180914601809363
:10CD70006D0121E045E060E284E491E00C94FF69FC
:10CD80008DEF93E00197F1F70E94EB691092FF2875
:10CD9000109281291092032A1092FE281092FD28E9
:10CDA000E9E3F1E080818E7F808380818D7F8083C5
:10CDB0008DE090E00197F1F7E9E3F1E08081816097
:10CDC000808323E040E06FE182E491E00E94FF690C
:10CDD0008DEF93E00197F1F780915D0180915E0105
:10CDE0000E94A16660E070E08EEB92E00E949F528C
:10CDF0000E94CE6581E090E0089580912514089509
:10CE0000CF93DF931F92CDB7DEB789830E94E8648A
:10CE1000898180932514282F40E06FE188E491E018
:10CE20000F90DF91CF910C94FF690E940067809171
:10CE3000390181FD03C086E00C94ED640895FA0188
:10CE4000809362019093630160936001709361012C
:10CE50003097C1F0808180936B01818180936A015A
:10CE600082818093690183818093680184818093AA
:10CE70006701858180936601868180936501878142
:10CE80008093640108958EEB92E00E94C05281E08D
:10CE90008093F6288091F7289091F8280196909336
:10CEA000F8288093F72881E090E008958091FE288B
:10CEB00092E8899FF0011124E150F74D10828F5FB5
:10CEC000833018F48093FE2802C01092FE28E0916F
:10CED000FE2882E8E89FF0011124E150F74D80819F
:10CEE00081110C9443671092F62808951F93CF93F5
:10CEF000DF932091FE2812E8129F90011124D9019E
:10CF0000A150B74D4C91411103C00E94566793C088
:10CF10005091390151FD8FC050918B2A552309F44E
:10CF20008AC047FF16C00E9456678091BF2A909121
:10CF3000C02AA091C12AB091C22A0196A11DB11D9B
:10CF40008093BF2A9093C02AA093C12AB093C22A8B
:10CF500072C04330B0F40E9456678091BB2A909112
:10CF6000BC2AA091BD2AB091BE2A0196A11DB11D77
:10CF70008093BB2A9093BC2AA093BD2AB093BE2A6B
:10CF80005AC050E0EA0122976C177D07B0F40E9466
:10CF900056678091B72A9091B82AA091B92AB0918A
:10CFA000BA2A0196A11DB11D8093B72A9093B82A81
:10CFB000A093B92AB093BA2A3EC0B9016050774D08
:10CFC0000E941290E091FE281E9FF0011124E1586A
:10CFD000F64D80818093EF280E945667809147012B
:10CFE0008093F0289091F528992311F0891710F477
:10CFF0008093F5286091F02870E084E00E944A5AFE
:10D000006091EF2870E083E00E944A5A4091D32A51
:10D010005091D42A6091D52A7091D62A4F5F5F4FE4
:10D020006F4F7F4F4093D32A5093D42A6093D52AD1
:10D030007093D62A02C0C0E0D0E0CE01DF91CF913C
:10D040001F910895CF93DF93EC0188819981009718
:10D05000E9F08730954021F01982188283E026C0DC
:10D060006238C1F41092F6280E94D1590E943859B2
:10D0700060E870E00E947667181619066CF40E944A
:10D080003359E0915103F0915203099587E095E0FF
:10D090009983888381E00AC08091F3289091F428D5
:10D0A00001969093F4288093F328F0CFDF91CF91ED
:10D0B000089591E0909324140E94AE640C94496604
:10D0C0008091390181FD06C040E06FE085E491E088
:10D0D0000C94F56980E108950F931F93CF93DF932C
:10D0E000182F21E02093241400918B2A809139017C
:10D0F00081FF16C080919400909195009093202B11
:10D1000080931F2B20930E2B20938A2A8091390124
:10D110008D7F8093390180918A2A8111FCCF00E0B4
:10D120000E94E86480918B2A882309F43FC0809193
:10D13000102B8823D9F18091940090919500E09173
:10D14000232BF091242B8E179F07A0F44091F32AF4
:10D150005091F42A6091F52A7091F62A4C57514E5D
:10D160006F4F7F4F4093F32A5093F42A6093F52A30
:10D170007093F62A20919400309195002E1B3F0B5E
:10D180004091F32A5091F42A6091F52A7091F62A81
:10D19000420F531F611D711D4093F32A5093F42ACF
:10D1A0006093F52A7093F62A1092102B8091390122
:10D1B00081FD03C089E10E94ED6486E00E94555A1A
:10D1C000892B51F00E946068C82F86E00E94555A52
:10D1D00081500E94AE6402C0C0E0D0E02091940073
:10D1E000309195003093222B2093212B81E0809366
:10D1F0000F2BF894809139018260809339018091DE
:10D2000039018D7F8093390162E0610F81EA93E1FA
:10D210000E94306A78942091852A3091862A2F5F67
:10D220003F4F3093862A2093852A0E94E86445E088
:10D2300060EE82E491E00E94F569182F86E00E947A
:10D24000555A892B19F08C2F0E94AE64002319F0D7
:10D250000E94CE6502C00E942D6580910F2B88230D
:10D26000D9F18091940090919500E091212BF0915B
:10D27000222B8E179F07A0F44091EF2A5091F02A9D
:10D280006091F12A7091F22A4C57514E6F4F7F4FA7
:10D290004093EF2A5093F02A6093F12A7093F22A78
:10D2A00020919400309195002E1B3F0B4091EF2A66
:10D2B0005091F02A6091F12A7091F22A420F531F87
:10D2C000611D711D4093EF2A5093F02A6093F12A5B
:10D2D0007093F22A10920F2B80918B2A882361F091
:10D2E00020919400309195003093242B2093232B90
:10D2F00081E08093102B07C023E040E06FE182E4DF
:10D3000091E00E94FF690E9449661130E9F01330F4
:10D31000A9F48091C72A9091C82AA091C92AB091F6
:10D32000CA2A0196A11DB11D8093C72A9093C82ACD
:10D33000A093C92AB093CA2A12E009C0153031F06F
:10D34000173029F411E003C010E001C013E0812F71
:10D3500090E0DF91CF911F910F910895CF93DF93CC
:10D36000EB010E945C66009729F4CE010E946C6874
:10D37000009751F02091882A3091892A2F5F3F4FE2
:10D380003093892A2093882ADF91CF910895CF93F3
:10D39000DF9380918B2A811104C00E94FF65D1E048
:10D3A00001C0D0E00E949264863111F0813119F4FD
:10D3B000C091470109C040E06FE186E491E00E941E
:10D3C000F569C82FCC0FC80FD1110E94B7658C2FFB
:10D3D000DF91CF9108951092281410922714EFE650
:10D3E000F0E08081806280830895FC018081862343
:10D3F00090E002C0959587954A95E2F70895F894D4
:10D40000FC015081362F30955323042E01C0220F8A
:10D410000A94EAF72623522B50837894089540917A
:10D420007B01FC014193A0E8B1E050E8540F9D015D
:10D430002F5F3F4F6C916193521711F0D901F7CFD5
:10D440004150E42FF0E0E058FE4F2181FC01E0580C
:10D45000FF4F2083FC01EF57FF4F21E02083089509
:10D4600060938001E1E8F1E061589F012F5F3F4F39
:10D47000DC014D91CD014083621711F0F901F5CF28
:10D4800008951F920F920FB60F9211240BB60F92B0
:10D490002F933F934F935F936F937F938F939F93BC
:10D4A000AF93BF93EF93FF93809147018093F02850
:10D4B0008091FD2822E8829FC00111248150974D60
:10D4C0000E940F6A8091FD288F5F833018F480934B
:10D4D000FD2802C01092FD280E944367FF91EF9142
:10D4E000BF91AF919F918F917F916F915F914F917C
:10D4F0003F912F910F900BBE0F900FBE0F901F907A
:10D5000018951F920F920FB60F9211240F900FBE15
:10D510000F901F9018951F920F920FB60F92112423
:10D520000F900FBE0F901F9018951F920F920FB67D
:10D530000F9211240F900FBE0F901F9018951F92FD
:10D540000F920FB60F92112410928A2A0F900FBEDD
:10D550000F901F9018951F920F920FB60F921124E3
:10D5600010928A2A0F900FBE0F901F9018951F924D
:10D570000F920FB60F9211248F9381E08093F628BB
:10D580008F910F900FBE0F901F9018951F920F92C2
:10D590000FB60F92112410928A2A0F900FBE0F908F
:10D5A0001F9018951F920F920FB60F9211248F9310
:10D5B0009F9380912714909128140196909328149A
:10D5C000809327149F918F910F900FBE0F901F9003
:10D5D0001895CF92DF92EF92FF920F931F93CF9304
:10D5E000DF937C018B016A0189E294E10E945F5321
:10D5F000EC01009751F0EC81FD81309711F0C801EA
:10D600000995CE010E940754F3CFA601B801C701C6
:10D61000DF91CF911F910F91FF90EF90DF90CF900E
:10D620000C94E9500F931F93CF93DF9300D0CDB7A5
:10D63000DEB78091932A9091942AA091952AB09177
:10D64000962A0196A11DB11D8093932A9093942A46
:10D65000A093952AB093962A0E947C6D8C0189E252
:10D6600094E10E945F53009779F0DC011296ED91EE
:10D67000FC911397309729F089839A8309959A81B1
:10D6800089810E940754EFCF0115110549F0C801A7
:10D690000F900F90DF91CF911F910F910C94E0505C
:10D6A0000F900F90DF91CF911F910F9108950E94DD
:10D6B0006F720E94D1590E94A36B8DE393E0909307
:10D6C0008E2A80938D2A0E947A6D2FEF31E040E000
:10D6D0005EE160E074E082E090E00C94436DBC0198
:10D6E00089E294E10C94BF53BC0189E294E10C946B
:10D6F000A453CF93DF93EC0140918F2A5091902A4D
:10D700006091912A7091922A4F5F5F4F6F4F7F4FC8
:10D7100040938F2A5093902A6093912A7093922A73
:10D720000E948F6D009761F00E945159E091410372
:10D73000F0914203BE0189EE9AE6099581E090E0FE
:10D74000DF91CF9108958FE294E10C945B530F9396
:10D75000CF93DF93EC017B836A8318865F834E83CC
:10D76000BC018FE294E10E94BF53E0912B14F09131
:10D770002C14309749F04C815D8101E020E030E0CD
:10D7800068858A819B810995DF91CF910F910895DA
:10D79000BC018FE294E10C94A4530F93DC01189622
:10D7A0001C921897E0912B14F0912C14309759F09B
:10D7B00000E020E030E040E050E060E012968D9123
:10D7C0009C91139709950F9108950F93DC01AB017C
:10D7D00014962D913C91159781E018968C9318978B
:10D7E00015967C936E931497E0912B14F0912C1462
:10D7F000309739F000E061E012968D919C9113977B
:10D8000009950F9108950F93DC01E0912B14F0918D
:10D810002C14309771F014964D915C91159701E09E
:10D820009A0118966C91189712968D919C91139766
:10D8300009950F910895E0912D14F0912E143097D1
:10D8400009F00994089590932E1480932D1408954F
:10D8500090932C1480932B1408958FE294E10C94F0
:10D860005F53EF92FF920F931F93CF93DF938C013F
:10D87000EB017A018FE294E10E945F530097D9F0A7
:10D88000DC0112962D913C9113972C173D0781F4E2
:10D890001696ED91FC911797309769F09701AE01BC
:10D8A000B801DF91CF911F910F91FF90EF900994F4
:10D8B0000E940754E3CFDF91CF911F910F91FF900A
:10D8C000EF9008950895CF93DF93C2E6D4E1688185
:10D8D000798120E030E042E85CE68CE494E10E944B
:10D8E000DF550E946D72688179810E94198A20E05B
:10D8F00030E046E95CE6BC018CE394E1DF91CF9136
:10D900000C94DF55809162149091631420916014FF
:10D9100030916114880F991F2817390708F4C9013D
:10D9200090936314809362140C94636CCF93DF9391
:10D930000E94D1590E943859EC01198218820E9424
:10D940002D6C28813981009719F1FC014085442311
:10D95000F9F0FC0142815381F901EE0FFF1FEE0F38
:10D96000FF1FEC0FFD1F53834283FC01448155814F
:10D970002F5F3F4FF901EE0FFF1FEE0FFF1FEC0F60
:10D98000FD1F51834083398328830E940754D9CFD8
:10D99000C901880F991F880F991F02960E94335959
:10D9A00088819981892B31F081E394E1DF91CF91D6
:10D9B0000C94B750DF91CF910895AF92BF92CF9260
:10D9C000DF92EF92FF920F931F93CF93DF9300D0DC
:10D9D000CDB7DEB76B010E943859FC01008111817F
:10D9E0001A8309830C30110518F4E12CF12C0DC0B9
:10D9F0001F930F938BE699E09F938F930E94C7909C
:10DA00000F900F900F900F9021C0E016F106F1F0EB
:10DA10000E943859F701EE0FFF1FEE0FFF1FE80FAE
:10DA2000F91FA280B3800E943859FFEFEF1AFF0A56
:10DA3000F701EE0FFF1FEE0FFF1FE80FF91F4081E8
:10DA40005181B501C6010E94316CDFCF0F900F905C
:10DA5000DF91CF911F910F91FF90EF90DF90CF90CA
:10DA6000BF90AF9008950F93013059F480915C14EA
:10DA700090915D1490936314809362140F910C94B1
:10DA8000636C0F910895EF92FF920F931F93CF93C2
:10DA9000DF938B01EA0179014AE253E0BC0181E3A3
:10DAA00094E10E949B5010935D1400935C14D093FA
:10DAB0005F14C0935E14F0926114E092601483E3EB
:10DAC0009DE6DF91CF911F910F91FF90EF900C9405
:10DAD000286C8CE494E10E9463568CE394E10E94EC
:10DAE000635681E394E10C94B55080916214909157
:10DAF000631408950C94F550CF93DF93E0912E03B7
:10DB0000F0912F030995EC01009729F06A817B8140
:10DB100081E00E944A5ACE01DF91CF9108950F9380
:10DB20001F93CF93DF93EC01E0913003F091310329
:10DB300009958C016A817B8181E00E944A5A81E0CB
:10DB400090E0012B11F480E090E0DF91CF911F91E4
:10DB50000F910895E0913203F0913303099420E08E
:10DB600030E00296FC0132974081442331F0FC0101
:10DB700031974081240F311DF4CFC9010895FC0174
:10DB8000208130E0322F22278181282B02C0220FF2
:10DB9000331F6A95E2F7832F9927FA01EC5CFC4F5B
:10DBA000208130E08223932328E030E0241B350BD2
:10DBB00002C0969587952A95E2F708956F927F9215
:10DBC0008F929F92AF92BF92CF92DF92EF92FF928D
:10DBD0000F931F93CF93DF938C01EB016A017901BF
:10DBE0002830310524F4A901B601CE014AC05901FB
:10DBF00023E0B594A7942A95E1F74115510521F04A
:10DC00004801612C712C03C0D801FB0120C048E001
:10DC100050E0B601CE01860D971D0E94BF6DF40144
:10DC200081934F01FFEF6F1A7F0A6A147B047CF324
:10DC3000C501B7FE02C080E090E0A70147705527FC
:10DC40004115510511F1080F191FB60118C0CF0178
:10DC50008C1B9D0B8A159B051CF481918D93F7CF2E
:10DC6000C501B7FE02C080E090E0A70147705527CC
:10DC70004115510551F0080F191F60E070E08C0F3D
:10DC80009D1F0E94BF6DF8018083DF91CF911F918E
:10DC90000F91FF90EF90DF90CF90BF90AF909F904B
:10DCA0008F907F906F9008958F929F92AF92BF92C6
:10DCB000CF92DF92EF92FF920F931F93CF93DF9358
:10DCC00000D0CDB7DEB70E9438598C0182E090E0D9
:10DCD0000E941659892B19F480E090E05DC0F8018C
:10DCE000818190E0982F88272081820F911D0E94CA
:10DCF00006517C01009781F30E9438594C01F701CD
:10DD00002681822F86958695869590E0422F4770D2
:10DD100021E030E011F420E030E0820F931F0E94F8
:10DD20001659892BC9F2F70104811581C12CD12C18
:10DD3000F8018081882379F1F801A180B12CB60126
:10DD400033E0759567953A95E1F7A6014770552739
:10DD5000680D791D883168F09501CE0101960E9409
:10DD6000DE6DBE016F5F7F4FF80180810E945E5AB9
:10DD70000DC01A8219829501CE0101960E94DE6DB6
:10DD800069817A81F80180810E944A5ACA0CDB1CA1
:10DD90000E5F1F4FCDCFC7010F900F90DF91CF9136
:10DDA0001F910F91FF90EF90DF90CF90BF90AF90B9
:10DDB0009F908F900895DC0150E0E0E1F0E0E61BD9
:10DDC000F70BE21BF30B02C0440F551FEA95E2F775
:10DDD0008C91852B8C9311968C911197842B119695
:10DDE0008C9308956F927F928F929F92AF92BF9281
:10DDF000CF92DF92EF92FF920F931F93CF93DF9317
:10DE00008C016B01EA017901283031051CF448814D
:10DE1000C8015CC0390153E0759467945A95E1F7E5
:10DE20006115710521F04E01A12CB12C03C0D80160
:10DE3000FE0127C0F40141914F0128E030E0B60116
:10DE4000C8018A0D9B1D0E94DB6EFFEFAF1ABF0A4F
:10DE5000A614B7047CF3C30177FE02C080E090E013
:10DE60009701277033272115310509F43FC0C80FEA
:10DE7000D91F488150E0B601621B730B685F7F4F6A
:10DE80001CC0CF018C1B9D0B861597051CF481913E
:10DE90008D93F7CFC30177FE02C080E090E0970139
:10DEA000277033272115310509F1C80FD91F488183
:10DEB00050E068E070E0621B730B02C05595479517
:10DEC0006A95E2F760E070E0800F911FDF91CF91DB
:10DED0001F910F91FF90EF90DF90CF90BF90AF9088
:10DEE0009F908F907F906F900C94DB6EDF91CF911D
:10DEF0001F910F91FF90EF90DF90CF90BF90AF9068
:10DF00009F908F907F906F9008956F927F928F92E5
:10DF10009F92AF92BF92CF92DF92EF92FF920F93B8
:10DF20001F93CF93DF9300D0CDB7DEB78C01FC01F8
:10DF30008681E82EE694E694E694F12C282F27704B
:10DF400081E090E011F480E090E0E80EF91EC70156
:10DF500002960E949A59009709F445C00E943F59C1
:10DF6000F8012281FC012083F8012381FC01218337
:10DF70000E943F5902965C01A70160E070E00E9498
:10DF80001B90F80104811581E12CF12CF8018081AE
:10DF9000882339F1F8018180912C670163E0D594E1
:10DFA000C7946A95E1F73701F7E06F227724CA0C2E
:10DFB000DB1C883128F00E94685A9401AC0108C02B
:10DFC0000E94555A9A8389839401AE014F5F5F4F37
:10DFD000B301C6010E94F26EE80CF91C0E5F1F4FE0
:10DFE000D5CF81E090E00F900F90DF91CF911F91FE
:10DFF0000F91FF90EF90DF90CF90BF90AF909F90E8
:10E000008F907F906F900895E0914F03F0915003AF
:10E010000994E0912803F09129030994E0915303B6
:10E02000F09154030994E0915503F091560309943B
:10E0300080E090E008950895E0912003F09121039D
:10E04000099480E090E008950F931F93CF93DF939E
:10E05000CDB7DEB7E0970FB6F894DEBF0FBECDBFE9
:10E060000E9485598C010E943859AE014F5F5F4F65
:10E07000602F0E94F477882309F446C088A998018C
:10E08000281B3109C9010E941659892BE9F12E81FB
:10E0900021110CC0BE016A5E7F4F88E10E945E5A6A
:10E0A000E0914303F091440309952EC08A859B8536
:10E0B0008D3C3BEA930711F0019631F5223019F0BF
:10E0C00088E090E002C082E090E001979C012F5F21
:10E0D0003F4F12161306F4F6E1E0F0E0EC0FFD1FDF
:10E0E000E80FF91F23852F3F81F3BE01645F7F4F47
:10E0F00089E10E945E5A89E10E94685A6CE978E2DF
:10E100000E945450892B31F6E0960FB6F894DEBF8A
:10E110000FBECDBFDF91CF911F910F910895AF92A8
:10E12000BF92CF92DF92EF92FF920F931F93CF9304
:10E13000DF93CDB7DEB7E0970FB6F894DEBF0FBE22
:10E14000CDBF8C016B01CE0101967C0180E3F7010C
:10E1500011928A95E9F781E089838CE00E94555AF3
:10E160008C831D821F828091661491E0980F90939A
:10E170006614898783E0B82EB8868DEC9BEA9B876E
:10E180008A8789E10E94685A6CEF72E00E945450BD
:10E19000892B31F082E08E838FEF8C878D8709C0C9
:10E1A00089E10E94685ABC01CE010C960E944B5036
:10E1B000BE828DEC9BEA9D8B8C8B6CE978E2CE0164
:10E1C00046960E944B500E9438599FA78EA70E94E6
:10E1D000855988ABC7010E94ED76B82E90E00E9469
:10E1E0009A59892B31F10E943F59BC014B2DC7012F
:10E1F0000E940B77E0901603F09017030E948F594E
:10E200005C010E943F59B501F701099501151105FF
:10E2100081F0009739F0019761F441E050E064E04B
:10E2200070E004C041E050E060E070E0C601F80139
:10E230000995E0960FB6F894DEBF0FBECDBFDF9113
:10E24000CF911F910F91FF90EF90DF90CF90BF90F3
:10E25000AF9008950E946D7280936614E091200340
:10E26000F09121030994892B29F0E0912003F0918A
:10E27000210304C0E0912203F09123030994CF937A
:10E28000DF93EC0189919991009729F060E070E0AB
:10E290000E949F52F7CFDF91CF910895CF93DF93E4
:10E2A000EC0189919991009719F00E94F151F9CFF1
:10E2B000DF91CF910895CF93DF93EC017B836A8345
:10E2C0000E94046399838883DF91CF910895FC01B4
:10E2D0008081918122813381820F931F918380837A
:10E2E0000895CF93DF93EC010E94046399838883A0
:10E2F000DF91CF910895CF93DF93EC010E940463E7
:10E3000028813981821B930B9C012F5F3F4F81E055
:10E3100090E04A815B814217530710F080E090E063
:10E32000DF91CF910895CF93DF93FC01C281D38118
:10E3300080819181C80FD91F0E9404639E01281B10
:10E34000390BC901DF91CF910895CF93DF93E5E1B8
:10E35000FBE2C7EDDAE2A9E0BBE211921192199259
:10E360001992199219921D928BE2ED32F807A9F7D2
:10E37000DF91CF910895CF93DF93FC01E75FF44DD8
:10E3800040819C01220F331F220F331F442301F1D0
:10E39000A0919400B0919500FC01EE0FFF1FEB5E81
:10E3A000F44D80819181AD01481B590BCA01E901EF
:10E3B000C952D54D488159816A817B81480F591FC7
:10E3C000611D711D488359836A837B83B183A08358
:10E3D000F901E952F54D6081718182819381DF916C
:10E3E000CF91089560E070E0CB010895FC01EE0F3D
:10E3F000FF1FEE0FFF1FE952F54D408351836283EB
:10E4000073830895CF93DF9329E03BE2C7EDDAE20F
:10E41000E5E1FBE2D9018D919D018823B9F040919E
:10E4200094005091950080819181BA01681B790B0D
:10E4300088819981AA81BB81860F971FA11DB11D7B
:10E4400088839983AA83BB83518340832496329621
:10E45000BBE225313B07F1F6DF91CF9108950C9493
:10E460007C760F931F93FC01CB0140916714509170
:10E470006814338322831583048371836083F0934C
:10E480006814E0936714452B11F40E94967680E09F
:10E4900090E01F910F9108958091671490916814F6
:10E4A0000097C1F01092681410926714DC01149662
:10E4B0006D917C9115971296ED91FC9113970995AA
:10E4C000E0916714F0916814309721F08081918178
:10E4D0000C94967608950C94A58C0C94A18C80EDE8
:10E4E00092E00E94D65288EC92E00C94D652CF93E0
:10E4F000DF930E944559892BA9F088EC92E00E9495
:10E50000F452EC01009721F10E9485599983888388
:10E510000E9480599B838A83CE0104960E94C15831
:10E520008CAB14C080ED92E00E94F452EC01009795
:10E5300079F002960E94D35899838883BE016E5465
:10E540007F4FCE018E579F4F0E94285ACE0102C0A6
:10E5500080E090E0DF91CF910895BC016E547F4F31
:10E560008E579F4F0C94285ACF93DF93EC01BC0138
:10E5700080ED92E00E943E53BE01892B19F080EDA0
:10E5800092E009C088EC92E00E943E53892B39F05A
:10E59000BE0188EC92E0DF91CF910C941953DF918A
:10E5A000CF9108950F931F93CF93DF93EC01BC019C
:10E5B00080ED92E00E943E53892B91F0FE01619123
:10E5C0007191CF010E94E459BE016E547F4FCE017C
:10E5D0008E579F4FDF91CF911F910F910C94395A15
:10E5E000BE0188EC92E00E943E53892BD1F00E943C
:10E5F000D159688179818A819B810E94E4598CA9D3
:10E6000090E00E949A590CA910E00E943F59BE0167
:10E610006C5F7F4FA801DF91CF911F910F910C94F8
:10E620001290DF91CF911F910F910895CF93DF93B7
:10E63000EC01BC0180ED92E00E943E53892B19F061
:10E64000CE0102960CC0BE0188EC92E00E943E53BF
:10E65000892B19F08A819B8102C080E090E0DF91D4
:10E66000CF910895FC01808191810895860F911DBD
:10E67000860F911D8E579F4F0895860F911D860F0F
:10E68000911D8E579F4FFC018081918108950895BF
:10E6900086EC9AE10E941855892B21F086EC9AE1CC
:10E6A0000C9405550895E091B21AF091B31A309781
:10E6B00009F0099480E00895EF92FF920F931F9361
:10E6C000CF93DF937C01EA01FC0180819181009767
:10E6D00041F08C30934071F1F7011182108283E098
:10E6E000F2C080E024E0829FF0011124EC54F54E4A
:10E6F000118210828F5F8430A8F38093B11A8091C9
:10E70000EC119091ED119093C51A8093C41A0E9458
:10E71000EA5180932D2B60E470E086EC9AE10E9430
:10E72000F1540E946A798CE093E0F7019183808331
:10E7300081E0C9C06230D9F480912E2B90912F2BAB
:10E74000892B89F380913F2B863029F48091572BB8
:10E7500081FD0E94487381E00E94A87A80912E2B4F
:10E7600090912F2B892BF9F20E946C75DCCF6330CE
:10E7700060F5611114C02097B1F2D0933C30C09382
:10E780003B3083E00E94A87A80912E2B90912F2B12
:10E79000892B11F00E9453730E944873C4CF6130DB
:10E7A00011F6209709F4BFCFD0933830C09337309B
:10E7B00085E00E94A87A80912E2B90912F2B892B97
:10E7C00009F4B1CF0E945373AECF6738E9F51092C8
:10E7D000B01A04EB1AE18091B01A8430B8F4F80151
:10E7E000828193818C179D0749F4808191810E94D9
:10E7F000757AF80111821082138212820C5F1F4F0A
:10E800008091B01A8F5F8093B01AE5CFE6E5F0E310
:10E81000838194818C179D0719F4148213821082CE
:10E82000B09620E3E63DF20799F7E3EDF0E381854A
:10E8300092858C179D0711F4158214823D9681E311
:10E84000E535F807A1F76FCF683809F06CCFC65CE3
:10E85000DA4109F068CF86EC9AE10E941855892BBD
:10E8600009F461CF1092B01AE091B01AE43008F0C8
:10E870005ACF20E2E29FF0011124E35CFF4C818D2E
:10E880008823D9F086EC9AE10E9405558091B01A50
:10E89000E0E28E9FC0011124835C9F4C90933C303A
:10E8A00080933B3082E00E94A87A80912E2B909139
:10E8B0002F2B892B11F00E9453738091B01A8F5F18
:10E8C0008093B01AD1CFDF91CF911F910F91FF901C
:10E8D000EF9008959093B31A8093B21A08952091FF
:10E8E000EC113091ED1160E0E4EBFAE1643098F462
:10E8F000408151814817590759F442815381421789
:10E90000530731F46093AF1A118210820C94757A18
:10E9100034966F5FEBCF6093AF1A089540E0E4EB5D
:10E92000FAE14430A8F451E0540F20813181232BC7
:10E9300061F44093AE1A918380832091EC11309161
:10E94000ED11338322830C948F7A3496452FE9CFCF
:10E950004093AE1A08952091EC113091ED11FC0115
:10E96000358F248F778F668F08952091EC11309129
:10E97000ED11FC0132872187748763870895CF9357
:10E98000DF93EA010E94187A009749F02091EC1178
:10E990003091ED11FC0132872187D487C387DF9145
:10E9A000CF9108950F931F93CF93DF9300D000D0A2
:10E9B000CDB7DEB78C01AB018FEF89838A838B8360
:10E9C0008C83B801CE0101960E94BF74009719F0A4
:10E9D000FC01158304830F900F900F900F90DF912F
:10E9E000CF911F910F91089540E050E062E088EDD3
:10E9F00092E00E94905210922F2B10922E2B08958D
:10EA0000AC0161E088ED92E00C947252AC0160E0E0
:10EA100088ED92E00C9472520F931F93CF93DF9383
:10EA20008A010E949679EC01009759F08091EC11CF
:10EA30009091ED119D8F8C8F1F8F0E8FCE010E94B4
:10EA40000675CE01DF91CF911F910F910895CF935D
:10EA5000DF93A0913B30B0913C30109719F0ED015D
:10EA60006C9605C0C0913730D0913830299680918E
:10EA7000363086FF22C01092AD1A40E0E4EBFAE196
:10EA80004430B8F42081318114968D919C91159772
:10EA90002817390759F482819381009739F0409300
:10EAA000AD1A998388831B821A8205C034964F5F02
:10EAB000E7CF4093AD1A0E944873888199810097EF
:10EAC00041F04A815B8160912D2BDF91CF910C94B5
:10EAD0009052DF91CF9108950F931F93CF93DF93BF
:10EAE00080913F2B863009F071C080912E2B909140
:10EAF0002F2B8115954009F069C0C4E9D2E0D0936D
:10EB00002F2BC0932E2B02E00093382B14E9109387
:10EB1000392B10925B2B10925A2B0E9464798095AE
:10EB2000909590935B2B80935A2B1092412B1092CF
:10EB3000402B0E945379809590959093412B809320
:10EB4000402B0E945373D0932F2BC0932E2B0093F6
:10EB5000382B1093392BA0913930B0913A30FD0108
:10EB6000E459FD4F8CE692E001900D920197E1F798
:10EB70006CE672E08EE49BE20E9412798091322B67
:10EB800080934E2B8091332B80934F2B8091342B8D
:10EB90008093502B8091352B8093512B10925B2BBF
:10EBA00010925A2B0E9464798095909590935B2BDC
:10EBB00080935A2B1092412B1092402B0E94537934
:10EBC000809590959093412B8093402BDF91CF912E
:10EBD0001F910F910C945373FC01680F791F80E013
:10EBE00048E1E617F70781F0219198E0322F3827A6
:10EBF000532F517030FD84278695513009F4806879
:10EC00002695915099F7EDCF08951F920F920FB668
:10EC10000F9211240BB60F922F933F934F935F9354
:10EC20006F937F938F939F93AF93BF93EF93FF93D4
:10EC3000809194009091950090931A2B8093192BBA
:10EC400081E080930B2B80917100807D8093710017
:10EC50000E944C7280910B2B8823D9F180919400F3
:10EC6000909195004091192B50911A2B841795077C
:10EC7000A0F48091DF2A9091E02AA091E12AB0913E
:10EC8000E22A8C57914EAF4FBF4F8093DF2A90936B
:10EC9000E02AA093E12AB093E22A209194003091D7
:10ECA0009500241B350B8091DF2A9091E02AA091DA
:10ECB000E12AB091E22A820F931FA11DB11D80931A
:10ECC000DF2A9093E02AA093E12AB093E22A1092DF
:10ECD0000B2BFF91EF91BF91AF919F918F917F91FE
:10ECE0006F915F914F913F912F910F900BBE0F90BD
:10ECF0000FBE0F901F9018959FB7F894E1E7F0E0D2
:10ED00008081807D808388B38F6288BB1092900061
:10ED1000E1E9F0E0108210929200109295001092BA
:10ED200094008081856080839FBF08952FB7F894F9
:10ED3000909399008093980088B38F6288BBE1E735
:10ED4000F0E08081826080832FBF0895CF93DF93AE
:10ED5000FC01DB0185E0EB0119928A95E9F78581D9
:10ED6000837011F082E08C938781837021F082E0C0
:10ED700012968C9312978581837081F087818370BE
:10ED800069F023893489818592852817390731F400
:10ED900081E0848312961C92129701C014828581AF
:10EDA0008370823021F0833021F080E003C082E064
:10EDB00001C088E011968C9311978781837082300F
:10EDC00021F0833021F080E003C082E001C088E0C0
:10EDD00013968C93DF91CF910895CF93DF9300D05A
:10EDE00000D01F92CDB7DEB7BE016F5F7F4F0E948C
:10EDF000A67689819A81890F8D5F9B81890F9C817D
:10EE0000890F9D81890F0F900F900F900F900F9099
:10EE1000DF91CF9108954F925F926F927F928F9280
:10EE20009F92AF92BF92CF92DF92EF92FF920F9399
:10EE30001F93CF93DF9300D000D000D0CDB7DEB7C3
:10EE40008C017B01BE016F5F7F4F4E830E94A676CF
:10EE5000B981AA815B804C808B2F90E003962A2F8A
:10EE600030E0820F931F850D911D642D70E0860F99
:10EE7000971F5D81850F911D4E8150E048175907FE
:10EE80000CF49AC0F801818180FB662460F8712C33
:10EE900043E0660C771C4A95E1F7828180FB882469
:10EEA00080F8912C54E0880C991C5A95E1F786283B
:10EEB00080818770882A838180FBAA24A0F8B12CE6
:10EEC00085E0AA0CBB1C8A95E1F78A28848180FB27
:10EED000CC24C0F8D12C96E0CC0CDD1C9A95E1F73F
:10EEE0008C28F7018082F80145814370F4E04F9F40
:10EEF000A0011124F80186818370F0E18F9FC00189
:10EF00001124482BF8018781F0E48F9FC001112460
:10EF1000482BF7014183F8018085F7018283B230E5
:10EF200059F4F8018185F7018383F8018285F7019F
:10EF3000848395E0C92E02C083E0C82EB0E080E053
:10EF400090E0200F311FDB2EDC0C0197BA1761F027
:10EF5000A901480F591FFA01B384A7014D0D511D96
:10EF6000FA01B082BF5FEFCF9D2DF2E05F120EC0BD
:10EF7000D701AD0DB11DF80183898C9381E08D0D12
:10EF8000D701A80FB11D9E5F84898C9340E020E0DB
:10EF900030E0060F171F842F890F215031094415C7
:10EFA00061F0D801A20FB31F55965C91D701A80F4D
:10EFB000B11D5C934F5FEFCF80E026960FB6F894BB
:10EFC000DEBF0FBECDBFDF91CF911F910F91FF909C
:10EFD000EF90DF90CF90BF90AF909F908F907F90F9
:10EFE0006F905F904F900895BF92CF92DF92EF9213
:10EFF000FF920F931F93CF93DF937C01D62EEA01EC
:10F0000082E0861708F0B2C0F701808186FBBB243E
:10F01000B0F89181292F269526952370C92EC29488
:10F02000C694C69453E0C522382F3770388383FBCB
:10F03000332730F9398384FB332730F93A8385FB52
:10F04000882780F98B83BC822D83892F82958370DA
:10F050008E83CF8282818887222391F133818481BC
:10F0600090E0982F8827830F911D9A8789878701C1
:10F070000B5F1F4F223079F46CEF72E0CE010B96DC
:10F080000E944B50F70186818B8785818C87870191
:10F09000095F1F4F20C02330F1F4F7013D9680E057
:10F0A00090E03E2F2F2F4291DE01A80FB91F1B9633
:10F0B0004C93019688309105B1F7032F122F0BC0A6
:10F0C00087010D5F1F4F6CEF72E0CE010B960E941F
:10F0D0004B501A861986CC20B9F1B1100DC0F80139
:10F0E0002081818190E0982F8827820F911D9C8B31
:10F0F0008B8B0E5F1F4F04C089859A859C8B8B8BF1
:10F10000F2E0CF120EC06CEF72E0CE0145960E9485
:10F110004B50F80181818D8B80818E8B0E5F1F4F4C
:10F120001BC0F3E0CF1218C0085F1F4FF80180E04A
:10F1300090E02291DE01A80FB91F55962C930196FD
:10F1400088309105B1F708C06CEF72E0CE014596AA
:10F150000E944B501C8A1B8AC8018E199F092D2DB5
:10F16000281B2FA71EA70DA7D81608F480E0DF9153
:10F17000CF911F910F91FF90EF90DF90CF90BF90B4
:10F180000895FB0141505109460F571FE417F50739
:10F1900078F4208130E0322F22276181260F311D43
:10F1A000820F931F8217930708F401963296EECFD1
:10F1B000E417F50751F4208130E0322F2227820F27
:10F1C000931F8217930708F401960895CF93DF9356
:10F1D000C091392BD0E064972091382B30E0322F4A
:10F1E0002227C20FD31F48E050E062E47BE29E0179
:10F1F000280F311DC9010E94C178AE016AE47BE28B
:10F200000E94C178009721F098278927982702C08B
:10F210008FEF9FEFDF91CF9108959093DF1A809346
:10F22000DE1A0895FC015381560F5093352B872F1A
:10F2300099274281480F4093342BA181A093332B0F
:10F24000E081E093322B242F30E02817390748F46F
:10F2500081E08A0F8093332B811103C0EF5FE0932D
:10F26000322B852F90E077278617970788F44F5F1A
:10F270004093342B41110CC08091332B8F5F8093CE
:10F28000332B811105C08091322B8F5F8093322BFD
:10F290000895AB01BC0180E090E00E94C1789827FE
:10F2A00089279827089544E150E066E37BE280E0F7
:10F2B00090E00E94C178009721F09827892798272D
:10F2C00008958FEF9FEF089586E00C94E67881E132
:10F2D0000C94E67880E0E82FF0E0EE0FFF1FE35497
:10F2E000FF4C118210828F5F8430A8F380E090E29F
:10F2F000899FF0011124E35CFF4C118E8F5F8430F5
:10F30000B0F380E094E09093D91A8093D81A80E00B
:10F310009DE0989FF0011124ED52FF4C158214825C
:10F320008F5F8A30B0F38093D71A0895CF932091DE
:10F33000D81A3091D91A2F5F3F4F21154DE7340766
:10F3400010F020E030E1522F432FEDE3F0E3C0E076
:10F35000C43059F0A18DAA2329F0A481B581A41746
:10F36000B50749F3CF5FB096F3CF3093D91A209306
:10F37000D81A1092D71A20E0E0E0F0E02430E8F448
:10F3800030E2239FD0011124A35CBF4C59963C91DD
:10F390005997311104C02093D71AFD0110C037309E
:10F3A00041F4309739F05A964C915A97328D341770
:10F3B00008F0DF012F5FFD01E1CF2093D71A3097CE
:10F3C000A1F122E0218F2091DA1A24872091DB1A03
:10F3D00025872091DC1A26872091DD1A278728EDC2
:10F3E00034E0338B228B358B248B21E030E0318B62
:10F3F000208B138E21E0228F23E0208F168A20E1BC
:10F40000278B2091D81A3091D91A322723273227F7
:10F410003583248377836683DC014D915D916D9103
:10F420007C914083518362837383CF01CF91089590
:10F43000CF93DF932091D81A3091D91A2F5F3F4F85
:10F4400021154DE7340710F020E030E1522F432F13
:10F45000E7EDF0E3C0E0CA3041F0A081B181CF5FB9
:10F460003D96A417B507B9F7E9CF3093D91A209381
:10F47000D81A40E05DE04A30A0F4A1E0A40F549F08
:10F48000F0011124ED52FF4C24813581232B39F4F6
:10F490004093D71A309741F480E090E023C04A2F80
:10F4A000EACF4093D71AF8CF2091D81A3091D91AC1
:10F4B0003227232732273583248377836683009777
:10F4C00029F4108211821282138209C0EC01888112
:10F4D0009981AA81BB8180839183A283B38380E4D5
:10F4E0008087CF01DF91CF91089540E04430A0F4B0
:10F4F000E42FF0E051E0540FEE0FFF1FE354FF4CF8
:10F50000208131812817390729F44093D71A1182B5
:10F5100010820895452FEACF4093D71A089540E00E
:10F52000443098F4E42FF0E051E0540FEE0FFF1F49
:10F53000E354FF4C20813181232B29F44093D71AC7
:10F54000918380830895452FEBCF4093D71A089578
:10F55000AF92BF92CF92DF92EF92FF920F931F93E1
:10F56000CF93DF93C0913B30D0913C30843009F48D
:10F57000DCC12EE53BE230933A30209339303093B2
:10F58000312B2093302B833059F4898D8F70833049
:10F5900009F06BC088899989892B09F0DFC67FC083
:10F5A000823009F080C08091DD1A8F5F8093DD1A70
:10F5B000811113C08091DC1A8F5F8093DC1A811156
:10F5C0000CC08091DB1A8F5F8093DB1A811105C01C
:10F5D0008091DA1A8F5F8093DA1A10922F2B109293
:10F5E0002E2B1092D2301092D130298D822F8D7F08
:10F5F000853041F48A8D8F5F8A8F843109F0AEC6E1
:10F60000198EACC6222309F4A9C688899989892B49
:10F6100009F441C08A8D9FEF980F9A8F81119EC681
:10F620008B8D883031F09FEF920F923048F4853007
:10F6300039F4198E80E8809336300E94277547C5CB
:10F64000853038F493E0082E01C0990F0A94EAF748
:10F6500001C090E39A8F8F5F8B8F822F8F708330E2
:10F66000A1F048F4813009F44FC3823009F076C626
:10F670001092572B4CC3863009F4C8C4883009F463
:10F68000C5C4843009F06AC6C1C484E080933630B2
:10F690000E9427754EC52F70233009F05FC688E0A1
:10F6A0008093363009C5853019F5E0913730F091F7
:10F6B000383084819581892B09F450C610923C30F2
:10F6C00010923B3082E59BE290933A308093393040
:10F6D0009093312B8093302B1092D2301092D130F6
:10F6E00010922F2B10922E2B88E0809336301BC166
:10F6F0008091362B853409F031C60091382B10E00B
:10F70000102F00278091392B080F111D80912E2B6F
:10F7100090912F2B8017910708F420C610932F2B60
:10F7200000932E2B80913C2B8F7309F017C680918C
:10F730003D2B811113C68091CD309091CE30C09178
:10F740005903D0915A038C179D0759F44091CF303B
:10F750005091D03020915B0330915C0342175307E6
:10F76000A1F02091462B3091472B2817390709F03B
:10F77000F5C52091482B3091492B8091CF30909145
:10F78000D0302817390709F0E9C50E94537901964E
:10F7900009F0E4C580913F2B863009F429C18131FD
:10F7A000E9F1813009F0DAC580914A2B883009F0FF
:10F7B000D5C510924A2B80914C2B90914D2B873FB1
:10F7C0003FEF930710F0099601C0089690934D2BD8
:10F7D00080934C2B8091422B9091432BA091442BF2
:10F7E000B091452B8093462B9093472BA093482BA9
:10F7F000B093492B8091CD309091CE30A091CF30F5
:10F80000B091D0308093422B9093432BA093442B04
:10F81000B093452B80E480933E2B7DC50C5111099C
:10F8200010932F2B00932E2B82E59BE290933A307E
:10F83000809339308091502B9091512B892B29F056
:10F840000E946779019609F089C520914C2B30916F
:10F850004D2B2115310509F481C583ED90E390937B
:10F86000383080933730A0904A2BB0904B2B40918A
:10F870005B0350915C0360915D0370915E03A09106
:10F880005F03B09160030091422B1091432BE090F5
:10F89000442BF090452BE0913730F091383081E3E4
:10F8A000E535F80708F05AC584819581009721F164
:10F8B0002817390709F586819781009719F0A8164E
:10F8C000B906D1F4808191818C179D0729F4C280FB
:10F8D000D380C416D506B1F08617970729F4C280E5
:10F8E000D380CA16DB0671F00817190729F4828144
:10F8F0009381E816F90631F03D96F0933830E093A5
:10F900003730C9CF10923C3010923B3082E0809368
:10F91000363082E59BE29093312B8093302B10920E
:10F92000D2301092D1300E9427758091D1309091C1
:10F93000D230009709F412C59C01245E3F4F3093EA
:10F940002F2B20932E2B3093382B2093392BE091A3
:10F950003730F0913830208520933E2B21E12093E1
:10F960003F2B089698278927982790934F2B8093B1
:10F970004E2B1092512B1092502B84819581909395
:10F980004B2B80934A2B8681978190934D2B8093AC
:10F990004C2B8091CD309091CE30A091CF30B09152
:10F9A000D0308093422B9093432BA093442BB09361
:10F9B000452B80819181A281B3818093462B9093C6
:10F9C000472BA093482BB093492B8EE59BE2909355
:10F9D0003A30809339300E946779809590950097EE
:10F9E00011F48FEF9FEF9093512B8093502B93C482
:10F9F0000E946479019609F0B1C480914C2B9091DA
:10FA00004D2B009709F4AAC420914A2B30914B2B1F
:10FA10002115310509F4A2C44091422B5091432B8A
:10FA20006091442B7091452BE6E5F0E3CDE3D0E304
:10FA3000F080FF20A9F0AC81BD818A179B0781F47B
:10FA4000AE81BF812A173B0759F4A881B9814A17B3
:10FA50005B0731F4AA81BB816A177B0709F46FC188
:10FA6000A096B096A0E3CD3BDA0711F72091572B73
:10FA70002F732230D9F49093D51A8093D41A40E092
:10FA8000443090F4E42FF0E0EE0FFF1FE354FF4CFE
:10FA9000208131814F5F8217930791F71092D71A17
:10FAA00020E0C0E0D0E07EC04093D71A8091572B71
:10FAB00082FD54C484E18093572B88E290E09093B8
:10FAC0002F2B80932E2B80E58093562B8091512BEA
:10FAD0009091552B9093512B3091502B9091542B0A
:10FAE0009093502B3093542B20914F2B9091532B6C
:10FAF00090934F2B2093532B90914E2B9093D71A8A
:10FB00004091522B40934E2B9093522B8F5F8093BA
:10FB1000552B81110FC081E0830F8093542B8111ED
:10FB200009C081E0820F8093532B811103C09F5F36
:10FB30009093522B80914A2B90914B2B9093D51AF6
:10FB40008093D41A20914C2B30914D2B30934B2B1A
:10FB500020934A2B90934D2B80934C2B8091422BDA
:10FB60009091432BA091442BB091452B8093462B31
:10FB70009093472BA093482BB093492B8091CD3085
:10FB80009091CE30A091CF30B091D0308093422B65
:10FB90009093432BA093442BB093452BA1C33730B4
:10FBA00089F02F5F2430C0F430E2239FC00111247C
:10FBB000FC01E35CFF4C318D3111F1CF2093D71A5A
:10FBC000EF010CC0209721F0428D3A8D341748F791
:10FBD000EC01C35CDF4CE5CF2093D71A209709F4E2
:10FBE000BDC3D0933C30C0933B3083E08A8F888F75
:10FBF0001E8A84E08F8B1B8E80914C2B90914D2B15
:10FC00009D838C8380914A2B90914B2B9F838E8375
:10FC10008091422B9091432BA091442BB091452B86
:10FC200088839983AA83BB8381E0898F8091DA1AC4
:10FC30008C878091DB1A8D878091DC1A8E8780916A
:10FC4000DD1A8F8781E090E0998B888B8091512B12
:10FC50008B878091502B8A8780914F2B8987809149
:10FC60004E2B888781E090E00E9412828091562B73
:10FC7000282F207F30E0213531050CF445C08295D6
:10FC80008F7090E00597880F991F880F991F30910A
:10FC9000D61A20E0E22FF0E0E817F9078CF5EA5CCD
:10FCA000F44D30A5311105C02093D71A1092D61A01
:10FCB0002BC0313011F42F5FEDCF3230E1F441A58C
:10FCC0004430C9F42093D71A3093D61A82A590E015
:10FCD000982F882723A5822B9093D51A8093D41A26
:10FCE000893DA4E09A0710F088ED94E09B8B8A8B05
:10FCF0009D8B8C8B09C041A5442311F0240FCACFE2
:10FD00002093D71A3093D61A80E18093572B809195
:10FD1000572B82608093572B82E080935E2B84E088
:10FD200080935F2B8093602B88ED8093612B8CE216
:10FD300090E090932F2B80932E2B80E67EC2D09361
:10FD40003C30C0933B30109236309091572B92FF4D
:10FD500003C0198E80E21AC28091562B82958F7053
:10FD6000880F880F8093D71A081B110904511109B5
:10FD700010932F2B00932E2B8F2D8F70823029F410
:10FD8000892F8F73823139F41FC0813021F4892F7C
:10FD90008F738230C9F0012B19F4892F8370A1F081
:10FDA00020914E2B888528133EC220914F2B8985A8
:10FDB000281339C22091502B8A85281334C22091F0
:10FDC000512B8B8528132FC294FF4AC068897989EB
:10FDD0006115710509F444C0CE010C960E94127998
:10FDE0003091522B8091322B38133AC02091532BF3
:10FDF0008091332B281334C09091542B8091342B55
:10FE000098132EC08091552B4091352B841328C018
:10FE10003C872D879E878F878B8D81111AC02E89F5
:10FE2000888D9A8D891B922F969596959695891B0C
:10FE3000280F2E8B87FD81959F89392F3695369512
:10FE4000931B980F9F8B822F869586958695890F99
:10FE5000888F81E080933630888D8A8F198A188A3E
:10FE6000498D842F8F7090E0FC013197E830F105C7
:10FE700008F074C2E057FF4F0C94DD8B8091363050
:10FE800080FF14C083E0898F80E480933630198A24
:10FE9000188A80912E2B90912F2B009709F408C17E
:10FEA00022E4209336300E94128202C18091572BA7
:10FEB0008F73823009F052C227CF8091363080FF95
:10FEC00070C08091572B8F73823109F06AC0809186
:10FED000562B282F207F30E0213531050CF445C00A
:10FEE00082958F7090E00597880F991F880F991F52
:10FEF0003091D61A20E0E22FF0E0E817F9078CF5F0
:10FF0000EA5CF44D30A5311105C02093D71A109248
:10FF1000D61A2BC0313011F42F5FEDCF3230E1F41F
:10FF200041A54430C9F42093D71A3093D61A82A53C
:10FF300090E0982F882723A5822B9093D51A809341
:10FF4000D41A893D24E0920710F088ED94E09B8B51
:10FF50008A8B9D8B8C8B09C041A5442311F0240F03
:10FF6000CACF2093D71A3093D61A83E0898F809115
:10FF70004E2B888780914F2B89878091502B8A87C1
:10FF80008091512B8B8781E090E00E94128282E465
:10FF900080933630198A188A10922F2B10922E2BAC
:10FFA00087C080E2809336300E942775E0913B3015
:10FFB000F0913C30118E7ACD8091572B80FF28C074
:10FFC00044FD26C088899989892B09F0C7C1809191
:10FFD0002E2B90912F2B01960E9412822091363069
:10FFE000822F80618093363080912E2B90912F2B21
:10FFF000892B19F02261209336300E94277581E009
:020000021000EC
:1000000090E0998B888B88E0898F1B8E81E10CC1F1
:1000100085FF1CC080915C2B90E0982F8827209151
:100020005D2B822B2091393030913A30280F391FC7
:1000300030933A302093393020912E2B30912F2B52
:10004000281B390B30932F2B20932E2B80912E2B96
:1000500090912F2B009749F044FD07C02091363036
:100060002260209336300E9412828091582B90E0BB
:10007000982F88272091592B820F911D9093D51A84
:100080008093D41A2C893D892817390710F0892BC1
:1000900021F43093D51A2093D41A8091D41A9091D8
:1000A000D51A9B8B8A8B80913630837009F456C1A8
:1000B0001092D2301092D1300E9427758091363044
:1000C00085FF07C01092D2301092D130198E84E192
:1000D000ABC084FF0AC01092D2301092D13081E0C0
:1000E00090E0998B888B84E08FCF2091D130309134
:1000F000D23021153105E1F080FF02C0198A188A3B
:1001000088899989009781F48A899B898217930746
:1001100020F49093D2308093D1308091D13090915F
:10012000D230998B888B04C09093D2308093D13099
:100130001B8E8091302B9091312B90933A3080938D
:1001400039308091D1309091D230892B59F0888903
:100150009989009739F0889690932F2B80932E2BB6
:1001600088E10BC08091363081FFF8C088E290E0D2
:1001700090932F2B80932E2B80E18093572B5CC084
:100180008091363080FFEAC0198E80E1809336304E
:100190000E942775E3C080912E2B90912F2B009702
:1001A00011F00E9412829091572B8091363090FF6F
:1001B0000BC080FF06C087E0898F1A8E198A188AC3
:1001C00019C086E0898F16C080FF1EC085E0898F28
:1001D000198A188AC3C080912E2B90912F2B0097DB
:1001E00011F00E9412828091572B80FF0DC087E092
:1001F000898F1A8E81E090E00E94128280E18093C4
:1002000036300E9427750FC080912E2B90912F2B96
:10021000892B49F4A3C08091363080FF9FC087E0CE
:10022000898F1A8E9BC080E18093572B88E290E0E3
:1002300090932F2B80932E2B80E58093562B8885CF
:100240008093522B89858093532B8A858093542BDE
:100250008B858093552B8C8580934E2B8D85809339
:100260004F2B8E858093502B8F858093512B86E06A
:1002700080933F2B8C819D8190934B2B80934A2BB5
:100280008E819F8190934D2B80934C2B8091CD300C
:100290009091CE30A091CF30B091D0308093422B4E
:1002A0009093432BA093442BB093452B8881998145
:1002B000AA81BB818093462B9093472BA093482B18
:1002C000B093492B898D84FF05C01092592B109251
:1002D000582B06C084E08093582B88ED8093592BCF
:1002E00080E480933E2B80912E2B90912F2B909326
:1002F000382B8093392B10925D2B10925C2B10922F
:100300005B2B10925A2B0E94647980959095909364
:100310005B2B80935A2B85E48093362B1092372BDE
:1003200010923D2B10923C2B8091DE1A9091DF1A97
:1003300001969093DF1A8093DE1A90933A2B809364
:100340003B2B1092412B1092402B0E9453798095A9
:1003500090959093412B8093402B04C010922F2BAB
:1003600010922E2B10923630DF91CF911F910F916A
:10037000FF90EF90DF90CF90BF90AF9008959827B7
:100380008927982708950E94E38B0895FC018091A6
:10039000302B9091312B26E330E3281B390BAB0136
:1003A000261737070CF4A9011416150654F45093B8
:1003B000D2304093D130E817F90719F0BF010C94FF
:1003C0001290089580E880936100109261000E946D
:1003D00098600E9407520E9474648091DD28909179
:1003E000DE28009729F001979093DE288093DD287E
:1003F000C090DF28D090E028E090E128F090E2283B
:100400000E943263C616D706E806F90611F30E9469
:1004100032636093DF287093E0288093E128909303
:10042000E228D7CF20913B3030913C30BC01C9014C
:1004300008960E941279E0913B30F0913C30809117
:10044000322B80878091332B81878091342B828758
:100450008091352B838708952F923F924F925F9220
:100460006F927F928F929F92AF92BF92CF92DF92C4
:10047000EF92FF920F931F93CF93DF93CDB7DEB729
:1004800063970FB6F894DEBF0FBECDBF7C011B0192
:100490006A01FC0117821682838181FF66C3BE0157
:1004A0006F5F7F4F4B01F7019381F10193FD8591C0
:1004B00093FF81911F01882309F453C3853239F4D6
:1004C00093FD859193FF81911F01853239F4B70126
:1004D00090E00E94959056016501E5CF10E0512C07
:1004E00020E02032A0F48B3269F030F4803259F0F1
:1004F000833269F420612CC08D3239F0803339F4B5
:10050000216026C02260246023C0286021C027FD0E
:1005100027C030ED380F3A3078F426FF06C0FAE0F5
:100520001F9F300D1124132F13C06AE0569E300D0B
:100530001124532E20620CC08E3221F426FD11C3EB
:10054000206406C08C3611F4206802C0883641F45D
:10055000F10193FD859193FF81911F018111C1CF1D
:100560009BEB980F933018F42061805E06C09BE9E6
:10057000980F933008F0AAC12F7E26FF16E02F7344
:10058000722E853621F4F22FF0647F2E08C0863655
:1005900021F4622F6068762E02C01111115077FE8F
:1005A00007C01C3348F444244394410E27E00BC099
:1005B000183030F4212F06C027E04CE3442E03C04E
:1005C00027E017E0412C560174E0A70EB11CF6019C
:1005D0006081718182819381042DA4010E941A8F10
:1005E0006C01098100FF02C003FF06C071FC07C057
:1005F00072FC08C0612C08C03DE2632E05C02BE2EE
:10060000622E02C090E2692E802F8C7099F16620D4
:1006100011F084E001C083E0851510F0512C0BC06F
:10062000581A73FC08C0B70180E290E00E949590D0
:100630005A94C9F7F3CF662029F0B701862D90E0D0
:100640000E94959003FD03C008E910E102C004E98F
:1006500010E1F72DF0717F2EF8018491882309F4C1
:1006600076C271108052B70190E00E9495900F5FA2
:100670001F4FF2CF77FE0FC04C0C04FF04C08A81DD
:10068000813309F44A94141474F5F8E0F41578F5FC
:1006900088E0482E2CC076FC2AC0812F90E08C1573
:1006A0009D059CF06CEFC6166FEFD60674F0772DA3
:1006B0007068772E0AC0E2E0F0E0EC0FFD1FE10F5A
:1006C000F11D8081803319F411501111F4CF77FEA0
:1006D0000EC044244394410E812F90E0C816D906E1
:1006E0002CF41C1904C04424439401C010E077FE8C
:1006F00007C01C141D043CF496012F5F3F4F05C03A
:1007000025E030E002C021E030E0662011F02F5FEC
:100710003F4F112331F0412F50E04F5F5F4F240FC7
:10072000351F452D50E02417350714F4521A01C027
:10073000512C872D897049F4552039F0B70180E29A
:1007400090E00E9495905A94F7CF662029F0B70167
:10075000862D90E00E94959073FC09C0552039F0D9
:10076000B70180E390E00E9495905A94F7CF77FE0E
:100770005FC09C2D8D2DD7FE02C090E080E0692ED9
:10078000782E40E050E0C601841991099D878C873E
:10079000960126193709280D391D812F90E0EE2783
:1007A000FF27E81BF90BFF87EE87FFEF6F167F0629
:1007B00069F4B7018EE290E02B8B3A8B488B598B12
:1007C0000E949590598948893A892B89C614D70483
:1007D00054F06C857D85661577052CF4F901E40FDE
:1007E000F51F818101C080E371E0671A71084F5FD6
:1007F0005F4FEE85FF856E167F066CF0B70190E0C7
:100800002B8B3A8B488B598B0E9495902B893A8978
:1008100048895989CACF6C147D0439F49A8196337A
:1008200018F4953311F404FF81E3B70190E04BC055
:100830008A81813309F00F7EB70190E00E94959084
:10084000111105C074FE18C085E490E017C0B7010F
:100850008EE290E00E94959082E066246394680E98
:10086000F401E80FF11D8081B70190E00E9495909E
:10087000115041F3862DF1CF85E690E0B7010E943B
:100880009590D7FC05C0C114D10439F404FF05C00C
:10089000D194C194D1088DE201C08BE2B70190E000
:1008A0000E94959080E36AE0C616D1042CF08F5F19
:1008B000FAE0CF1AD108F7CFB70190E00E949590E7
:1008C000B701C601C0960E94959041C1833631F0B0
:1008D000833779F0833509F058C021C0560172E0A2
:1008E000A70EB11CF6018081898301E010E064014C
:1008F00014C05601F2E0AF0EB11CF601C080D180E9
:1009000026FF03C0612F70E002C06FEF7FEFC601CA
:100910002B8B0E9441908C012B892F7715C056019B
:10092000F2E0AF0EB11CF601C080D18026FF03C0FB
:10093000612F70E002C06FEF7FEFC6012B8B0E942A
:1009400003908C012B892068722E23FD1AC0852DFF
:1009500090E008171907A8F4B70180E290E00E9420
:1009600095905A94F4CFF60177FC859177FE8191AA
:100970006F01B70190E00E94959051105A94015078
:1009800011090115110579F7E2C0843611F0893695
:1009900051F5560127FF09C0F4E0AF0EB11CF60176
:1009A00060817181828193810AC0F2E0AF0EB11C37
:1009B000F60160817181882777FD8095982F022F3D
:1009C0000F7697FF08C090958095709561957F4F41
:1009D0008F4F9F4F00682AE030E0A4010E94CF9122
:1009E000C82EC8183EC0022F853721F40F7E2AE09A
:1009F00030E01DC0097F8F3691F018F4883559F02A
:100A0000B0C0803719F0883711F0ABC0006104FF27
:100A100009C0046007C024FF08C0066006C028E0C3
:100A200030E005C020E130E002C020E132E05601B4
:100A300007FF09C0F4E0AF0EB11CF60160817181BF
:100A40008281938108C0F2E0AF0EB11CF601608193
:100A5000718180E090E0A4010E94CF91C82EC81857
:100A60000F7706FF0BC0202F2E7FC11650F404FF16
:100A70000AC002FD08C0202F2E7E05C0DC2C202FCE
:100A800003C0DC2C01C0D12E24FF0DC0FE01EC0DF3
:100A9000F11D8081803311F4297E09C022FF06C038
:100AA000D394D39404C0822F867809F0D39423FD85
:100AB00013C020FF06C01C2DD51418F4150D1D19E8
:100AC000D52CD51468F4B70180E290E02B8B0E94FE
:100AD0009590D3942B89F5CFD51410F45D1801C0EF
:100AE000512C24FF12C0B70180E390E02B8B0E94B1
:100AF00095902B8922FF17C021FF03C088E590E065
:100B000002C088E790E0B7010CC0822F867859F0C8
:100B100021FD02C080E201C08BE227FD8DE2B7011A
:100B200090E00E949590C11638F4B70180E390E000
:100B30000E9495901150F7CFCA94F401EC0DF11D6D
:100B40008081B70190E00E949590C110F5CF5520AB
:100B500009F4C2CCB70180E290E00E9495905A94CB
:100B6000F6CFF7018681978102C08FEF9FEF6396E2
:100B70000FB6F894DEBF0FBECDBFDF91CF911F91AE
:100B80000F91FF90EF90DF90CF90BF90AF909F902C
:100B90008F907F906F905F904F903F902F9008952F
:100BA0005058BB27AA270ED04EC23FD230F044D2B5
:100BB00020F031F49F3F11F41EF4FFC10EF4E095D4
:100BC000E7FBF5C1E92F50D280F3BA17620773072C
:100BD0008407950718F071F49EF568C20EF4E0954D
:100BE0000B2EBA2FA02D0B01B90190010C01CA01E7
:100BF000A0011124FF27591B99F0593F50F4503E92
:100C000068F11A16F040A22F232F342F4427585F83
:100C1000F3CF469537952795A795F0405395C9F79B
:100C20007EF41F16BA0B620B730B840BBAF0915053
:100C3000A1F0FF0FBB1F661F771F881FC2F70EC0F2
:100C4000BA0F621F731F841F48F4879577956795C5
:100C5000B795F7959E3F08F0B3CF9395880F08F0AE
:100C60009927EE0F979587950895DFD158F080E882
:100C700091E009F49EEFE0D128F040E851E059F40A
:100C80005EEF09C09AC112C2E92FE078EDD168F396
:100C9000092E052AC1F3261737074807590738F0E8
:100CA0000E2E07F8E02569F0E025E0640AC0EF6346
:100CB00007F8009407FADB01B9019D01DC01CA01C4
:100CC000AD01EF9347D0BFD10AD05F91552331F0EA
:100CD0002BED3FE049E450FD49EC63CF0895DF93ED
:100CE000DD27B92FBF7740E85FE3161617064807E0
:100CF0005B0710F4D92FE1D19F938F937F936F936C
:100D000046D3E0E3F1E06CD19ED12F913F914F911A
:100D10005F919AD2DD2349F09058A2EA2AED3FE094
:100D200049EC5FE3D0785D274DDFDF918CC11BD1AB
:100D300008F481E008950CD086C17ED140F075D1D1
:100D400030F021F45F3F19F032C15111B0C135C10B
:100D50008BD198F39923C9F35523B1F3951B550B08
:100D6000BB27AA2762177307840738F09F5F5F4F7E
:100D7000220F331F441FAA1FA9F333D00E2E3AF0BF
:100D8000E0E830D091505040E695001CCAF729D0D9
:100D9000FE2F27D0660F771F881FBB1F2617370728
:100DA0004807AB07B0E809F0BB0B802DBF01FF2758
:100DB00093585F4F2AF09E3F510568F0F8C077C105
:100DC0005F3FECF3983EDCF3869577956795B79592
:100DD000F7959F5FC9F7880F911D9695879597F9AD
:100DE0000895E1E0660F771F881FBB1F6217730726
:100DF0008407BA0720F0621B730B840BBA0BEE1F3B
:100E000088F7E095089519F40EF0D1C04FC1D5C010
:100E100033D1C8F39638C0F707F80F92E8942BE364
:100E20003AEA48EB5FE712D20F920F920F924DB75A
:100E30005EB70F92CAD1EDE5F1E0D2D04F915F914C
:100E4000EF91FF91E595EE1FFF1F49F0FE57E06817
:100E50004427EE0F441FFA95E1F74195550B36D123
:100E60000F9007FE2AC1089597FB0EF4A9D03EC04B
:100E7000E89409C097FB3EF4909580957095619534
:100E80007F4F8F4F9F4F9923A9F0F92F96E9BB27EA
:100E90009395F695879577956795B795F111F8CF66
:100EA000FAF4BB0F11F460FF1BC06F5F7F4F8F4FD1
:100EB0009F4F16C0882311F096E911C0772321F0C7
:100EC0009EE8872F762F05C0662371F096E8862F5F
:100ED00070E060E02AF09A95660F771F881FDAF7B6
:100EE000880F9695879597F90895E894F92F96EBD2
:100EF000FF2381F0121613061406440B9395F69502
:100F000087957795679557954040FF23B9F71BC0A4
:100F100099270895882351F49850D2F7872B762F7C
:100F2000652F542F432F322F20E0B1F312161306F2
:100F30001406440B88233AF09A95440F551F661FF8
:100F4000771F881FCAF755234AF4440F551F11F421
:100F500060FF04C06F5F7F4F8F4F9F4F880F969544
:100F6000879597F90895990F0008550FAA0BE0E8A7
:100F7000FEEF16161706E807F907C0F0121613065B
:100F8000E407F50798F0621B730B840B950B39F49B
:100F90000A2661F0232B242B252B21F408950A2601
:100FA00009F4A140A6958FEF811D811D089597F941
:100FB0009F6780E870E060E008959FEF80EC0895FF
:100FC00090958095709560955095409530952195B8
:100FD0003F4F4F4F5F4F6F4F7F4F8F4F9F4F089542
:100FE000DF93CF931F930F93FF92EF92DF927B01DA
:100FF0008C01689405C0DA2EEF0126D1FE01E89439
:10100000A5912591359145915591AEF3EF01DADD2A
:10101000FE019701A801DA9479F7DF90EF90FF9035
:101020000F911F91CF91DF91089500240A94161615
:10103000170618060906089500240A9412161306C6
:10104000140605060895092E0394000C11F4882354
:1010500052F0BB0F40F4BF2B11F460FF04C06F5F70
:101060007F4F8F4F9F4F089557FD9058440F551F46
:1010700059F05F3F71F04795880F97FB991F61F01A
:101080009F3F79F087950895121613061406551F91
:10109000F2CF4695F1DF08C0161617061806991FFD
:1010A000F1CF86957105610508940895E894BB27F2
:1010B00066277727CB0197F908959B01AC0160E083
:1010C00070E080E89FE337CE72CF64C1D5DFE8F3EC
:1010D0009923D9F3940F511DBBF39150504094F0D4
:1010E00059F0882332F0660F771F881F91505040C7
:1010F000C1F79E3F510544F7880F911D969587953E
:1011000097F908955F3FACF0983E9CF0BB27869519
:1011100077956795B79508F4B1609395C1F7BB0FC4
:1011200058F711F460FFE8CF6F5F7F4F8F4F9F4FED
:10113000E3CFBDCF0AD029ED3BE54EED5EE378C0AD
:101140000EF028C13ACF689432CF96DFC8F39923C6
:10115000D1F3C6F3DF93CF931F930F93FF92C92F61
:10116000DD2788232AF02197660F771F881FDAF77B
:1011700020E030E040E85FEB9FE3883920F0803EDC
:1011800030F021968F770DDDE5E8F1E003C009DD51
:10119000E2EBF1E025DF8B01BE01EC01FB2E6F5786
:1011A00071097595771F880B990B64DE28E132E78A
:1011B00041E35FE349D0AF2D9801AE01FF900F915D
:1011C0001F91CF91DF91FEDC3ECFFA01DC01AA0F27
:1011D000BB1F9B01AC01BF5728F4222733274427AC
:1011E00050781FC0B75188F4AB2F0024469537952F
:1011F0002795011CA395D2F3002069F0220F331F1D
:10120000441FB395DAF30DD0CBCC61307105A0E863
:101210008A07B94630F49B01AC01662777278827F7
:101220009078309621F02083318342835383089550
:101230000BD009CFFADE28F0FFDE18F0952309F075
:10124000B6CEBBCE112433CF0FDFA0F3959FD1F3E1
:10125000950F50E0551F629FF001729FBB27F00D64
:10126000B11D639FAA27F00DB11DAA1F649F6627B9
:10127000B00DA11D661F829F2227B00DA11D621F08
:10128000739FB00DA11D621F839FA00D611D221FC2
:10129000749F3327A00D611D231F849F600D211DA6
:1012A000822F762F6A2F11249F5750408AF0E1F049
:1012B00088234AF0EE0FFF1FBB1F661F771F881F92
:1012C00091505040A9F79E3F510570F070CEEFCE7F
:1012D0005F3FECF3983EDCF3869577956795B7957D
:1012E000F795E7959F5FC1F7FE2B880F911D9695A7
:1012F000879597F90895FA01EE0FFF1F30962105A3
:10130000310599F16115710561F48038BFE39B07E0
:1013100049F168949038810561F08038BFEF9B07F0
:1013200041F0992342F5FF3FE1053105210511F117
:10133000E8940894E795D901AA2329F4AB2FBE2F8E
:10134000F85FD0F310C0FF5F70F4A695E0F7F739AF
:1013500050F019F0FF3A38F49F779F930CD00F901C
:1013600007FC905808953EF028CE60E070E080E8D9
:101370009FE308954FE79F775F934F933F932F939A
:10138000E4DE2F913F914F915F9152DF41CD9B0160
:10139000AC014ECF9F3F31F0915020F48795779567
:1013A0006795B795880F911D9695879597F908953C
:1013B0000E94E089332312F48A1B9B0B0C94F18961
:1013C000A29FB001B39FC001A39F700D811D112486
:1013D000911DB29F700D811D1124911D08950E94D1
:1013E000E089B7FF0895821B930B08950E94E0895E
:1013F000A59F900DB49F900DA49F800D911D112469
:101400000895B7FF0C94F6890E94F689821B930B0E
:101410000895DB018F939F930E94F689BF91AF914E
:10142000A29F800D911DA39F900DB29F900D11243E
:101430000895AA1BBB1B51E107C0AA1FBB1FA6171B
:10144000B70710F0A61BB70B881F991F5A95A9F76D
:1014500080959095BC01CD01089597FB072E16F459
:10146000009407D077FD09D00E94198A07FC05D0A7
:101470003EF4909581959F4F0895709561957F4FAB
:101480000895A1E21A2EAA1BBB1BFD010DC0AA1FC5
:10149000BB1FEE1FFF1FA217B307E407F50720F0DD
:1014A000A21BB30BE40BF50B661F771F881F991F58
:1014B0001A9469F760957095809590959B01AC01A1
:1014C000BD01CF010895052E97FB1EF400940E94E4
:1014D0008E8B57FD07D00E94418A07FC03D04EF443
:1014E0000C948E8B50954095309521953F4F4F4FE2
:1014F0005F4F0895689401C0E894F92FF12B12F022
:101500000C94AE8AA0E0B0E0E8E8FAE80C94AC8B6A
:10151000092E059422F40E94968B112392F4F0E890
:101520000F26FFEFE094F09400951095B094C094CE
:10153000D094A194BF0ACF0ADF0AEF0AFF0A0F0B6B
:101540001F0B0E943D8B07FC0E94968BCDB7DEB728
:10155000ECE00C94C88B689401C0E8948F929F9241
:10156000CF93DF930E943D8BDF91CF919F908F901F
:101570000895DF93CF931F930F939A9DF02D219F92
:10158000F00D8B9DF00D8A9DE02DF10D039FF00D68
:10159000029FE00DF11D4E9DE00DF11D5E9DF00DD1
:1015A0004F9DF00D7F936F93BF92AF925F934F93D8
:1015B000D5010E94E0898B01AC01D7010E94E0892E
:1015C000EB01E80FF91FD6010E94098B2F913F9183
:1015D000D6010E94E089C60FD71FE81FF91FAF91FF
:1015E000BF910E94098B2F913F910E94E089C60F05
:1015F000D71FE81FF91FD6010E94E089E60FF71FE9
:101600009801BE01CF0111240F911F91CF91DF915D
:1016100008950E94E089460F571FC81FD91F08F47C
:1016200031960895E894DF93CF93FC01DB010E948B
:10163000E0897F936F93E9019A01AC01BF93AF9367
:101640003F932F93DF010E94E08926F46C1B7D0BF2
:10165000820B930B9E01EB01FC010E94098BAF9161
:10166000BF912F913F910E94098BBE01CF01F901DB
:101670002F913F91CF91DF91089588249924F4010F
:10168000E401B0E49F93AA279A158B049C04ED050E
:10169000FE05CF05D007A10798F4AD2FDC2FCF2F83
:1016A000FE2FE92D982C892E982F872F762F652FC6
:1016B000542F432F322F2227B85031F7BF9127C024
:1016C0001B2EBF91BB27220F331F441F551F661FC0
:1016D000771F881F991F881C991CEE1FFF1FCC1FA6
:1016E000DD1FAA1FBB1F8A149B04EC05FD05CE0558
:1016F000DF05A007B10748F08A189B08EC09FD092F
:10170000CE09DF09A00BB10B21601A94E1F62EF48B
:101710009401AF01BE01CD01000C08959095809514
:10172000709561957F4F8F4F9F4F0895609570958D
:101730008095909530954095509521953F4F4F4F0E
:101740005F4F6F4F7F4F8F4F9F4F08952F923F9264
:101750004F925F926F927F928F929F92AF92BF92C1
:10176000CF92DF92EF92FF920F931F93CF93DF936D
:10177000CDB7DEB7CA1BDB0B0FB6F894DEBF0FBECA
:10178000CDBF09942A88398848885F846E847D8417
:101790008C849B84AA84B984C884DF80EE80FD8019
:1017A0000C811B81AA81B981CE0FD11D0FB6F8948F
:1017B000DEBF0FBECDBFED010895EE0FFF1F0590F8
:1017C000F491E02D099469279627692778278727C0
:1017D000782708950F93083090F0982F872F762F51
:1017E000652F542F432F322F22270850F4CF220F7A
:1017F000331F441F551F661F771F881F991F0A95A7
:10180000B2F70F91089597FB10F8169400080F9304
:10181000083098F00850232F342F452F562F672F6C
:10182000782F892F902DF4CF0594979587957795EC
:10183000679557954795379527950A95AAF70F917C
:1018400008952A0D3B1D4C1D5D1D6E1D7F1D801FC3
:10185000911F08950024A7FD00942A0F301D401DFC
:10186000501D601D701D801D901D08952A193B0993
:101870004C095D096E097F09800B910B08952A15AB
:101880003B054C055D056E057F05800791070895B2
:101890000024A7FD00942A17300540055005600577
:1018A00070058005900508958F929F92AF92BF9228
:1018B000CF92DF92EF92FF92CF93DF93EC0168819A
:1018C00079818A819B81611571058105910521F4DA
:1018D00064E279ED8BE597E02DE133EF41E050E0F4
:1018E0000E94638A49015A019B01AC01A7EAB1E455
:1018F0000E94F6896B017C01ACEEB4EFA501940166
:101900000E94048AC60ED71EE81EF91EF7FE06C006
:1019100081E0C81AD108E10880E8F80AC882D982B3
:10192000EA82FB82C6019F77DF91CF91FF90EF9013
:10193000DF90CF90BF90AF909F908F9008950C94C0
:10194000548C82EE92E00C94548CA0E0B0E0809332
:10195000E2029093E302A093E402B093E5020895BB
:101960002F923F925F926F927F928F929F92AF924F
:10197000BF92CF92DF92EF92FF920F931F93CF937C
:10198000DF938B01EA016115710521F0DB018C9376
:1019900011969C93209739F09E01225031092332F1
:1019A000310508F0FBC07C016701BFEFCB1ADB0AF1
:1019B0005601F7016080862D90E00E94F28F892BFE
:1019C00011F07601F1CFFDE26F120AC0570182E0FB
:1019D000A80EB11CD70111966C90772473940BC09C
:1019E000BBE26B1207C05701E2E0AE0EB11CD7019B
:1019F00011966C90712CCE018F7E892B89F4B0E307
:101A00006B1222C0F50180818F7D883541F56180A0
:101A1000F2E0AF0EB11C872D8260782EC0E1D0E0DD
:101A2000C830D105F1F04CF4C230D10511F5C12C0C
:101A3000D12CE12CB0E4FB2E2FC0CA30D10531F0FF
:101A4000C031D10521F115C0209751F7CAE0D0E08F
:101A5000ACECCA2EDC2CEC2CACE0FA2E1DC020978E
:101A6000F9F6C8E0D0E0C12CD12CE12CF0E1FF2E3A
:101A700013C060E070E080E090E89E01442737FDED
:101A80004095542F0E94418A69017A0105C0C12CFA
:101A9000D12CE12CE8E0FE2EF50160E020E030E002
:101AA000A9014E01AA2497FCA094BA2C1F0170ED45
:101AB000572E560CA9E0A51570F48FEB860D8A31D0
:101AC00018F499EC592E06C08FE9860D8A3130F54D
:101AD00089EA582E560C852D90E08C179D07F4F45A
:101AE00067FD18C0C216D306E406F50680F0C501EE
:101AF000B4010E94098A9B01AC01250D311D411DD5
:101B0000511D213031054105B0E85B0710F06FEF42
:101B100001C061E03196D1016C90C8CF872D8170F2
:101B20000115110571F0662329F03197D801ED9365
:101B3000FC9307C071FE19C03297D801ED93FC9356
:101B400014C067FF12C0882329F020E030E040E095
:101B500050E804C02FEF3FEF4FEF5FE782E290E0E5
:101B600090935C3180935B3116C0882341F050958F
:101B70004095309521953F4F4F4F5F4F0CC057FF19
:101B80000AC082E290E090935C3180935B312FEF4A
:101B90003FEF4FEF5FE7B901CA0104C060E070E0BA
:101BA00080E090E0DF91CF911F910F91FF90EF9037
:101BB000DF90CF90BF90AF909F908F907F906F906D
:101BC0005F903F902F9008952F923F925F926F9277
:101BD0007F928F929F92AF92BF92CF92DF92EF92BD
:101BE000FF920F931F93CF93DF938B01EA0161154F
:101BF000710521F0DB018C9311969C93209739F0AD
:101C00009E01225031092332310508F0D8C07C01F1
